:020000040000FA
:1000000092EF01F01200FFFF10EF04F01200FFFF6B
:1000100000000901C80E926F66806650010B06E071
:100020000901925103E009019207F7D7120000007D
:100030000901C80E926F66846650040B06E0090140
:10004000925103E009019207F7D71200D9CFE6FFDA
:10005000E1CFD9FF3F0E6816676A666AFE0EDB5075
:100060006712FD0EDB506812678AE552E7CFD9FFB1
:100070001200D9CFE6FFE1CFD9FFFE0EDB506A6E4A
:1000800067AE02D0FF0E30D00F0E671408080CE0E8
:100090000F0E67140B0808E06850040B03E168506A
:1000A000010B1FE0000E20D00F0E6714080804E0BB
:1000B0000F0E67140B0818E10901C80E926F685003
:1000C000010B04E0925102E09207F9D76850040B4B
:1000D00001E0010E496E1F0E66144910F7E166AC8F
:1000E00002D0FE0E01D0000EE552E7CFD9FF12007C
:1000F000D9CFE6FFE1CFD9FF0000FE0EDBCFE6FF50
:10010000B8DFE552006E005003E091DF005000D0F0
:10011000E552E7CFD9FF120000007ADF700EE66EDD
:10012000E7DFE552000901E028D0800EE66EE0DF4F
:10013000E552000901E021D0E66ADADFE552000964
:1001400001E01BD0400EE66ED3DFE552000901E06E
:1001500014D0016A1E0E015C0FE20150EA6A000F22
:10016000E96E060EEA22EF50E66EC2DFE5520009A4
:1001700001E003D0012AEED75ADF12000000016A25
:100180001E0E015C09E20150EA6A000FE96E060EDC
:10019000EA22EF68012AF4D712000000016A1E0E5D
:1001A000015C09E20150EA6A000FE96E060EEA22DC
:1001B000EF6A012AF4D712000000EFDFE66A080EAA
:1001C000E66E44DFE552E552090E696E21DF700EDE
:1001D000E66E8EDFE552000901E01CD0800EE66E6F
:1001E00087DFE552000901E015D0C80EE66E80DF1A
:1001F000E552000901E00ED0E66A7ADFE552000917
:1002000001E008D0E00EE66E73DFE552000901E080
:1002100001D00DDF12000000CFDF0601050E026FD6
:100220000601340E036F0601460E146F0601050E1B
:10023000176F0601040E186F0601640E196F060190
:10024000010E1A6F0601670E1B6F0601020E1C6F6E
:100250000601600E1D6F60DF1200000037D836D82F
:100260008D8A8D8C84848C80120009018E6B09012B
:100270008A07000E8B5B09018D5109018C5D04E03A
:1002800084948C908D9A8D9C8E2FFED709018D5170
:1002900009018C5D06E009018CB18C8009018CB3E9
:1002A00084848E2FFED78CC98DF9120000000900BE
:1002B000F5CF89F90900F5CF88F9090188510901BD
:1002C00086270901895109018723120000000901CD
:1002D000886B896B0901540E885D3D0E895905E2D2
:1002E0000901882B000E8923F5D7120000000901AF
:1002F000886B896B0901220E885D060E895905E21B
:100300000901882B000E8923F5D7120000008250C6
:10031000010B03E08250020B02E1010E02D0000E3D
:1003200000D01200C16A0F01DF0E256F0F01F70E1A
:10033000246F0F01E00E236F3A0EC06EEF0E896E30
:100340008A6A8B6A9E0E8C6E900E8D6E8E6A8F6A94
:10035000010E906E916AEF0E926E070E936E930EE1
:10036000946E600E956E030E966E7F0E976E060E5F
:10037000986EFE0E996E9A688A8AC79EC698C78C38
:10038000F00EC616C680C68A240EAC6E190EAF6E6D
:10039000900EAB6EF29EA698636AFE0E626E010E20
:1003A000616E7F9E7F9C7F84550E7E6EAA0E7E6E50
:1003B0007F82F28E01DFB0DE50DF0901916BA6DF94
:1003C000000904E10A0E0901915D09E2640E0901C8
:1003D000915D05E27BDF7ADF0901912BF0D77F94F5
:1003E00009019151630802E216EF02F00901866BE0
:1003F000876BF66A080EF76EF86A58DF000009018D
:100400008851891102E102EF04F050DF800EF618E6
:1004100005E1FD0EF71802E1010EF81801E0F5D72D
:1004200009018651871102E102EF04F001D81200A0
:10043000F2DE09018C6B09018BA703D00901010EC3
:100440008C6F13DF9EAA17D0AECF8FF9490E09012A
:100450008F5D0AE14B0EAD6E49DF580EAD6E46DF83
:10046000330EAD6E43DF02D08FC9ADFF440E0901DC
:100470008F5D01E101D0DDD709018A6B8B6B09012A
:10048000020E8C6F09018AA902D009018C6BEDDE86
:100490002FD8020EF85C05E1420EAD6EF86A0ED858
:1004A000FF000CD8410EAD6EEAD712000000550EC9
:1004B0007E6EAA0E7E6E7F8200001200940E7F6E0A
:1004C000F5DF000EE96E090EEA6E0A000901100E52
:1004D000846F0901080E856FEE50F56E0F00852FB1
:1004E000FBD7840E7F6EE2DF842FF3D77F94120058
:1004F00000000901906B0901846B09018451496E68
:100500004A6AD8904A5004E6840E495C000E4A5864
:1005100014E29EAAFED7AECF8FF909018451EA6A90
:10052000000FE96E090EEA228FC9EFFF09018F5112
:10053000090190270901842BE0D7090190510BE1B3
:10054000030E0901825D07E280C9F6FF81C9F7FF4A
:1005500082C9F8FF03D04E0EAD6ECBD71200FFFF5D
:10056000FFFFFFFFFFFFFFFFFFFFFFFFFFFFFFFF9B
:10057000FFFFFFFFFFFFFFFFFFFFFFFFFFFFFFFF8B
:10058000FFFFFFFFFFFFFFFFFFFFFFFFFFFFFFFF7B
:10059000FFFFFFFFFFFFFFFFFFFFFFFFFFFFFFFF6B
:1008000000001200280EE66E4CECFEF0E552EAEF16
:10081000FDF01200FFFFFFFFFFFFFFFFFFFFFFFFE5
:1008200048EF24F01200FFFFFFFFFFFFFFFFFFFF75
:100830000000E7ECC9F0DC0E496EDB0E4A6E010EDB
:1008400091EFD5F0E7ECC9F0430E496EDC0E4A6E2D
:10085000010E91EFD5F0E7ECC9F0280E4B6EDD0EDE
:100860004C6E010E4D6EFE0EDBCF4EF0EFECCBF07A
:10087000B0ECD9F0E3EFC9F0E7ECC9F0B10E496E86
:10088000DA0E4A6E010E91EFD5F0E7ECC9F09C0E3E
:10089000496EDA0E4A6E010E91EFD5F0E7ECC9F021
:1008A000110E496ECE0E4A6E010E91EFD5F085EC19
:1008B000D5F0050D23ECD6F00A0E49260A0E4A2281
:1008C000FD0EDB504924E96E000E4A20EA6EEF501F
:1008D000E3EFC9F02EC1E6FFBEDFE5521200350E90
:1008E000012411EFD4F0E7ECC9F03A0E496ECF0EB7
:1008F0004A6E010E91EFD5F09DEFCFF045ECD2F0AE
:100900004AEFDBF000ECD5F04AEFDBF0E80E496E81
:10091000030E4A6E4AEFDBF0010155513C0DF3CF57
:1009200016F2F4CF17F2120000ECD5F037C23DF00A
:1009300038C23EF0B5EFDAF0E66AFFEC26F0E55299
:100940001200010E9FEFCAF0020E9FEFCAF087C29D
:10095000E6FFF6EFD8F0E66AF6EFD8F001018AB7C5
:100960003B0C300CF7ECD1F019E3FFECD6F002E6CB
:1009700016ECD4F013E2F7ECD1F010E3FFECD6F074
:1009800002E616ECD4F00AE2F7ECD1F007E3FFEC54
:10099000D6F002E616ECD4F001E2010C000C020ED7
:1009A0000101805D0BE2805102E0010E01D0000EDA
:1009B000E8B08A88E8B003D08A9801D08A98070EF8
:1009C000936EF18E8051010803E2F19E170E936E33
:1009D00012002150100B08E0640E02010B5D04E3CD
:1009E000A1ECCBF001E02198120004ECD5F001015C
:1009F000AC6BB59F1200020E0101805D03E18150D6
:100A0000100B06E0030E805D04E18150100B01E045
:100A1000000C010CF0DF000901E1000C010156A1FE
:100A2000010CD70E1CECDAF01E0803E2F00E005C9D
:100A300001E3000C010C7A0EE66EE40EE66E010E88
:100A400012ECCAF0DCECD2F006E1BDECD0F003E031
:100A500001011E0EAC6F66C100F05EECCFF00A0E15
:100A6000665D02E2200E1A6F1200730EE66EE40E4F
:100A7000E66E010E12ECCAF0DCECD2F006E1BDEC41
:100A8000D0F003E001011E0EAC6F67C100F0005012
:100A90000FE00101030E016F9DECE1F001012D0E4D
:100AA000196F0A0E675D04E2200E196F2D0E1A6F82
:100AB00012006C0EE66EE40EE66E010E12ECCAF049
:100AC00068C100F000500AE00101030E016F5EEC06
:100AD000CFF00A0E685D02E2200E1A6F12000101CB
:100AE00048511200800E071403E02050010B01E072
:100AF000000C010C800E071406E02050010B03E1EE
:100B00000201215101E0000C010C0201010E3A6FBB
:100B10007E0E00ECCBF001011E0EAC6F120033EF25
:100B2000D3F085ECD5F004080FE00AECCBF00EE032
:100B3000FE0EDB500A0808E0FE0EDB500D0804E054
:100B4000FE0EDB50090802E1010E01D0000EE3EFBA
:100B5000C9F007019551D880945502E294C795F7E2
:100B600094079251922BEA6A000FE96E0C0EEA226A
:100B7000EF5012000101E651100B03E00401FA519D
:100B80000AE1420EE66E460EE66E70ECA1F0E5520A
:100B9000E5520101E6891200D9CFE6FFE1CFD9FF86
:100BA000FE0EDB50D80805E1300EF36EFE0EF3CFDB
:100BB000DBFF060EAB1406E0AB980000000000005F
:100BC000AB8840D1FE0EDB50100805E0FE0EDB5076
:100BD000110801E037D10201050E146FFE0EDB5043
:100BE000110837E1020124510DE12050800B0AE188
:100BF000050105014751010B0AE1050105014751B6
:100C0000400B05E1100EE66E8FD9E55222D00501AA
:100C100005014751400B02E00F0E01D0060EE66EB3
:100C200083D9E552C4C1E6FF7FD9E552C5C1E6FFCD
:100C30007BD9E552C6C1E6FF77D9E5520A0E01011C
:100C4000C703F3500101C825E66E6ED9E5520501D0
:100C500047910401F051496E4A6A4A3404E249500E
:100C6000D208000E4A5405E20701042B07010407CD
:100C7000E9D00501475104E10501485101E1E2D005
:100C80000201245101E0DED02050800B01E0DAD0D7
:100C90000490050148A10BD04E0EE66E420EE66EA2
:100CA00070ECA1F0E552E5520501486BCBD005018F
:100CB00047A11AD001010101E651080B03E004012C
:100CC000FA510DE1410EE66E460EE66E70ECA1F0B3
:100CD000E552E5520101E687050147B34BDF050107
:100CE000479305014791AED0050147A304D042DFE9
:100CF00005014793A7D0050147A726D0440EE66E0D
:100D00004D0EE66E70ECA1F0E552E5520480440E03
:100D1000E66E4D0EE66E70ECA1F0E552E552030E64
:100D20000101D45D04E0030E0101D55D08E1540E1C
:100D3000E66E440EE66E70ECA1F0E552E552050158
:100D40004797050147857ED0050147A524D0570E5A
:100D5000E66E420EE66E70ECA1F0E552E5520480BC
:100D6000570EE66E420EE66E70ECA1F0E552E552CB
:100D7000530EE66E490EE66E70ECA1F0E552E552B8
:100D80004A0EE66E460EE66E70ECA1F0E552E552B4
:100D90000501479557D0050147A90BD0410EE66ED6
:100DA000500EE66E70ECA1F0E552E5520501479950
:100DB00049D0050147AB0BD0410EE66E520EE66EF0
:100DC00070ECA1F0E552E5520501479B3BD00501CF
:100DD00047AD13D04F0EE66E520EE66E70ECA1F0EA
:100DE000E552E552540EE66E520EE66E70ECA1F03E
:100DF000E552E5520501479D25D0050147AF22D0B8
:100E00004E0EE66E4C0EE66E70ECA1F0E552E55229
:100E1000560EE66E440EE66E70ECA1F0E552E55219
:100E2000420EE66E530EE66E70ECA1F0E552E5520E
:100E3000570EE66E430EE66E70ECA1F0E552E552F9
:100E40000501479F200EF36EFE0EDBCFF4FFF3503B
:100E5000F45C04E3FE0EDB507E0807E2FE0EDBCFFF
:100E6000E6FF5FDEE552000944E00401F051496EFF
:100E70004A6AD8904A5004E6FF0E495C000E4A5870
:100E800038E2FE0EDB503B0804E0FE0EDB507C082F
:100E900002E10401F92BFE0EDB50210804E0FE0EF6
:100EA000DB5040080AE13B0E0401FE5D04E07C0ECD
:100EB0000401FE5D02E10401F92BFE0EDBCFFEF41E
:100EC0000401F151EA6A000FE96E0B0EEA22FE0EF0
:100ED000DBCFEFFF0401F12B0401F02B0401F051F3
:100EE00008E10401FE6BFEC4F9F4FEC4F1F4FEC493
:100EF000F2F4E552E7CFD9FF1200ACA212000401D0
:100F0000F8515FECD6F0006E0050E66E3AECCFF090
:100F100000C0EFFF3B0E005C03E07C0E005C01E1D3
:100F200029900401F82B1200E7ECC9F0ACA2FED71F
:100F300095ECD5F03AECCFF0FE0EDBCFEFFFE3EF10
:100F4000C9F0CCEC10F0010EE66EE1EC10F0E552C9
:100F500084948C908D9A8D9CF29E0000F66A080E07
:100F6000F76EF86A940E7F6E550E7E6EAA0E7E6E38
:100F70007F82000000EC00F012000401F007F25143
:100F8000EA6A000FE96E0B0EEA22EF50006EF22BB8
:100F90001200BDECCAF00AE11F50020B07E102018A
:100FA0008951020B04E18951010B01E1000C010C94
:100FB000D9CFE6FFE1CFD9FFE6522050200B01E167
:100FC00076D08250010B03E18250020B03E02F50D8
:100FD000400B6DE00101E7890601880EFD6F130EDD
:100FE000FE6F33AC45D0CCEC10F00601880EFD6FDF
:100FF000130EFE6F010EE66EE1EC10F0E552A8EC68
:1010000096F033AC2DD00601880EFD6F130EFE6FE7
:101010000101016B640EE66EE40EE66E010EE66EF3
:1010200044ECE2F0E552E552E55290ECDFF0010EBF
:10103000E66ED2ECE4F0E552000901E0FF00500E4C
:10104000E66EA5ECFDF0E5528250010B08E18250FE
:10105000020B05E10101E799A8EC96F0FF00D1D75A
:101060000601880EFD6F130EFE6F12EC11F01FD0FB
:101070002F9CCCEC10F0010EE66EE1EC10F0E55286
:101080008EECDBF09EECDBF05C0EE66EE40EE66EC2
:10109000010EE66E44ECE2F0E552E552E55290ECCA
:1010A000DFF00101E799A8EC96F012EC11F0E5529F
:1010B000E552E7CFD9FF12005FECD5F0DF6AC60E2C
:1010C0004C6ED00E4D6E010E4E6EFD0EDBCF4FF00E
:1010D000506A516A090E416E426A436A4FC03CF041
:1010E00050C03DF051C03EF0D4ECF9F039C04FF0A3
:1010F0003AC050F03BC051F0D4ECD0F0DFCF52F00A
:10110000536A546A77ECCEF00800F5CF00F0F55042
:101110000DE0090EDF5C0AE2FE0EDB5003E10BEC92
:10112000E2F002D02EECE2F0DF2AC9D7E552E3EF7D
:10113000C9F02750200B06E00501105102011911DA
:101140002D1101E1000C010C0101E651400B0CE0F6
:101150000201685109E1080E155C07E0290E155CD3
:1011600004E00A0E155C01E0000C010CF1EC21F02A
:101170001BECD4F02D6B3751381102E020944DDA7E
:101180008CEF65F00701BE51010B07E03AECCCF0A3
:1011900004E0050ED45D01E0000C010C0101269D68
:1011A000010E0D6E26BF0D681200030E9FECCAF0F3
:1011B000258E12006A0E52EFCAF06B0E52EFCAF083
:1011C00001018E51010B08E073EC0FF0000904E0FF
:1011D00001013B51800B01E0000C010C040E9FEC5F
:1011E000CAF001013C0EAC6F12000101AC510DE1DF
:1011F0002DAC08D04D0EE66ED40EE66E010EF6EC68
:10120000CDF001D0EBDF258E2D8C1200258E050E42
:101210009FEFCAF09BECCCF000010E6EE66A02EC88
:10122000D7F00F6E120087C1E6FFA80E42ECCAF09D
:1012300093C100F007ECD5F007E10A0E0101950318
:10124000F350FE0BE842006E0050E66EA90E42EF2E
:10125000CAF0E7ECC9F0FE0EDB5004ECCBF0EF5027
:101260000BE1FE0E64ECCBF007E37EECD1F004EC76
:10127000CBF0100EEF6EEFD7E3EFC9F0E7ECC9F05B
:10128000FE0EDB5089ECCBF0EF5030080BE1FE0E88
:1012900064ECCBF007E37EECD1F089ECCBF0200ED0
:1012A000EF6EEED7E3EFC9F0830E096EFA0EECECA9
:1012B000CBF000500E6E0EC00FF00E6AFB0E73ECFA
:1012C000DBF000505FEFCCF03AC18BF2120001016D
:1012D0003A51130804E2010E3A6F2BA63A6B5AEF0B
:1012E000BCF085ECD5F0020802E1BAC7B9F7FE0EF2
:1012F000DB0402E1B9C7BAF7E3EFC9F01CECD8F0A0
:101300006CEFD2F042C1ABF242C1AAF21CECD8F0B1
:10131000EF50400B03E00201020EAA6F0101D5510C
:101320004DECCBF0EF50400B03E00201020EAB6F2F
:1013300012005FECD5F02850010B17E184ECD1F0DE
:1013400016E14A5014E11750010B03E01C0E155C26
:101350000CE01750100B03E0150E155C06E01F5053
:10136000100B05E00C0E155C02E1000E01D0010E21
:10137000DF6E2C50800B03E12C50400B02E0010E7D
:10138000DF6E2890DF50E552E3EFC9F01A9C238A04
:1013900012000101E38B11C512F50501106B279AAC
:1013A00012000BECD1F01EE00901E6511BE051ECFC
:1013B000D7F0E6C9E6FFB6EC10F0E5520901E751B7
:1013C00005E0E7C9E6FFB6EC10F0E5520901E76B6E
:1013D000E7C9E6F9010136990450010B01E03689AD
:1013E000DAEF08F0010136AF05D004A002D01A8868
:1013F00012001A8A1200E7ECC9F00BECD1F00CE0F5
:10140000FE0EDB5009E0C5DFD7ECD7F00901E6AFEF
:1014100002D001013689CEDEE3EFC9F0E7ECC9F076
:101420000BECD1F011E0FE0EDB500EE0FD0EDB50B8
:101430000BE0AFDFD7ECD7F039ECD3F0FE0EDBAE2C
:1014400002D001013689B6DEE3EFC9F0E7ECC9F05E
:10145000010136AD12D051ECD7F0D7ECD7F0FD0E2C
:10146000DB5002E039ECD3F001013699FE0EDBBE11
:101470003689DB5008E09EDE06D0FE0EDBAE02D0E1
:101480001A8801D01A8AE3EFC9F083ECDAF0DBCFD7
:10149000FBF60201D25101E105D80201190ED26F0B
:1014A000E3EFC9F063ECD5F0010EFBC6DBFF0BECFC
:1014B000D1F062E02050200B5FE00601FB51FC5DA3
:1014C0005BE067DF77DE01013689890EEAECCAF05E
:1014D0000101E3A50BD0530EEAECCAF0570EEAEC7B
:1014E000CAF0520EEAECCAF00101E395640E28EC52
:1014F000D6F0FBECD8F0DF50300805E2DFCFE6FF96
:10150000B6EC10F0E552640EDEECD0F03AC0DBFF32
:101510008CECCAF0FBECD8F00101E7A503D0520E29
:10152000EAECCAF0DF50300808E30601FB5163081B
:1015300004E30101E751040B08E0300EDF5C02E137
:10154000540E01D0DF50EAECCAF00101E7A303D04A
:10155000520EEAECCAF08CECCAF0010EDBCF3EF082
:101560000BECD5F0300FDF6E300EDF5C02E1540E75
:1015700001D0DF50EAECCAF0FBC6FCF6020EE15CDB
:1015800002E2E16AE552E16EE3EFC9F0690E52EF63
:10159000CAF0060EC1ECD6F0280E16ECCAF0C6EF63
:1015A0000AF0010136BFF5DF12000601980ED8805F
:1015B000B0553A0EB15509E20E50B05D0101D86F39
:1015C0000F500601B159010108D0B0510E2401019C
:1015D000D86F0601B1510F200101D96F1200190E09
:1015E0003D6E3E6A0EC042F00FC043F0B6ECF9F01B
:1015F0003BC037F23CC038F2180E426E436A37C225
:101600003DF038C23EF000ECFEF03DC037F23EC087
:1016100038F21200EB0E52EFCAF00101E693199A6C
:10162000139244EC19F0F6DF0201376B386B199412
:101630000FEF0DF003ECA8F00A0E16ECCAF0E30E63
:1016400097ECCBF0006E0050F5E11200E7ECC9F02A
:10165000F1DFEC0E20ECD8F046EC74F000C709F096
:10166000FC0E016E0FC000F013EC3BF0012A0EC01F
:1016700000F013EC3BF0096AE3EFC9F0660E52ECA0
:10168000CAF019801200670E52ECCAF019901200CD
:101690005FECD5F06EEC20F0DF6EE0ECD2F007E00E
:1016A00019A00ED0F0DFDF500BE1006A07D019B0AF
:1016B00007D0E4DFDF5004E1010E006E7CEC75F032
:1016C000E552E3EFC9F0A4ECCAF003E03450400B5C
:1016D00004E001015751040B01E1000C010C5FEC27
:1016E000D5F001018AA10AD06EEC20F0DF6EDF0494
:1016F00003E0020EDF5C02E1010E01D0000EE552B4
:10170000E3EFC9F0ECDF000905E16EEC20F004081E
:1017100001E0000C010CF6DF000904E1E4ECD2F07A
:1017200001E0000C010C5FECD5F01E50010B0EE047
:101730003FECCDF00BE0A4ECCAF003E00FECD1F0ED
:1017400005E11950020B02E1000E01D0010EDF6E1F
:10175000DF5002E08CEC04F0DF50E552E3EFC9F01B
:101760005FECD5F01D50040B1AE01D50080B17E07C
:101770001E50010B14E03FECCDF011E005011051BB
:101780000EE12050040B0BE12050010B08E1A4EC0A
:10179000CAF003E00FECD1F002E1000E01D0010E1F
:1017A000DF6EDF5002E08CEC04F0DF50E552E3EF37
:1017B000C9F08A0EB6ECCEF0010136AD05D0410E6F
:1017C000E66E4E0E78EFCAF036BF258E120063EC3F
:1017D000D5F0C20EDE6E010EDD6E6EEC20F001085B
:1017E00004E06EEC20F002080BE1F40EDE6E010E58
:1017F000DD6E0101345104E0260EDE6E020EDD6E58
:1018000000ECD6F00CE024ECD8F002010051495C69
:1018100001514A5804E2DECF00F2DDCF01F201C2ED
:10182000E6FF00C2E6FF740E0DECCAF0020EE15CAA
:1018300002E2E16AE552E16EE3EFC9F01D9CFCECC7
:10184000D1F0BBDCE50EB6ECCEF0258E120085ECB7
:10185000D5F00A0DF3CF5AF3F4CF5BF3000E03017A
:101860005A27030E5B23E3EFC9F06B0E005C05E221
:101870000201AA510101245F1200FFECD6F004E638
:10188000990E495C000E4A5804E20201AA51010176
:10189000242712001200280E0101D8806855040D7B
:1018A000F328016E0150E66EAA0E42EFCAF0E7EC93
:1018B000C9F02AA40AD00FECCCF0F5EC26F064ECC9
:1018C000DAF00101500EAC6F2A94E3EFC9F0149ED8
:1018D0000A01DA51800B03E1BDECCAF001E1148E7C
:1018E00012000101D451080DB7ECCCF0010ED890D4
:1018F0004B364C36E806FBE10250080D4B50F32402
:10190000496E4C50F4204950016E12000A01DA8FE2
:10191000DEDF0201805158ECCBF01AE220ECD4F06B
:1019200017E202687F0501E1026A030E7F5D02E1B2
:10193000010E026EFF0E025C16E0670E096ED1DF2B
:10194000080EE66ED40EE66E0A0EDCECD7F00BD075
:101950004AEC75F01EAC03D00201098902D00201E5
:10196000068B0501478502017F6B0101B58F500E83
:10197000AC6F2496318C12000201996999C28BF7E1
:1019800099C28AF799C289F799C288F799C287F7ED
:101990000701906991698E698F698EC78CF78FC72F
:1019A0008DF71200040E0101805D03E18150100BE0
:1019B00007E0050E805D03E18150100B01E1000C92
:1019C000010C12005FECD5F00101A85103E19E511A
:1019D000200821E2DF6A090EDF5C10E2DF5019EC1B
:1019E000CCF0EF50040B08E0100EDF24E66E35EC6F
:1019F0002DF0E552000902E1DF2AEDD7090EDF5C88
:101A00000AE2100EDF262986DFCFE6FFF3EC2CF08A
:101A1000E552DF5001D0000EE552E3EFC9F01F861A
:101A2000FCECD1F0B599B59B2582238A1200D9CF61
:101A3000E6FFE1CFD9FFE6528C9600000000FE0ED3
:101A4000DBCFE6FFA2EC5CF0E5520000C950DF6E90
:101A500000008C86030EE66E75ECFEF0E552DF505A
:101A600000D0E552E552E7CFD9FF1200AFEC5CF0B1
:101A7000F00EC616C680C68A1200800EE66EE8EC2E
:101A8000D2F009ECFDF064ECDAF036EF0DF01282E2
:101A900012800601019102011E0E306F1200129099
:101AA0001FA2128012921FB212821200A5ECD6F071
:101AB0004DECCBF0EF50E840E8403F0BDF6E000EFE
:101AC000DF94DF96DF98DF9ADF9CDF9E0A0E006EC0
:101AD000FE0EDB500DE1DF5002E1010E006EDF046F
:101AE00002E1020E006E020EDF5C44E1050E41D001
:101AF000FE0EDB50030804E1DF5002E1010E006E30
:101B0000FE0EDB5004080EE1DF0402E1320E006E2F
:101B1000020EDF5C02E15A0E006E030EDF5C02E192
:101B2000640E006EFE0EDB50050810E1320E006EF2
:101B3000DF0402E1640E006E020EDF5C02E17D0E46
:101B4000006E030EDF5C02E1FA0E006EFE0EDB0497
:101B500004E0FE0EDB5002080DE1DF5002E1010E51
:101B6000006EDF0402E1050E006E030EDF5C02E191
:101B7000190E006EE552E3EFC9F0ECECD8F0C4C1E9
:101B800000F0000406E10101C551460802E2020E20
:101B9000006E030E005C06E10101C551280802E257
:101BA000040E006ED5CA03F049ECD2F005E03751BF
:101BB000080B02E0040E036ED60E4A6ECC0E4B6E7E
:101BC000010E4C6E0050EFECCAF0035064ECCFF005
:101BD000EF504924016E0D0E4A6ECD0E4B6E010E74
:101BE0004C6E0050EFECCAF003506AECCFF0EF50AF
:101BF0004924026E20ECDAF0E66A7D0E49ECCCF066
:101C0000ECECD8F0280E026E016E49ECD2F00EE03A
:101C10003751080B0BE01CCA01F021CA02F0015039
:101C200002E0025003E1280E026E016E20ECDAF0B1
:101C30007C0E0DECCAF0ECEFD8F0129A1FB2128AAB
:101C40002EDF25ECD4F01CEC6AF01F50020B06E0EE
:101C50000101D551D45D02E01A8C12001AAC02D0F9
:101C6000C6EC09F01200080E0B5C04E300ECD6F0A1
:101C700001E1000C010C095004E00701010E1FEC0A
:101C8000D7F0096AB2EC04F0000907E0750EE66EC1
:101C9000280EE66E010EB5ECD9F01200B2EC04F09D
:101CA000000909E07E0E096E080EE66EB60EE66EBD
:101CB000020EB5ECD9F0096A120083ECDAF0DBCF42
:101CC00048F1B9ECD9F001ECD2F01BECD4F0139848
:101CD000E3EFC9F00101485112E0060E28ECD6F0FE
:101CE00048C13EF06EECD8F0006E005001E1002AD1
:101CF00000500101485F48C15BF26EEFCCF02094C8
:101D000055EFCEF007015A5106E1080E97ECCBF0E3
:101D10000501261501E1000C010C2C9E2C9CABEC5E
:101D20002EF0FCEF96F0E7ECC9F029ECD4F007E1D7
:101D30002B50010B04E101018A51200B09E140C243
:101D400043F23FC242F23EC241F240ECD3F009D02E
:101D5000FE0EDB5006E043C240F242C23FF241C2F7
:101D60003EF204802BA002D004902B90FBEC40F0BC
:101D70000101320EAC6FE3EFC9F025B41200189ADE
:101D800017B8188A12000301916B926B936B946BD6
:101D900091C38DF392C38EF393C38FF394C390F3E7
:101DA000030E016EFF0E015C32E0056A030E026E47
:101DB000FF0E025C22E00250EA6A890FE96E030E10
:101DC000EA22EF504B6E4C6A0150EA6A850FE96EC9
:101DD000030EEA22EF5078ECCDF01FECD1F0EF507B
:101DE0005FECCCF005505FECCCF01FECD1F00EC0F6
:101DF000EFFF0FC005F00206DBD70150EA6A8D0F36
:101E0000E96E030EEA2205C0EFFF0106CBD71200F0
:101E100085ECD5F0006E00AE04D0006C01010E0E12
:101E2000116F0101040E2EECD4F012510AE111C120
:101E300012F1100E116F135104E112C113F1100EC3
:101E4000126F130E156FE3EFC9F03AECCCF003E11B
:101E5000030E0A5C01E0000C010C3AECCCF005E149
:101E6000020E0A5C03E00A0401E0000C010C3AECEB
:101E7000CCF003E1020E0A5C01E0000C010C3AEC2C
:101E8000CCF007E10A5005E1CF51040B01E0020C50
:101E9000010C000C3AECCCF005E1020E0A5C03E008
:101EA0000A0401E0000C010C0601EC5106E03AECDA
:101EB000CCF003E10A50000801E3000C010C3AECFD
:101EC000CCF004E10A0403E00A5001E0000C010C2C
:101ED0003AECCCF006E1020E0A5C04E0030E0A5C68
:101EE00001E0000C010CA4ECCAF003E0F0ECD2F02D
:101EF00001E1000C010C0101D45104E10A01DA51A5
:101F0000040B01E1000C010C0101D45104E10A01B0
:101F1000DA51080B01E1000C010C4DECD2F009E0A4
:101F20000301B85177ECDBF006ECCCF0210E0DECA0
:101F3000CAF012004DECD2F002E08DEF0FF0E66A2D
:101F4000E66A210E0DEFCAF03AECCCF010E1D05168
:101F5000040B05E00A040CE0020E0A5C09E0CF5114
:101F6000040B05E00A5004E0030E0A5C01E0000CDB
:101F7000010C0101D45103E1D051400B04E1E4DF35
:101F8000000901E1000C010C13ECD1F001E0030C9D
:101F90000FECD5F001E0080C51ECD2F001E11B0C84
:101FA000D45109E0030ED45D05E10A5004E0030EAC
:101FB0000A5C01E0030C010C13ECD1F001E00A0C07
:101FC0000FECD5F001E0380C51ECD2F001E1640CDB
:101FD000D45101E0500C380CEFDFE66ED5DFE66E31
:101FE000D60EE66E0A0E25EFCAF08EEC41F0190E01
:101FF00001240A01D880D75503E2190E0124D76FB6
:10200000F4ECD2F0D75D03E2F4ECD2F0D76FD46BEE
:10201000338870EFCFF013ECD1F004E10FECD5F082
:1020200001E1000C010CEF0E896E8A6A8B6A9E0E2C
:102030008C6E900E8D6E8E6A8F6A010E906E916A14
:10204000EF0E926E070E936E930E946E600E956E69
:10205000030E966E7F0E976E060E986EFE0E996EAC
:102060009A6812001F98258A0101B59B02011A5136
:102070001FE0020E685D03E1F8ECD2F019E0070101
:10208000BE9BBE9B32BCBE8B7EEC09F00601EA050E
:10209000EB6F020EEA5D01E2EB6BEBC600F00101B3
:1020A000D45102E0EDC600F00050E66E96ECD6F09A
:1020B00002011A6B25821200C08EA70E3CECCDF0F7
:1020C00033ECD4F0A70E3CECCDF0C3500E26C45038
:1020D0000F220EC04DF00FC04EF0D8904E324D3250
:1020E0000EC04FF00FC050F0D89050324F32D89001
:1020F00050324F324D504F244B6E4E5050204C6E4C
:102100000EC051F00FC052F0040ED890523251322E
:10211000E804FBE151504B5C496E52504C584A6EFA
:102120000EC053F00FC054F0060ED8905432533204
:10213000E804FBE1495053240E6E4A5054200F6EC0
:102140000EC0CDF20FC0CEF2C09E1200CDC20EF076
:10215000CEC20FF0E66AB2EC26F0E5520101200E85
:10216000166F1C6F188F410E1B6F1200E7ECC9F041
:1021700005011151EA6A000FE96E080E29ECD8F04A
:10218000112B115182ECCAF002E638ECD4F001E3D5
:10219000116B102BE3EFC9F0B2EC04F0000910E072
:1021A0002DECCDF0020E0101395D02E1010E396F17
:1021B00062DD91EC48F072DD9CEC48F05AEC79F06D
:1021C0001200E7ECC9F00101E7890601880EFD6FF6
:1021D000130EFE6FAEEC16F08A988A8663EC25F03B
:1021E0000101766B140EE66E18ECC3F0E552FE0E9C
:1021F000DB500CE043EC0BF0C6EC0AF057ECC4F0FB
:10220000F6ECC4F0A5ECE2F0EFECE0F00601506B68
:1022100097EC3DF00601516B0101B96BEF0E926E28
:10222000E3EFC9F0F29E80ECFEF0F26AF06AB96A60
:102230009D6A000EA66EA16E9E6E8D8C8D8A8C900E
:102240008484070E936E0000000000008A9A00004C
:10225000000000000000270E936E4E0E996E0000E5
:102260000000000003000000000000000000FF006C
:1022700012005FECD5F020AA3BD03DECD4F006E391
:10228000EFECD8F035E206ECD2F032E21B50080B4E
:102290002FE13DECD4F006E3EFECD8F029E206ECB8
:1022A000D2F026E23DECD4F006E3EFECD8F020E2E9
:1022B00006ECD2F01DE20050DF6EDF5058ECCBF0A0
:1022C00013E206ECD2F010E2DF5042ECD4F004E668
:1022D000B40E4B5C000E4C5807E2540EE66EE40E52
:1022E000E66E010E47ECD3F0E66A6BDFE5529ADF4B
:1022F000E552E3EFC9F0E7ECC9F09EECDBF00FEC40
:10230000CCF07EECCAF090ECDFF08FECCDF08FECEF
:10231000CDF08FECCDF0FA0E23ECD7F0FA0E23ECD3
:10232000D7F0E3EFC9F033ECD4F055ECD2F055EC34
:10233000D2F0460E28ECD1F00F50496E4A6A9F0E3B
:10234000E2ECD7F0006E0050800801E2006A020162
:10235000FC0ED880CD55080ECE5502E2040E0FD0EB
:10236000080ED880CD55070ECE5502E2030E07D0D9
:10237000140ED880CD55050ECE5503E2020E002670
:1023800007D0200ED880CD55030ECE5501E2002A8D
:102390000050800801E2006A080ED880CD55070E73
:1023A000CE5502E2030E07D0140ED880CD55050E8F
:1023B000CE5503E2020E00261200200ED880CD5525
:1023C000030ECE5501E2002A120063ECD5F0C08E58
:1023D000AF0E3CECCDF0010157A9C5D0500ED8800E
:1023E000C354050EC45401E3BAD0D00EC35C0A0E28
:1023F000C45801E3B4D03C0E496E4A6ACDC23DF0E8
:10240000CEC23EF0B5ECDAF000503C0802E23C0EE1
:10241000006E76ECDAF007014950C35CD06F4A5089
:10242000C458D16F140ED05F050ED15B010157ABBC
:102430009AD0D0C7D8F1D1C7D9F147ECD4F0070E64
:102440007CECD0F0FDE16A0E4924096E47ECD4F033
:1024500080ECD8F0D0ECCDF00101E7AF10D0E79FD1
:10246000C80EC1ECD0F004E3840E80ECD0F002E2A0
:10247000070119D00EC0D2F70FC0D3F76DD0C80E28
:10248000C1ECD0F004E3840E80ECD0F011E207013F
:10249000C80ED25D000ED35906E3840ED880D25503
:1024A000030ED35560E2260ED26F020ED36F54D0C6
:1024B000010E07014A6AD225496ED3514A2228ECFF
:1024C000D7F00CE3D2C74BF0D3C74CF04B06000E4D
:1024D0004C5A4B500E5C4C500F5845E20101D45100
:1024E0000CE107010E50D25D0F50D35903E2D22BFD
:1024F000000E1CD0D207000E2ED007010E50D25D68
:102500000F50D35915E2D2510E5C0101D86F07016B
:10251000D3510F5874ECD2F003E2050ED86FD96B8B
:10252000D8510701D2270101D9510701D32314D073
:102530000E50D25D0101D86F0F500701D35974ECD2
:10254000D2F003E2050ED86FD96BD8510701D25FE4
:102550000101D9510701D35B4AEC32F004D00701E5
:10256000060E1FECD7F0C1ECCAF00701A7274A50AE
:10257000A823A7C749F0A8C74AF02DECD7F0070158
:10258000A75F4A50A85B080ED880C354090EC454F4
:1025900062E333ECD4F00B0E28ECD1F0040E55ECD2
:1025A000D2F0E804FCE1360ED8800E56060E0F5627
:1025B000CDC249F0CEC24AF07CECD0F0FDE14950EA
:1025C0000E264A500F2220BA0ED0B2C249F0B3C232
:1025D0004AF02DECD7F00201B25F4A50B35B0E50C7
:1025E000B2270F5013D0B2C249F0B3C24AF0640E02
:1025F00001ECCAF049500201B25F4A50B35B57EC9C
:10260000D6F02DECD7F00201B2274A50B323020EC8
:102610004A6AB425496EB5514A22B251495CB35158
:102620004A5813E3020ED880B455000EB55513E294
:10263000B4C24BF0B5C24CF0020E4B5E000E4C5AC9
:102640004B50B25D4C50B35906E24AEC32F0B2C284
:10265000B4F2B3C2B5F2C09E0EECCBF002E2E16A76
:10266000E552E16EE3EFC9F063ECD5F0C08EAB0E3E
:102670003CECCDF0C1ECCAF00701A9274A50AA23CF
:10268000A9C749F0AAC74AF02DECD7F00701A95F06
:102690004A50AA5BC09E0EECCBF002E2E16AE55222
:1026A000E16EE3EFC9F063ECD5F0070114A108D0A7
:1026B000149177ECD5F07D0E976E060E87ECD8F06E
:1026C000C08E9B0E3CECCDF0C1ECCAF00701AB27ED
:1026D0004A50AC23ABC749F0ACC74AF02DECD7F059
:1026E0000701AB5F4A50AC5BC09E0EECCBF002E240
:1026F000E16AE552E16EE3EFC9F085ECD5F007E160
:10270000C00E016E01015FA304D0E00E01D0B00E37
:10271000016E01010D51012656EC3BF0FE0EDB501F
:1027200013E00F0E005C03E3005030080DE2230EAF
:10273000006E0901EB5108E0020E0101395D04E071
:102740000901EB51D0ECD5F00050E3EFC9F05FEC9C
:10275000D5F0BCEC0CF0BDECCAF008E10701B16BA0
:102760000A01D56BDA934AEC75F012D0FBECCDF090
:10277000EFCFB1F7D4C1DFFFD5CA00F0080EE66E87
:10278000E66ADF5084ECD6F0BDECD9F009ECCDF070
:10279000149C0101D45103E0030ED45D06E1030E45
:1027A0000A01D45D07E1148C05D0020E0A01D45D44
:1027B00001E1148CDAA304D0D8CAB6F7D9CAB7F7A6
:1027C00057EC19F01CECD8F0EFCFBEF70701BE9F15
:1027D0000101D45103E0030ED45D02E10701BE8F75
:1027E00044EC1FF073ECCCF0A5ECDFF06EEC25F0C0
:1027F00082EC09F0E552E3EFC9F0D2ECDAF084ECB8
:10280000D6F009EFCDF01CECD8F06CECD2F0BDECBA
:10281000CAF00FE00A01DAA306D0B6C7D8FAB7C7E4
:10282000D9FA57EC19F0E9DF0101FBECCDF0B1C7A3
:10283000EFFF12005FECD5F0DF6A080EDF5C04E208
:1028400002ECD9F0DF2AF9D7E552E3EFC9F05FECEB
:10285000D5F0DF6A080EDF5C0CE272ECCBF0EFCF54
:1028600049F0FE0EDB50495C02E1010E03D0DF2A85
:10287000F1D7000EE552E3EFC9F0E7ECC9F018BE5E
:1028800008D095ECD5F073EC04F0E5527F0B93EC97
:10289000CAF0E3EFC9F0E7ECC9F018BE15D029A0E3
:1028A00003D07DEC07F0FBD746ECCFF00DE046EC13
:1028B000CFF093ECCAF0D950FC0F2EECD8F0EE2AF2
:1028C000000EEE22EE22F0D7E3EFC9F0E7ECC9F0FC
:1028D00018BE25D029A003D07DEC07F0FBD7D7EC9C
:1028E000CBF0E80E426E030E3EECCCF0492493ECA4
:1028F000CAF0DEECCBF00FECD9F0D7ECCBF0640EE5
:1029000095ECD7F0640E09ECD9F00A0E95ECD7F0EF
:102910000A0E09ECD9F0300E492493ECCAF0E3EF2B
:10292000C9F0E7ECC9F018BE0FD01EAE0DD04F0EA7
:10293000E66EE40EE66E010E48ECCAF00FECCCF049
:10294000AADFE552E552E552E3EFC9F05FECD5F0BE
:102950000201CF2B1EAE19D0660EE66EF20EE66EA9
:10296000010EE5ECCAF095ECD5F087DFE552FE0EDE
:10297000DB28E66E82DFE552FE0EDB50020FE66ECC
:102980007CDFE5523B0E93ECCAF095ECD5F05FDFAF
:10299000E552000915E1DF6A080EDF5C11E272EC16
:1029A000CBF0EF50FF080AE172ECCBF0FE0EDBCF6C
:1029B000EFFF02ECCEF026C7EFFF02D0DF2AECD704
:1029C00007012669E552E3EFC9F05FECD5F0DF6A55
:1029D000080EDF5C0FE272ECCBF0EF50FF0808E06E
:1029E00002ECCEF0EF50016E72ECCBF0EF5005D060
:1029F000DF2AEED70201CF6BFF0EE552E3EFC9F0FD
:102A000063ECD5F0DF6A080EDF5C0FE272ECCBF00E
:102A1000010EEFCFDBFFDB50FF0805E002ECD9F041
:102A2000010EDB5005D0DF2AEED70201CF6B000E7E
:102A3000FCECD2F002E2E16AE552E16E4950E3EFCC
:102A4000C9F05FECD5F03250100B04E1020E070123
:102A50005A5D02E1DF6A03D08EECD8F0309ADF5085
:102A6000E552E3EFC9F063ECD5F03250100B04E10E
:102A7000020E07015A5D03E1DE6ADD6A08D08EECC2
:102A8000D8F0E66A02ECD7F085ECD0F0309A0EEC84
:102A9000CBF002E2E16AE552E16EE3EFC9F05FECF0
:102AA000D5F007015E6B5F6B2DA802D0010E2ED012
:102AB000080E97ECCBF0DF6E07015E2B000E5F2354
:102AC000ECECD8F0200EDF1406E00701580E5E5D36
:102AD000020E5F59EDE307015E51605D5F51615980
:102AE00004E25EC760F75FC761F7580E5E5D020ED5
:102AF0005F590BE301018B5105E15CC726F7360EE8
:102B000020ECCBF02D88000E01D0010EE552E3EF52
:102B1000C9F0E7ECC9F04BECD3F0E3EFC9F0E1EC1E
:102B2000D6F003E200ECD3F004D0FE0EDB50F60F3B
:102B3000410FE3EFC9F0020E006E020178B9008E7A
:102B400035C101F00150280802E2280E016E005044
:102B5000E66E060E0102F350E66E780E0DECCAF03A
:102B600076EC20F0016A01013551280807E27C0E5D
:102B700051ECD4F003E2280E355D016E0150E66E93
:102B80003A0E42EFCAF05FECD5F06EEC20F0DF6E4B
:102B90000F0EE66EDF5007E0030EDF5C04E001017C
:102BA0008A51020B02E1000E01D0010E000905E07E
:102BB0000A0E01017A03F35001D0000EE66E7E0E7C
:102BC0000DECCAF0E552E3EFC9F064C178F2F0EC25
:102BD000D2F002E165C178F21200F0ECD2F003E12C
:102BE00078C265F102D078C264F1EFDF9BEF15F097
:102BF0008DC20EF08EC20FF015ECD9F05E0E0DEC0A
:102C0000CAF08FC20EF090C20FF015ECD9F05F0E33
:102C10000DECCAF092C2E6FF91C2E6FFE66A7B0EB7
:102C200049EFCCF00601B46BB56B020EA9ECCDF008
:102C30000601B42B000EB523B451B65DB551B7599A
:102C400004E2B4C6B6F6B5C6B7F6E80ED880B455F9
:102C5000030EB5550BE201018B5105E15CC726F768
:102C6000390E20ECCBF02D883186010C84B0DDD7F5
:102C7000000C5FECD5F0FE0EDBCF5CF72D50100B97
:102C800003E13150100B02E1000E20D031A604D038
:102C90000A0EA9ECCDF001D0C5DF95ECD5F017EC0C
:102CA0000DF0E552DF6EE66A17EC0DF0E55201011A
:102CB0003851100B0AE03050200B07E1E7A102D099
:102CC0002E0E01D0210E04ECD6F0DF50E552E3EFDA
:102CD000C9F0A6ECD5F00101E791E3EFC9F0A6EC4D
:102CE000D5F0FC0E8FECCAF00101E791E3EFC9F0DB
:102CF000A6ECD5F01BECD9F00101E791E3EFC9F0A8
:102D0000A6ECD5F01BECD9F0FA0E8FECCAF0F90E58
:102D10008FECCAF00101E791E3EFC9F0D9ECDAF0EA
:102D2000D8C1E6FF02ECD7F0D9C1E6FF02ECD7F03C
:102D30000EC0E6FF02ECD7F00FC0E6FF02ECD7F0C2
:102D40000101E791E3EFC9F01D0E20EFD8F01E0E50
:102D500020EFD8F0D9CFE6FFE3EFC9F02AB203D0D5
:102D6000600E52ECCAF02A8212002AA203D0610E31
:102D700052ECCAF02A9212002AB203D0600E52EC32
:102D8000CAF02A8212002AA203D0610E52ECCAF0C5
:102D90002A921200E7ECC9F031B206D0620E52EC72
:102DA000CAF0FE0EDBCF1BF2E3EFC9F0E7ECC9F08F
:102DB000B00E52ECCAF0FE0EDBCF1CF2E3EFC9F00E
:102DC000E7ECC9F007018651320D56ECD4F013EC54
:102DD000D5F012E1FE0EDB500FE10101D45104E108
:102DE00029510A0D56ECD4F0C5ECD0F005E00101F4
:102DF000E80ED86F030ED96FE3EFC9F05FECD5F0A2
:102E0000D6CA85F707011E0E866F0101D45105E170
:102E1000D8ECCDF03EC086F710D0030ED45D0DE1A6
:102E2000030E0A5C03E10701140E06D0AEECCDF0F0
:102E300004E0E8ECD7F00701866FD7CA00F007017D
:102E4000BEAF10D0190E006E0A01D75D06E204EC89
:102E5000D3F033ECD8F0005E05D0190ED75D33EC1B
:102E6000D8F00026190E005C05E3190E005C07017E
:102E7000862705D0190ED88000540701865F080EFA
:102E8000006E21A20FD00101D45102E1020E18D030
:102E9000D40506E0020ED45D03E0040ED45D11E11A
:102EA000010E0ED00101D45102E1080E09D0D40563
:102EB00006E0020ED45D03E0040ED45D02E1070ECD
:102EC000006E07018551FE0BE8420024056EDF6AA3
:102ED0000550865D13E2DF2A8551FE0BE842862508
:102EE000016E01500024FE0BE842866F0050015C29
:102EF00002E20050016E0050015C856FBDECCAF02B
:102F000005E10701320E856F1F0E866F51ECD2F07E
:102F100004E2DFCFE6FF54DFE55217ECD5F05EE0C8
:102F20000701BE51800B27E0DF5025E15FDB13EC8A
:102F3000CFF00A01D751190808E2190ED75D06EC47
:102F4000D7F00101D8274A50D92313ECD5F008E275
:102F500004ECD3F006ECD7F00101D85F4A50D95BFE
:102F600001010A0ED903F3CFD9F1D803F3CFD8F179
:102F7000F450D92704D0DFCFE6FF22DFE552070166
:102F80008551320DB8ECCAF03AECCCF001E1D98FA2
:102F9000200E006E07018851005C10E18C51010188
:102FA000D8190CE107018D510101D91907E1070179
:102FB0008E510E1802E18F510F180DE000C088F7F6
:102FC000D8C18CF7D9C18DF70EC08EF70FC08FF71F
:102FD000005096ECD8F063DD8DEC0FF0BDEC0DF0F9
:102FE00057EC4EF0E552E3EFC9F0B2ECCDF00050F3
:102FF00001E1120017ECD5F070E00101DC0ED86F92
:10300000050ED96FF00E0E6E0A0E0F6E030E005CE9
:1030100001E1D98F000403E0020E005C45E16FEC92
:103020000BF0000915E001018951640DB8ECCAF0FC
:1030300013ECCFF0010E0F0B05E0D890D933D83345
:10304000E806FBE1640E0101D827000ED9232CD03D
:103050000101345129E03451080DF3CFD6F1F4CFFA
:10306000D7F15C0ED627000ED723D6C149F0D7C1C1
:103070004AF0F00ED88049560A0E4A56010E0F0B40
:1030800003E094ECD0F0FDE149500101D625D86F62
:103090004A50D721D96FD6C10EF0D7C10FF0F00E2C
:1030A000D8800E560A0E0F56040ED45D08E1340E79
:1030B000D86F080ED96FA00E0E6E0F0E0F6E050E94
:1030C000D45D08E10E0ED86F060ED96FC40E0E6ED9
:1030D000090E0F6E300E96ECD8F04FEF15F0320E51
:1030E000E66E730E42EFCAF0640E52EFCAF063EC64
:1030F000D5F0A4ECCAF001E192D00AECCBF001E0EB
:103100008ED007015A5101E08AD059ECD2F001E08B
:1031100086D0195101E083D001013B51800B04E1BD
:10312000050ED45D01E07BD0080E97ECCBF0DF6E8E
:10313000BDECCAF06EE1E49FDFB8E48FE651040B0A
:1031400068E09451010865E20201D95162E1D85169
:1031500060E10101E651010B5CE1E451800B54E0B8
:10316000A1ECCBF051E01D50400B4EE10201685143
:103170004BE12050200B48E0195146E1245144E135
:103180002C50800B41E12C50400B3EE12F50200B86
:103190003BE12350800B38E13050400B35E12450A7
:1031A000010B32E1DAEC08F0D9DD0101030E9E6F6C
:1031B000280E9F6F440EA06FA26BA2C1A1F1F4EC88
:1031C000C5F00701148F149377ECD5F00701159122
:1031D0007EECD5F007010B89BCECC4F0E00E0701D2
:1031E0000A150609E66E120E4EECDBF00701099F88
:1031F0007F0E09116AECD5F0820E52ECCAF0010183
:103200009405190DF3CFD8F20101E4BF02D0DDEC33
:1032100008F001013BAF03D0010EDF1401D0000E16
:10322000FCECD2F002E2E16AE552E16E4950E3EFD4
:10323000C9F001013B51800B06E0A4ECCAF003E0A9
:103240000AECCBF001E0000C010C53C1E6FFF1DF0A
:10325000000903E001016E5101D0000EE66E340E4C
:103260000DECCAF06FC1E6FF350E42EFCAF0650EF5
:1032700052EFCAF02050400B06E00101E551040B6B
:1032800002E1E58501D812005FECD5F054C1DFFF03
:10329000F0ECD2F002E158C1DFFF080EDF02F3507C
:1032A000E66E750E42ECCAF0E552E3EFC9F0070195
:1032B000B6510C0803E3B7510C0805E2B66B0C0ECF
:1032C000B76F0A01DA931200016A0D0E015C07E084
:1032D00052ECCFF002E001501200012AF6D7000CA8
:1032E0000C0E016E015007E052ECCFF002E00150ED
:1032F00012000106F7D7000C0701B46BB56BD7DFDE
:10330000B6C701F00701B751D880015409E36FEC4B
:1033100004F0F3500701B413F450B513012AF2D7A7
:103320001200016A13ECD1F00BE05CECD6F006E27F
:1033300049500508000E4A5401E2012A420E0DD000
:103340000FECD5F012E05CECD6F006E24950140820
:10335000000E4A5401E2012A440E012411ECD4F07B
:10336000F3CFB4F7F4CFB5F712005CECD6F014E26B
:1033700049504608000E4A540FE20701F40EB46F9C
:10338000B569BDECCAF001E1AFD00701B66B0C0E18
:10339000B76F0A01DA83A8D0006AD75158ECCBF096
:1033A00006E249500D08000E4A5401E2002AD751A6
:1033B00058ECCBF006E249501308000E4A5401E2E3
:1033C000002AD751180801E2002AD751190801E252
:1033D000002AD75158ECCBF006E249501F08000EE6
:1033E0004A5401E2002AD75158ECCBF006E249508A
:1033F0002508000E4A5401E2002A0101D45103E0DD
:10340000030ED45D1CE15CECD6F006E249500508E1
:10341000000E4A5401E2012A7AECDBF006E2495040
:103420000A08000E4A5401E2012A7AECDBF022E29B
:1034300049501308000E4A541DE2012A1BD05CECCF
:10344000D6F006E249501E08000E4A5401E2012A55
:103450007AECDBF006E249502808000E4A5401E2FB
:10346000012A7AECDBF006E249503208000E4A5499
:1034700001E2012A690E4C6EDB0E4D6E010E4E6E9E
:1034800000504F6E506A516A030ED8904F36503636
:103490005136E806FAE1D4ECD0F00150526E536A8E
:1034A000546AD89052365336543677ECCEF0090031
:1034B000F5CFB4F70A00F5CFB5F74DECD2F005E043
:1034C0000701B485B589B49DB59B030E0A01D45D8F
:1034D00002E0D45109E1F8DE0701B66F01DF070110
:1034E000B76F0A01DA83E3DE0A01D40514E10701AC
:1034F000B705056E0A0EB75D01E20506E5DE0701B8
:10350000B66F0550D880B65502E205C0B6F7F4DEB6
:103510000A01DA831200020ED45D12E10701B62916
:10352000056EB651020801E2052ADADE0701B76F1F
:103530000550B75D02E205C0B7F7DEDE0A01DA83A7
:1035400012001E0E006E0101D45104E1D8ECCDF042
:103550003E500AD0C5ECD0F002E0140E05D0AEEC1F
:10356000CDF003E0E8ECD7F0006E0A01D651FE0B77
:10357000E842056E1200050E00ECCBF0050E0A01C4
:10358000D803F350006E0101012B5EECCFF01B8FCE
:103590001200080E00ECCBF00A01D951050D37ECF2
:1035A000D8F00101200E196F19C118F11B8F1200FC
:1035B00037ECCFF0C9ECD0F03B51200B06E1BDEC6D
:1035C000D0F003E001011E0EAC6F38EC64F0A1EC0A
:1035D000CCF0300E0101195D02E1200E196F1B8F36
:1035E000016B2A0E006E238825EF26F00101D451CD
:1035F00002E129510BD0030ED45D11E1030E0A5CE8
:1036000002E1640E03D00A5004E1960E0E6E0F6ABA
:103610001200240E2E259CECCBF00E6E0F6A1200C9
:1036200090DF0701BEAF11D021ECD9F00A01D751CC
:10363000190804E2190ED75D5FECCCF0190ED75DC6
:1036400018E204ECD3F050EFD3F00A01D751190877
:1036500003E2190ED75D0026190ED75D03E204ECD4
:10366000D3F0005E005077ECDBF0190ED75D01E17E
:10367000BDDF1200570E00ECCBF0DCECD2F006E11F
:10368000BDECD0F003E001011E0EAC6FC9DF4DECC4
:10369000D2F00BE00101410E166F500E176F0301BF
:1036A000B8510F6AE8307F0B0E6EA1ECCCF001012F
:1036B000200E196F19C118F14DECD2F009E001018B
:1036C000460E186F2951E8240301B85D07E103D0C5
:1036D00013ECD5F003E101012A0E196F01011B8FD4
:1036E00012000A01D45102E163DF0AD0D40502E1DD
:1036F00042DF06D0020ED45D02E14BDF01D0BADF1B
:10370000C9ECD0F03B51200B06E1BDECD0F003E05A
:1037100001011E0EAC6F1200E7ECC9F0070EE126A6
:10372000C4EC0FF00A01D65D04E2C4EC0FF00A010C
:10373000D66FDCEC0FF00A01D880D65504E2DCEC41
:103740000FF00A01D66F0BEC10F0000903E00A013C
:10375000190ED76FF6DE13ECD5F004E3190ED75D22
:10376000002603D004ECD3F005260550005C03E3EB
:103770000550005E0AD0006AD40507E1DC51D75D30
:1037800004E2DCCAD7FADDCAD6FA00C0D8FAD9DE1C
:103790000550002613ECD5F004E3190ED75D002682
:1037A00009D004ECD3F0056E0550D880005402E235
:1037B0000550005EEFECD8F00BE249505408000EC3
:1037C0004A5406E2540E006EDCCAD7FADDCAD6FAB5
:1037D00000C0D9FA00C0C5F7190ED75D03E3190E72
:1037E000D75D03D0190ED880D7550701B26FB36BE0
:1037F000BEAF02D00A0E01D0320EB303F3CFB3F73F
:10380000B203F3CFB2F7F450B327FE0EDB5004E05F
:103810002050800B01E165DF3450040B0DE10A01FB
:10382000DA51020B09E013ECD1F006E10FECD5F010
:1038300003E14DECD2F003E074DD349401D05CDDA3
:103840000701010EB06F01012AA303D00701070E83
:10385000B06FD5CADFFF0A01D56B0701B05101086F
:1038600053E208ECD3F050E1D251010B4DE1050ECB
:10387000D45D4AE0040ED45D47E0D40503E0020EB7
:10388000D45D0FE1AEEC04F00A01D95D0AE2D52B5C
:1038900023ECDAF004E61E0E495C000E4A5834E2CE
:1038A0001ED00101D4511DE10A0123ECDAF004E637
:1038B0001F0E495C000E4A5801E2D52B23ECDAF0CA
:1038C00004E60F0E495C000E4A5809E3D65142EC5B
:1038D000D4F004E60B0E4B5C000E4C5815E2D52BD1
:1038E00013D00A0123ECDAF004E62D0E495C000E39
:1038F0004A5801E2D52B23ECDAF004E60F0E495CBE
:10390000000E4A5801E2D52BDF500A01D55D0AE0CE
:10391000D5CADFFFA5ECDFF0D5CAE6FFAB0E42EC5F
:10392000CAF0248A1EAC03D00201098902D0020128
:10393000068B05014785F0EC39F0070EE15C02E2E9
:10394000E16AE552E16EE3EFC9F0006A800E066EAF
:10395000056E05500502F350015CF4500258D8B0D2
:1039600008D000C005F006420650051206BE09D078
:10397000F0D705C000F006420650051206BE01D081
:10398000E8D700D01200E7ECC9F02A8448C102F061
:1039900085ECCBF03FE05A0E025E010EE66E7DEC48
:1039A00013F0E552016E02504B0817E24B0E025C19
:1039B000036E060E4A6E4AC043F001C03EF05AEC58
:1039C000FEF03EC049F049C043F003C03EF05AEC5F
:1039D000FEF03EC003F00350015E0F0E015C02E2F8
:1039E0000F0E016E0150300802E2300E016E01C070
:1039F000C1F702500A0DB8ECCAF00150496E4A6A8C
:103A000053ECD6F03D50026E23B604D00250E824A9
:103A10000201D56F5BECD4F00701C06FFE0EDB50E6
:103A2000020801E187D0C0C701F00101E6A502D07C
:103A3000040E016E01504B6E4C6A025078ECCDF0D2
:103A4000030ED8900E360F36E806FBE155ECD3F0A6
:103A50000A0E4F6E4FC043F00BC23EF06EECD8F032
:103A60004D6E4E6A00504B6E4C6A800E3D6E3E6A43
:103A7000BAECDAF0A8ECCFF052ECDBF010ECCDF0C1
:103A8000036A2CDB016E1C50040B2FE0010403E0E1
:103A9000020E015C2AE13450400B27E1FE0EDB50A0
:103AA00024E001C202F0025020E0025082ECCAF091
:103AB00002E660ECD4F019E20250FE0BE842D88036
:103AC000005413E20250E824005C0FE2FE0EDB0417
:103AD00006E10C0E02010027000E012305D00C0E9A
:103AE0000201005F000E015B032A03500EE1880E05
:103AF000D8800E54130E0F5404E2880E0E6E130E6F
:103B00000F6E0EC000F20FC001F22450020B06E14E
:103B10002250400B03E03150800B0AE0036A006A38
:103B200031AE06D0000E0201026F036B006F016B15
:103B3000E7EC0BF0E3EFC9F0E7ECC9F006ECCCF0F2
:103B400095ECD5F06FEC16F064ECDAF0E3EFC9F029
:103B5000E7ECC9F0EDECD7F0770E0BECD2F0FE0EEF
:103B6000DB5003E0100E0BECD2F0E3EFC9F0B2EC47
:103B7000CDF0050E005C09E01BECD5F006E16FEC22
:103B80000BF0000902E1000E01D0010E000902E075
:103B9000000E03D001013451E824E66E3C0E42EFE2
:103BA000CAF0C6EC3FF0E3DF0201A85103E00101D7
:103BB000345106E00201A85105E10101345102E04F
:103BC000F5EC17F02A841200A5ECD6F003E0010111
:103BD000285101D0000EDF6E21B204D0040EDF02A6
:103BE000F3CFDFFFDFCFE6FF760E42ECCAF0DF90C7
:103BF000DF42DF5005E1FE0EDB5002E0010EDF6E1A
:103C0000DFCFE6FF790E42ECCAF0E552E3EFC9F0F0
:103C1000E7ECC9F0016A080E015C16E2FE0EDB500B
:103C2000012465ECD4F0026E100E025C040DF3501A
:103C3000006E3AECCCF001E1006ACCECDAF0005016
:103C400052ECCAF0012AE7D7140E16ECCAF0E3EFE3
:103C5000C9F017ECD5F00CE0220E52ECCAF00101CD
:103C6000D45102E1180E01D0080EE66ED1DFE55204
:103C70004FEF15F017ECD5F00DE0310E52ECCAF015
:103C80008BEC0BF0000902E0100E01D0000EE66E86
:103C9000BFDFE5524FEF15F0270E0101B95D02E1DC
:103CA00029EF1EF03AEF1EF0020199510101625D09
:103CB00018E062C199F26251020B05E1D051200B6C
:103CC00002E1000E01D0010E000902E0000E01D059
:103CD000380EE66E0F0EE66EC80EE66EA10E49ECCB
:103CE000CCF01200A7ECCCF0840E52ECCAF02A9271
:103CF000AEEC16F0E66A720E42ECCAF03C0EE66ECE
:103D0000710E42ECCAF0FEEC16F037EC19F04BECF9
:103D10000CF013EC09F0B8D8E6ECD6F0E66A130E16
:103D200042ECCAF0010162855C95BEDF9CEC4EF06E
:103D3000E668B30E42ECCAF03DD857EC4EF0DFEC2B
:103D40004FF0DDEC08F0F8EC15F0E5EC15F09BEC2D
:103D500015F044EC19F08EDF6EECCCF008DFC3EC0C
:103D600015F025EC19F0010EE66EF2DEE552A7EC37
:103D7000CCF00601B26B090EB36F6BDF01015F512E
:103D8000200B02E0640E01D0320EE66E1F0E42ECF4
:103D9000CAF0010EE66E0F0E42EFCAF01200046A7E
:103DA00001015FAF04D011BC048011BE04823CB994
:103DB00004841200010112983B51100B01E012889B
:103DC0003B51100B0FE02150020B0CE01E50200B5A
:103DD00009E0050ED45D06E0040ED45D03E0030E99
:103DE000006E06D031C100F01BECD5F001E0006A96
:103DF0000050E66EA60E42EFCAF0016A0701BEB39C
:103E000002D04BC101F04CC102F0BE51020B09E0DF
:103E10000101D45104E10601EA51010802E34DC158
:103E200002F00F0E0101D8804155E66E20ECDAF069
:103E30007DC1E6FF47C1E6FFA00EE66E80EC16F0FE
:103E4000496E060EE15E495070C1E6FF6E0E42EC0F
:103E5000CAF00701BEB10FD00101D2AD03D0D29D8F
:103E600057EC4EF01450100B06E01450200B03E1F9
:103E70001498DFEC4FF00701BE51010B02E0AE0ECB
:103E800001D0AD0E52EFCAF0FDEF1EF05FECD5F0A1
:103E9000B2ECCDF0000403E0020E005C08E1E66A3B
:103EA0003350040B02E0030E36D0000E34D0005025
:103EB00005E1010EE66E4CDEE55253D0050E005CC6
:103EC0002CE10E6A0F6A01015751080B0BE1E65114
:103ED000040B08E002018951040B04E0D00E0E6EC1
:103EE000070E0F6E06ECCCF08D0E0DECCAF0020141
:103EF0008951040B08E12050400B03E0330E875D2D
:103F000002E0000E01D0010E000902E0875101D04D
:103F1000000EE66E040EE66E26D0030E005C21E174
:103F20000AECCBF01EE0020E0A5C03E189ECD1F052
:103F300011D0E80E0E6E030E0F6E06ECCCF03E0EA6
:103F40000DECCAF0DF6A010196ABDF2ADFCFE6FF96
:103F5000020EE66E140E0DECCAF00501040E266F7B
:103F600005D0E66AE66A140E0DECCAF0E552E3EFFE
:103F7000C9F05FECD5F002012F6B0601BF6BBFC625
:103F8000BEF6329E0101D45124E10601EA51010836
:103F900003E31350010B17E0016AEA05EB6F020E11
:103FA000EA5D03E302011A5102E00601EB6BEBC686
:103FB000E6FF96ECD6F0E66A030EE66E120E0DEC06
:103FC000CAF0328E04D0E6ECD6F00601EB6B5CDF73
:103FD0005BD0030ED45D56E162991350010B06E1EC
:103FE00013ECD1F003E11FECD5F048E0AEECCDF0DE
:103FF0000AE02D0EDF6E010E016E026A13A015D0CD
:1040000002012F6F12D0C5ECD0F00DE0020E016E50
:10401000026A1F0EDF6E010196BB07D0010E026E11
:104020003F0EDF6E02D0016A026A20ECDAF0120E57
:104030000DECCAF0EDC6E6FF96ECD6F0328E13EC2E
:10404000D1F002E0010162890701200E516F3F0E9D
:10405000DF5C02E1100E516F640EDF5C02E10A0EBC
:10406000516F4B0EDF5C02E10D0E516F2D0EDF5CC8
:1040700002E1160E516F4E6B526B02D0E6ECD6F099
:1040800013DE02D0E6ECD6F06FEC39F0E552E3EF48
:10409000C9F0BF0E1CECDAF0E840E8403F0B005CD2
:1040A00002010B6F060E00C0E7FF070B04E0E742BA
:1040B000E79EE806FCE1E75002010B5F0B07640E88
:1040C0000B5D09E22150100B06E10101395103E1BA
:1040D0002188B9ECD9F00BC200F012001FB203D056
:1040E0000101D45112000101D55112000C0E52EC05
:1040F000CAF09BECCCF00E6E0F6AFF0E0E1804E1B6
:104100000F5002E10E680F681200416B426B436B67
:10411000446B400E456FD8903C373B373A373937C0
:1041200038373737363735374437433742374137F3
:104130004051445D3F5143593E5142593D514159CF
:1041400009E34051445F3F51435B3E51425B3D5167
:10415000415B3C2B452FE0D712000101D09711BEE7
:10416000D087D19911BCD18912008FECD1F0010117
:104170000490D051080B01E004800492D151100B3F
:1041800001E00482119E04B0118E119C04B2118CC6
:1041900007010A970A990A8504A00ED00101D0519F
:1041A00007010A99010B01E00A890101D0510701B9
:1041B0000A97020B01E00A870A51100B06E1010180
:1041C000775103E10450020B02E007010A95070151
:1041D0000A9104B20A81BEECC4F0CFEF1EF05FEC8E
:1041E000D5F025ECD9F0200E72ECD8F00050026E1C
:1041F0000F0E72ECD8F001012B51005C29E1250E65
:10420000025C26E1050E9DECD7F03AECCCF013E20F
:10421000010EE66E0A0EDF24E5ECD5F055ECCAF08F
:104220000F0E01010617D451065D05E0288206C174
:10423000D4F1C1ECCCF0BDECCAF007E1030EE66EA0
:10424000100EDF24E66E9DECD8F0096A010E02D054
:10425000096A000EE552E3EFC9F0E7ECC9F01EACC5
:1042600003D00201098102D00201068305014781C2
:1042700047872B8C2C8ADEECCBF0EE50ED1013E050
:104280000101442B640E445D03E2A9DF00091DE136
:1042900001014407FF0E445D03E0A1DF0009F8E1DE
:1042A0000101442B12D001014407FF0E445D03E0DD
:1042B00096DF00090AE10101442B640E445D03E22C
:1042C0008EDF0009F8E101014407E3EFC9F0E7ECF4
:1042D000C9F0290E496ED60E4A6E010E05ECDBF0D0
:1042E0007F0B006EFE0EDB50040806E1FD0EDB5076
:1042F000310802E2020E006E23ECD5F006E1FD0E5D
:10430000DB50310802E2040E006EE3EFC9F0040E48
:104310000101435D01E3436B395102E0190E04D002
:10432000160E43259CECCBF0006E0050E66EE66A5C
:104330003C0EE66EE0ECFBF068EFD5F02190020158
:10434000320E246F295102E0140E246FC80E366F0E
:104350001DAC2998D95102E0DDEC08F01D50400B4E
:1043600003E02A50800B02E1AEEC16F0020109874F
:104370000985098309817A6B0901EB6B1200E7EC6F
:10438000C9F0FE0EDB500EE029A006D0FE0EDB5079
:10439000030B02E17DEC07F0280EA9ECCDF0FE0E38
:1043A000DB06EFD7E3EFC9F011C512F50501106B7D
:1043B000279C0101E491120027BA09D013C549F1E5
:1043C00014C529F1249223BC24822FEC65F0278A9E
:1043D00001013699DDEC08F00201216B239A259248
:1043E000120055ECCEF0E0DF2750200B05E00AEC80
:1043F000CBF002E0080E076EDFDF2F98120027AA2D
:1044000002D00101E88B0750220A01E19ED1030A84
:1044100001E17FD1010A01E1EFD03F0A39E0010A51
:1044200001E0ADD1278C49C113F529C114F5239CB6
:1044300024B2238C27BA15D0010136AD11D0E7B7CD
:1044400006D03651070B050DF3500A0F496F640E65
:10445000296F36B902D0430E296F19EC65F001D0EF
:10446000C0DF1FECD5F007E0200E06014A5D03E037
:10447000200E32ECCDF01D901F0E076E02012D5163
:1044800001E17ED12750200B01E17AD1076A23D1C7
:104490000501105101E188D00AECCBF016E027505D
:1044A000200B13E00501235107E1020E265D0DE10B
:1044B00082EC0EF0000909E102012D5101E12D2BE2
:1044C000080E076E1F0E086E12000501100712512C
:1044D000EA6A000FE96E080EEA22EFCF02F7122B0C
:1044E000125182ECCAF002E638ECD4F001E3126B10
:1044F0000AECCBF00BE02750200B08E002C7E6FFE8
:104500006DEC3CF0E552200E076E12003C0E0701E8
:10451000025D04E12482238C229C32D13E0E025D96
:1045200006E12492239C1EBC2BD1228C29D1740E2F
:10453000025D01E125D10601EA510AE02750200B76
:1045400007E0298A02C7E6FF02EC70F0E552299ADB
:10455000800E0701025D0FE25B0E496EDA0E4A6EB5
:10456000010E4B6E200E025D71ECCDF0ECECC9F04B
:104570000800F5CF02F7800E025D03E10201040E90
:10458000526F07010251800805E2800E025DFD0FA7
:104590000201526F800E0701025D01E3B4D00251A7
:1045A00001E1EED0200ECFD027AAE9D010ECD2F056
:1045B00007E007010251800803E3200E32ECCDF042
:1045C00010DF0AECCBF005E0279C080E076E100EFA
:1045D000086E2750200B01E1D3D00201555101E1B3
:1045E000CFD0189A55BF188A196B010EE66E7F0E50
:1045F00055157CECD2F0C4D01750800B06E0275044
:10460000200B09E10B0E155C06E01D50040B03E0C6
:104610001D50080B58E12750200B09E01750800B64
:1046200006E05DECD2F003E00B0E155C1CE18CECB7
:1046300065F0D7DE209427AAA3D00AECCBF003E0E4
:104640000201010E2D6F1BECD4F00601EA5101E1CD
:1046500097D007010251800801E292D02F88200EE6
:1046600032ECCDF08DD0230E155C10E1010EE66E1C
:1046700093EC0EF0E5521EAC03D00201098702D084
:10468000020106810501478D179E7AD0B1EC96F0A4
:10469000000914E02750200B11E00C50006E020EB0
:1046A00098ECD0F00C50026E00500C6E0250E66E8A
:1046B000A6EC74F0E5520201196B62D027AA60D013
:1046C0001EEC99F05DD00AECCBF008E02750200BEF
:1046D00005E0080E076E1F0E086E52D0FE0E070191
:1046E00002150EE0228E010E016F02A102D0030E10
:1046F000016F02910243210E076E0501200E07D0C3
:104700000201020E526F220E076E05011F0E156F79
:1047100037D00701015112E00107238045EC65F015
:10472000076A1DA006D0020E076E27BA02D018EC49
:10473000CFF0210E086E1D80229E22D00201010EB4
:10474000526F228E220E076E1BD00201525114E0CE
:104750002390520745EC65F0030E076E1DB007D09D
:10476000070E076E27BA03D0006A7CEC75F0220EA4
:10477000086E229E1D9004D015C507F001D031DED1
:104780000101E89B1200020171510101D8804855D6
:1047900002E271C248F12B510A0825E2100E2B5D8E
:1047A00019ECCCF0060EF3ECDAF0016EE651040BD6
:1047B00013E01B50080B10E101501E0802E21E0E10
:1047C000016E6E0E02010B5D02E2140E016E5A0EB6
:1047D0000B5D02E20F0E016E01500101D8804855B9
:1047E00002E201C048F139512CE10A0E2B5D05E1CE
:1047F0004851640802E2640E486F02010B5182ECDA
:10480000CAF002E660ECD4F006E201014851640807
:1048100002E2640E486F640E02010B5D06E20101C4
:104820004851320802E2320E486F010148517808BF
:1048300008E2010E2B5D03E32B51050802E2780E1E
:10484000486F2150100B05E04851320802E2320E49
:10485000486F85ECCBF015E1010148511E080BE2D1
:10486000640E02010B5D0DE301014851320809E3BA
:104870000CECD3F006E001015FB309D05F83F6EFE3
:10488000C4F001015FA303D05F93F6ECC4F0120003
:10489000DACFE4FFE2CFDAFFE9CFE4FFEACFE4FFCB
:1048A000E652FC0EB36EF30EB26E02011107020166
:1048B000115105E10201320E116F01012181010147
:1048C000E7A92CD00601FD07000EFE5B0601FD5195
:1048D000FE1124E1F29EF26AF06AB96A9D6A000E46
:1048E000A66EA16E9E6E8D8C8D8A8C908494070E20
:1048F000936E0000000000008A9A00000000000093
:104900000000270E936E4E0E996E0000000000000E
:1049100003000000000000000000FF001E801D8654
:104920001D8481B20BD001014FA302D01E9006D08E
:1049300001014FA102D01D9601D01D9481B40BD06E
:1049400001014FA302D01E9006D001014FA102D059
:104950001D9401D01D9687B60BD001014FAB02D03C
:104960001E9006D001014FA902D01D9601D01D94C2
:1049700081B00BD001014FAB02D01E9006D00101D7
:104980004FA902D01D9401D01D9602011207020109
:10499000125137E10201050E126F0101B05116E00C
:1049A0000101B007020102015151020B05E01D5047
:1049B000040B02E102015181020102015151080B75
:1049C00005E01D50080B02E1020151850101B151C2
:1049D00006E0FF0E0101B15D02E00101B12B1FAE47
:1049E00004D00601DE2B000EDF230701505109E041
:1049F000070150070701505104E151C750F7010169
:104A000021830101AF5102E00101AF0701012697A7
:104A100001012695010126A102D00101268501018F
:104A200026A302D0010126870101269301012691C8
:104A300088A202D00101268188A002D0010126832C
:104A40000F0E010126150101236F01012351EA6AAE
:104A5000C50FE96E060EEA22EFCF22F1010E010129
:104A6000221513E01F50080B05E0010101013B5125
:104A7000010B0BE12050200B08E0010122AF03D015
:104A80000101240702D00101242B9EAA11D00701A5
:104A9000942B07019351932BEA6A000FE96E0C0ED9
:104AA000EA22AECFEFFF0701945102E192C793F7DC
:104AB000A19207014607E552E5CFEAFFE5CFE9FFFE
:104AC000E5CFDAFF110001013BAB07D03B9B238A06
:104AD0000601425102E0426B436B12000701BEB176
:104AE00003D0119A119812001198BEA31188119A3F
:104AF000BEB3118A12000B0E00ECCBF0258E120013
:104B0000A4ECCAF003E00AECCBF006E01394010138
:104B100056A30ED013840CD0139402013D5107E12B
:104B20000101E651800B03E13B51040B01E01384CA
:104B3000139613A4138613981350040B04E185EC09
:104B4000CBF001E013881200ECC1E9FFEDC1EAFFF0
:104B5000EECF49F0EECF4AF0EECF4BF0EECF4CF077
:104B6000EFCF4DF0EAC1E9FFEBC1EAFF49C0EEFF2C
:104B70004AC0EEFF4BC0EEFF4CC0EEFF4DC0EEFF53
:104B80001200E7ECC9F081ECCEF0FB0EDBCFECF1CC
:104B9000FC0EDBCFEDF10101A30EEA6F010EEB6F0E
:104BA000D3DFECEC31F0D850010B06E0FF0E010131
:104BB0009E5D02E0010E01D0000EE3EFC9F063EC50
:104BC000D5F00050E66E16ECFEF0E552140EE66EDF
:104BD00075ECFEF0E5528AECFEF085ECFEF0000983
:104BE000FCE1C450006E0050F80812E2C20410E06C
:104BF000050EC25C0DE0090EC25C0AE00D0EC25C3F
:104C000007E0110EC25C04E0390EC25C01E0000650
:104C1000020EE15C02E2E16AE552E16EE3EFC9F007
:104C20005FECD5F00050DF6E3C0E496ECE0E4A6E42
:104C3000010E0CECDBF00150006E009E0BECE2F07C
:104C400001AEF2D7E552E3EFC9F05FECD5F00050CA
:104C5000DF6E2350100B1DE10050E66E73EC04F084
:104C6000E552800B16E01B0EDF5C08E10101200E0F
:104C7000166F500E176F410E186F07D00101450EC9
:104C8000166F520E186F18C117F1200E196F040E0F
:104C9000016F2A8823A808D0380E496ED00E4A6EBC
:104CA000010E0CECDBF007D0DFCFE6FF73EC04F075
:104CB000E552016EDF2A2AA802D0019E2A980150EF
:104CC000006E009E2EECE2F001AEE4D72398E55290
:104CD000E3EFC9F0E1ECD6F003E200ECD3F004D04E
:104CE000FE0EDB50410FF60F006E0BECE2F0E3EF2F
:104CF000C9F0E1ECD6F003E200ECD3F004D0FE0EF4
:104D0000DB50410FF60F006E2EECE2F0E3EFC9F03E
:104D1000C2ECD9F0DFDFE5528FECD0F0DBDFE552FB
:104D2000E3EFC9F0C2ECD9F0E4DFE5528FECD0F04C
:104D3000E0DFE552E3EFC9F0E7ECC9F05BECD3F05C
:104D4000020E0101002780ECE1F0DF50006E050E3D
:104D50000101005F80ECE1F0030E0101005FE5520C
:104D6000E3EFC9F0E7ECC9F05BECD3F0FE0EDB50EB
:104D7000020F0101016F9DECE1F0DF50006EFE0EAD
:104D8000DBCF01F19DECE1F0E552E3EFC9F000C0AB
:104D900059F28EECDBF0FF0E005C01E041DF010117
:104DA000B589120000C05AF29EECDBF0FF0E005CE9
:104DB00001E04BDF0101B58B12008EECDBF0FF0E42
:104DC000005C01E02DDF0101B58D640EAC6F24960F
:104DD00012009EECDBF0FF0E005C01E036DF01010B
:104DE000B58F640EAC6F24961200E7ECC9F037EC77
:104DF000CFF00FECCCF07EECCAF0E3EFC9F0E7ECBB
:104E0000C9F037ECCFF095ECD5F0010EE66E5CEC16
:104E100008F0E552E552E3EFC9F0E7ECC9F0AFEC7A
:104E20006FF00101190EAE6FFC0EDBCFB2F1FD0E7B
:104E3000DBCFB3F1FE0EDBCFB4F1E3EFC9F0830EAD
:104E4000096EE00E73ECDBF0800E005C08E2AFEC64
:104E50006FF00101190EAE6F0201E00EA96F120092
:104E600083ECDAF0DBCF4AF0800E4A1407E0D7EC8F
:104E7000CBF0496C4A1E000E4A2202D0D7ECCBF090
:104E8000B0ECD9F0E3EFC9F0E7ECC9F012A60FD00F
:104E9000060150B503D00101E5ECCEF0288ABCBF75
:104EA000289AFE0EDB5001E0287A0BEC41F0E3EF8C
:104EB000C9F083ECDAF0DBAE08D0DB50FF0DFE0E5C
:104EC000F3CFDBFF31ECD1F007D031ECD1F0DB5088
:104ED000FF0DFE0EF3CFDBFFDB50E3EFC9F05FEC1D
:104EE000D5F007015A5101E05DD11D50400B01E0A2
:104EF00059D13250040B01E154D10101D45104E1E4
:104F00008450020B01E14DD10B0E97ECCBF0060162
:104F1000BC6FAEECCDF001E0A5D0140E0601E76E3B
:104F2000BC19E8AE02D0BC3503D0E750D880BC55E0
:104F300002E2140EBC6FEC0EE76EBC19E8AE02D0B4
:104F4000E73402D0E750BC5D02E2EC0EBC6FBE510C
:104F5000E76EBC19E8AE02D0BC3503D0E750D8806C
:104F6000BC5502E2BE2B0BD0BE51E76EBC19E8AEB9
:104F700002D0E73402D0E750BC5D03E2BE07BEC6F4
:104F8000BCF6200E496E4A6AC1C63DF0C2C63EF06C
:104F900062ECD3F03DC0C0F6C0C649F04A6A49BED3
:104FA0004A6849500601C15F4A50C25BBCC649F01D
:104FB0004A6A49BE4A684950C1274A50C223C0C6FE
:104FC000E6FF77DFE552016E010EE66E0E0E01245C
:104FD000ADECCCF002011A5101E1E3D01BAA05D0DF
:104FE000BCC6E6FFD7EC75F0E55281ECCCF02AE0C8
:104FF0001250080B03E1040E1A1528E000ECD6F05D
:1050000001E0010E496ED45103E1D051400B07E09D
:10501000D45103E0CF51040B02E0000E01D0010E89
:10502000491809E012A602D0E66A09D00601BC516F
:10503000010124270BD012A605D0010EE66E24DF55
:10504000E55204D00601BC510101245F0601BC51A8
:1050500001E0A7D002011A51320801E3A2D0320EBA
:105060001A6F9FD01B0EE66E33EC15F0E552F3CFAE
:10507000BCF6F4CFBDF6026A016A0601BC51E76EC8
:10508000BD19E8AE02D0BD3503D0E750D880BD557C
:1050900005E2BC51BD5DACECCFF0026E0601BD5126
:1050A000E76EBC19E8AE02D0BC3503D0E750D8801B
:1050B000BC5505E2BD51BC5DACECCFF0016E060104
:1050C000BF51D880025402E202C0BFF6BE51D88060
:1050D000015402E201C0BEF6000EE76EBF19E8AE51
:1050E00002D0BF3503D0E750D880BF5505E2010E8E
:1050F000E66E0D0EADECCCF0010E0601E76EBF19A9
:10510000E8AE02D0BF3503D0E750D880BF5505E2E6
:10511000010EE66E0C0EADECCCF0020E0601E76E51
:10512000BF19E8AE02D0BF3503D0E750D880BF55D5
:1051300005E2010EE66E0B0EADECCCF0000E0601A2
:10514000E76EBE19E8AE02D0BE3503D0E750D88076
:10515000BE5505E2010EE66E0F0EADECCCF0010E71
:105160000601E76EBE19E8AE02D0BE3503D0E750A7
:10517000D880BE5505E2010EE66E100EADECCCF007
:10518000020E0601E76EBE19E8AE02D0BE3503D0AE
:10519000E750D880BE5505E2010EE66E110EADEC6B
:1051A000CCF03294E552E3EFC9F063ECD5F0FC0E9D
:1051B000DB506AE102012A5167E10490FE0EDB50E8
:1051C000140804E2140E1BECCFF00480FE0EDBCFBB
:1051D00049F05651D880495403E2FE0EDBCF56F217
:1051E00001012A51100B03E0050ED45D05E10450C6
:1051F000010B02E0FE0EDB2A010E67C1DBFF050E8C
:10520000D45D02E1010EDB6A010EDB50280803E2E7
:10521000DE52280EDD6E050EDEECD0F03EC0DBFF68
:10522000DF6A150EDF5C22E2006AFE0EDB5004E04E
:10523000FE0EDB50DF5C13E301012A51100B07E087
:10524000050ED45D04E002015651DF5C08E0010167
:105250006751040806E2010EDB50DF5C02E1010E3B
:10526000006E0050EDECCEF0DF2ADBD71350010BBF
:1052700069E00201215166E10101D45103E0030E0E
:10528000D45D60E132845ED0FC0EDB0430E10201CB
:105290002A5106E0FD0EDB5003E12250400B55E1A0
:1052A00023ECD5F003E2080E1BECCFF0FD0EDB5033
:1052B0000C0805E20C0EF36EFD0EF3CFDBFF8EEC57
:1052C000CEF0150EDF5C3EE2FE0EDB5004E0FE0E7B
:1052D000DB50DF5C07E3090EDF5C07E3FD0EDB500C
:1052E000DF5C03E2010EEDECCEF0DF2AEAD7FC0E24
:1052F000DB50020827E123ECD5F003E2080E1BEC9B
:10530000CFF0FD0EDB500C0805E20B0EF36EFD0E28
:10531000F3CFDBFF8EECCEF0150EDF5C13E2FE0E5A
:10532000DB5004E0FE0EDB50DF5C07E3090EDF5CC0
:1053300007E3FD0EDB50DF5C03E2010EEDECCEF087
:10534000DF2AEAD7FE0EDBCF0AF2020EE15C02E2B0
:10535000E16AE552E16EE3EFC9F00101D551F4ECE9
:10536000CEF0CCECCCF00150080D4950F3240A01EA
:10537000DF6F4A50F420E06F12000101C951C45D93
:105380000CE1CA51C55D09E1CB51C65D06E1CC51C6
:10539000C75D03E1CD51C85D01E0000C010C0101C6
:1053A000D551D45D01E0000CD4510BE1D051400B3C
:1053B00001E0010E496EDD51400B01E0010E495C38
:1053C0002DE0030ED45D23E1DC5179ECCBF00A5CD7
:1053D0001EE1AEECCDF00CE00101D051040B01E078
:1053E000010E4A6EDD51040B01E0010E4A5C16E02D
:1053F000AEECCDF00CE10101CF51040B01E0010E48
:105400004B6EDC51040B01E0010E4B5C07E0010127
:10541000D45103E0030ED45D01E1000C010CADDFBB
:10542000000903E0BCDF000901E1000C010CF7DF1B
:10543000000928E0BDECCAF001E1010CD551F4EC03
:10544000CEF0080EE66EE66AD551F2ECD7F00150C8
:10545000A5ECDAF0D451100DF3CF4FF0F4CF50F0AB
:105460002A0E4F260A0E50220701B151080DB4EC46
:10547000CFF092ECFAF0516E060EE15E5150000949
:1054800001E1010C000C1AB202D0BFECCFF0D4C184
:10549000D5F134AA17D0010138A306D0DE93D1B3D9
:1054A000DE83DE95D1B5DE85DD9DD0BDDD8DDD955C
:1054B000D0B5DD85DC95CFB5DC8526ECDAF09DEC4A
:1054C000D6F01AD00101D55103E1DD9DD0BDDD8DAF
:1054D000030ED55D11E126ECDAF09DECD6F0AEECD2
:1054E000CDF006E00101DD95D0A506D0DD8504D024
:1054F0000101DC95CFB5DC8534AA0DD0500EE66EE7
:10550000E66A2A0EE66E0A0EE66E7A0EE66E0A0E5F
:1055100055ECCDF00FD0050ED45D0CE0100EE66E0C
:10552000E66A13ECDBF0D551F2ECD7F074ECD4F072
:1055300009ECCDF0050E0101D55D08E0D551EA6A10
:10554000CF0FE96E0A0EEA22B1C7EFFF1200C9C100
:10555000C4F1CAC1C5F1CBC1C6F1CCC1C7F1CDC13F
:10556000C8F1D5C1D4F134AA08D084ECD2F02A0E07
:10557000E66E0A0E55ECCDF014D0BDECCAF011E089
:10558000100EE66EE66ACCECCCF053ECCBF0D451C6
:10559000100DB7ECCCF04CECD4F074ECD4F009EC7A
:1055A000CDF0BDECCAF004E0FBECCDF0B1C7EFFFED
:1055B0001200E7ECC9F03BDF000916E103EC14F040
:1055C000FE0EDB5002E15FDF01D0C1DF15ECD2F04F
:1055D000248A1EAC04D002010983098102D0020191
:1055E0000683050147834781E3EFC9F003EC14F01C
:1055F0000101C4510CE0C40503E13C0EC55D07E3A5
:10560000C95105E0C90514E13C0ECA5D11E22DEC5B
:10561000CDF0348A10D8349AA7EC13F01C8A2DEC04
:10562000CDF01C9A188420ECCFF0189495EFD1F0AF
:1056300002D8A7EF13F00DC103F0C9C19AF2CAC195
:105640009BF2CBC19CF2CCC19DF2CDC19EF2D5C1E3
:1056500000F079ECD4F0DEC1E2F134AA08D084EC99
:10566000D2F0540EE66E060E55ECCDF011D0050EBC
:10567000005C0EE0100EE66EE66A0101CCECCCF0A8
:1056800053ECCBF0540EE66E060EE66E65ECD3F0EE
:10569000016A050E005C03E00050F4ECCEF0F3DE8E
:1056A00003C00DF19AC2C4F19BC2C5F19CC2C6F100
:1056B0009DC2C7F19EC2C8F100C0D4F134AA1ED069
:1056C000010138A30ED0D193E2B3D183D195E2B5D5
:1056D000D1851296D1B312861294D1B51284A4EC5E
:1056E0009AF00101D09DE1BDD08DD095E1B5D08576
:1056F000CF95E0B5CF8563ECD6F018D00101D45139
:1057000003E1D09DE1BDD08D030ED45D0FE163ECCC
:10571000D6F0AEECCDF006E00101D095E1A506D0C3
:10572000D08504D00101CF95E0B5CF8534AA09D04A
:10573000500E6CECD3F02A0EE66E0A0E55ECCDF04E
:105740000AD0050E005C07E0100E6CECD3F013ECF1
:10575000DBF065ECD3F001C0B1F7BDECCAF004E0BA
:10576000FBECCDF001C0EFFF04903BB104803B9116
:105770003BB33B813B9304B03B83129C3BB1128C07
:10578000129E3BB3128E15ECD2F0248AB5DB1EAC10
:1057900006D00201098709850983098102D0020127
:1057A000068305014881BF0E476F1200E7ECC9F080
:1057B0000101628554EC1EF0E3EFC9F0370E005C86
:1057C00002E2370E006E00509F0802E29F0E006E4C
:1057D000630E005C08E2370E005CE824496E090E97
:1057E000E1ECCAF005D0630E005C33ECD8F0090F91
:1057F000006E0201D05102E0030E00260050150891
:1058000002E2150E006E1200A9ECD6F00201215141
:1058100010E12050010B0DE124510BE13250100B2F
:1058200008E12750200B05E0D85103E130A003D058
:105830003090000E70D0FE0EDB5002E0990E01D0C9
:105840000A0E97ECCBF085ECD0F08C0E7EECD4F009
:105850000201D05103E0790E7EECD4F02C5129E105
:10586000020EDB5065ECCCF024E30A0E97ECCBF093
:10587000496E020EDB50495C1CE311AE0DD0119E47
:10588000ADEC20F00201068D090E9FECCAF073EC1E
:10589000D3F027ECD5F00DD00201D05107E107017C
:1058A0000A93BEECC4F043EC53F011840201FA0EEB
:1058B000D06F010EDB50006E00509F0802E29F0E79
:1058C000006E00504B6E4C6A05011851070D79ECC3
:1058D000D3F0030E0F0B03E094ECD0F0FDE149C0D0
:1058E00018F56CDF0050DF6E00C0A2F7090E016EE4
:1058F00001012AB901061350010B06E00150D880BE
:10590000005402E20150006EE66AE66A0050E66E5C
:1059100040ECCEF0DF50496E030EE15C02E2E16A3A
:10592000E552E16E4950E3EFC9F085ECD5F0020B8A
:105930001CE00101E651400B18E00201685115E13D
:10594000080E155C06E0290E155C03E00A0E155CD6
:105950000CE1080E155C02E1010E20D0290E155C49
:1059600002E1020E1BD0030E19D0016A0A0E015C7F
:1059700019E2FE0EDB50010B06E0230E012478EC49
:10598000CCF0155C0AE0FE0EDB50020B09E02D0E98
:10599000012478ECCCF0155C03E101500C6E02D0D0
:1059A000012AE4D7E3EFC9F0E7ECC9F0800E0C6EF2
:1059B00017AE17D0179E1750010B03E11750100BAD
:1059C00010E0100E0C6E95ECD5F0AFDFE5522C0E0A
:1059D000155C02E1200E0C6E0B0E155C02E1400E10
:1059E0000C6EE3EFC9F0E7ECC9F0CAECCFF095EC30
:1059F000D5F027EC0CF0E55240ECD8F00101A86F8F
:105A0000A851640DB8ECCAF03BECD8F05C0F9CECEC
:105A1000CBF0006E32ECD7F080ECD3F000504B6E40
:105A20004C6A01014B50495CD86F4C504A58D96FB1
:105A300029A60BD09E5180ECD3F00101D851495CCE
:105A40000E6ED9514A580F6E06D09E510F6AD82556
:105A50000E6ED9510F2200ECD5F053ECD6F03DC0BC
:105A6000A8F139C09EF1E3EFC9F0E7ECC9F0CAEC48
:105A7000CFF0DB5019ECCCF0030EF3ECDAF00101BF
:105A8000A85D02E0000E1BD0FE0EDB5019ECCCF03E
:105A9000020EF3ECDAF09E5D006E00BE006C040EA8
:105AA000005C0AE3AEECD6F009E0945107E0A8519F
:105AB00005E0190E005C02E2010E01D0000EE3EFDA
:105AC000C9F0010EE66E70DFE55200680A0E0C5C4C
:105AD00002E20C501DD0200E0C5C02E10E0E18D01C
:105AE000400E0C5C02E10F0E13D0100E155C02E1AB
:105AF0000A0E0ED0180E155C02E10B0E09D0110E25
:105B0000155C02E10C0E04D0190E155C02E10D0EBD
:105B1000006EFF0E005C1DE00050E66E8E0E42EC43
:105B2000CAF0300EE66E8F0E42ECCAF0C80E16ECCC
:105B3000CAF017A808D09BECD1F0000904E0140EBD
:105B400016ECCAF0F8D7E66A8F0E42ECCAF0179E40
:105B5000010C000C75ECD8F0920E491810E14A5077
:105B60000EE1006AC7EC26F0B80E61ECD2F001013C
:105B7000AC6B21860201776B696B289E072A75EC56
:105B8000D8F0930E49185CE14A505AE1010EE66ED6
:105B90000BDFE5520A0E0C5C32E202017751050878
:105BA00033E36951020830E3772B28BE692B010EDD
:105BB000016E070E015C13E2012804ECCBF0EF50FC
:105BC000006E060E015C05E1800E010115150C103A
:105BD000006E79ECD8F000C0EFFF012AEAD701018E
:105BE000159F36AD2DD00C5002E1540E02D0300E70
:105BF0000C24006E800E001025ECCFF010D0200E8B
:105C00000C5C12E128AE02D0258E1AD0288E01013C
:105C1000158FD20E25ECCFF0010136AD11D0050164
:105C2000930E4B6F1E0E0BD0400E0C5C04E1980ED1
:105C3000076E1A8805D0100E0C5C02E19A0E076EF2
:105C400075ECD8F0980E491801E077D04A5075E10C
:105C5000010E016E070E015C0DE279ECD8F0EF9EAB
:105C600079ECD8F0EF500E0803E179ECD8F0EF6A48
:105C7000012AF0D70FC1A8F10A0E01011003F35059
:105C800011259E6F0A0E1203F35013259F6F0A0E03
:105C90001403F3CFA0F1A26BA2C1A1F1040E020183
:105CA000775D0DE269510BE112C1A8F10A0E010105
:105CB0001303F35014259E6FA06BA0C19FF1020146
:105CC000690508E111C1A8F19FC19EF1A0C19FF132
:105CD0000101A06B020E0201695D0EE110C1A8F185
:105CE0000A0E01011103F35012259E6F0A0E1303D1
:105CF000F35014259F6FA06B9A0E076EE2EC0CF028
:105D0000006E005013E10101A85103E19E513808D3
:105D100002E2258E1200DFECCDF00A0E005C06E1F7
:105D20000101E351010B02E006EF09F000C02BF185
:105D3000298420ECCFF09EEC21F075ECD8F09A0E7F
:105D4000491808E14A5006E10101B59BB59903D80D
:105D50000C0E076E120083ECD4F02582238A120009
:105D60003EC2A7F13FC2A6F140C2A5F10101A46B5A
:105D7000A36B1FA402D0C8EF31F0ECEF31F0049018
:105D80002C50100B01E004807FECC5F02C50100B60
:105D900001E0010E496E0450010B495C02E02AEC5F
:105DA000CFF01200F7ECDAF001018DA715D0FE0E4E
:105DB000DB5008E0FD0EDB5005E1DF68CFA102D02B
:105DC000010EDF6EFE0EDB5007E1FD0EDB5004E03E
:105DD000010EDF6ECFB1DF68DF5021E015ECCBF0B4
:105DE000A76BA7C1A4F1A7C1A3F1C6ECD9F001E04C
:105DF000010E496EDF0402E0000E01D0010E4918C9
:105E000002E0C6DA01D0E8DA7CEC04F01EAC03D084
:105E10000201098102D00201068305014781E55292
:105E2000E3EFC9F00101A76BA66BA56B02018851D6
:105E3000E824496E640EF7ECD7F05AECFEF03AC055
:105E4000A4F1320E28ECD6F088C23EF05AECFEF0F7
:105E50003EC0A3F1020189A102D0C8EF31F0ECEFFE
:105E600031F0B2ECD6F09AC23BF03C6A3D6A3E6A31
:105E7000FCECCEF019ECFCF037C0DEFF38C0DEFFE2
:105E800039C0DEFF3AC0DDFFDD52DD529BC249F072
:105E90004A6A4B6A4C6A100E406E270E416ED2EC75
:105EA000CAF0D5ECCCF09CC249F04A6A4B6A4C6A05
:105EB000640E406E416AD2ECCAF0D5ECCCF00A0E0A
:105EC00002019D03F3509E25496E4A6A4B6A4C6A53
:105ED000D5ECCCF0DECF3BF0DECF3CF0DECF3DF0BA
:105EE000DDCF3EF0DD52DD52040EE15C02E2E16AFC
:105EF000E552E16EE3EFC9F007AE6ED02B50400BD8
:105F000003E02C50200B31E0800E0101C41505E1A7
:105F1000C4510CE11F0EC55D09E2C46B1F0EC56FB5
:105F2000C86BC8C1C7F1C8C1C6F11FD0100E2B5D28
:105F30001CE2360E006E0050C45D03E300C0C4F1E5
:105F40000DD0200EC45D11E32C0EC45D0EE2260EB2
:105F5000C45D02E2200E01D02C0EC46FC86BC8C114
:105F6000C7F1C8C1C6F1C8C1C5F12B50400B03E051
:105F70002C50200B31E1800E0101C91505E1C951FA
:105F80000CE11F0ECA5D09E2C96B1F0ECA6FCD6B13
:105F9000CDC1CCF1CDC1CBF11FD0100E2B5D1CE2D9
:105FA000360E006E0050C95D03E300C0C9F10DD08C
:105FB000200EC95D11E32C0EC95D0EE2260EC95DEF
:105FC00002E2200E01D02C0EC96FCD6BCDC1CCF1F9
:105FD000CDC1CBF1CDC1CAF12B50400B03E02C5009
:105FE000200B1DE02050400B03E11250080B0FE185
:105FF0002050400B12E01F50020B03E11250040B23
:1060000006E11F50020B09E01250080B06E015ECE8
:10601000CBF0A6DED5ECCFF002D0E0ECCFF02B50E9
:10602000400B03E02C50200B16E11F50020B11E037
:106030001250040B0EE0E0ECCCF092DE9EC1BFF1FA
:106040009FC1C0F1A0C1C1F1A1C1C2F1A2C1C3F100
:1060500002D0EBECCFF01F50020B18E10201895186
:10606000010B03E18951020B11E0BDECCAF006E01F
:106070002050800B0BE0050E9D5D08E12050400B89
:1060800005E0EBECCCF0CEDED5ECCFF001013BA986
:1060900074D0BAC19AF2BBC19BF2BCC19CF2BDC123
:1060A0009DF2BEC19EF2DDDE3BC0C8F73CC0C9F721
:1060B0003DC0CAF73EC0CBF7BFC19AF2C0C19BF248
:1060C000C1C19CF2C2C19DF2C3C19EF2CADE3BC0F7
:1060D000CCF73CC0CDF73DC0CEF73EC0CFF70701AF
:1060E000C851CC5FC951CD5BCA51CE5BCB51CF5BA0
:1060F0000101D2A108D0400E0701CC271F0ECD23ED
:10610000000ECE23CF23049C1E50200B01E0048CF4
:10611000D8800701CF51FF0A08E6680ECC5DC50E96
:10612000CD59FF0ECE59FF0ECF5919E3CF35000ED2
:10613000CF1909E6D880980ECC553A0ECD55000EF1
:10614000CE55000ECF550BE3CCC70EF0CDC70FF0E8
:1061500006ECCCF0A50E0DECCAF01E8A01D01E9AFA
:106160000450400B01E0010E496E1E50200B01E06F
:10617000010E495C02E073ECCCF02BAC96D0800EA3
:10618000071401E192D0100E01012B5D01E38DD0C7
:106190002CBA0DD0F6ECCFF0C9C1A3F1CAC1A4F15D
:1061A000CBC1A5F1CCC1A6F1CDC1A7F10CD0EBECD0
:1061B000CCF0C4C1A3F1C5C1A4F1C6C1A5F1C7C14A
:1061C000A6F1C8C1A7F1DFECCDF02C50200B2EE0DA
:1061D000005001012B5D2AE000C00DF100C02BF141
:1061E0002BC1D3F187ECD3F004ECCFF0056E2CAAD1
:1061F00006D0050EE66E052419ECD2F005D0050E8A
:10620000E66E05509DECD0F055ECCAF00E0E05245C
:10621000ECECCBF00101D29B00BAD28B096AFCEC0A
:1062200035F020820201010E246F01D0A8DD0701A4
:10623000C2510101C45D04E0BDEC0DF0C4C1C2F760
:1062400001012B5132E12B50080B2FE0020E3A5D79
:106250002CE15AECD7F004E055ECD2F0E806FCE172
:106260000701C6510E1802E1C7510F181EE0006A5F
:106270005A0E0E1807E10F5005E1590EC61901E13B
:10628000C7510AE0590E0E1808E10F5006E15A0EE8
:10629000C61903E1C75101E1002A0EC0C6F70FC0BD
:1062A000C7F70050E66E02D8E5521200E7ECC9F0DD
:1062B000010139516BE12B5169E12B50080B66E06C
:1062C000FE0EDB5003E1020E3A5D60E15AECD7F0BE
:1062D00004E055ECD2F0E806FCE10EC0C6F70FC0B2
:1062E000C7F7190EC1ECD0F003E2036802681DD0B5
:1062F000410EC1ECD0F015E257ECD6F0190E495E14
:10630000000E4A5A4950016E2CECD6F00800F550A8
:10631000026E2CECD6F0F62AA2ECD0F0F550036E0B
:1063200004D069C302F06AC303F0010196A904D046
:1063300069C302F06AC303F0FE0EDB5007E10701F8
:10634000C351025C03E1C451035C20E002C0C3F707
:1063500003C0C4F7410EC1ECD0F011E20101965127
:10636000100B0DE1010EE66EE66A0350E66E025078
:10637000E66E09ECCEF00B0E1EECD2F005D0FE0E50
:10638000DB5002E08DECD3F08FECD1F0E3EFC9F0FD
:106390000101A751A227A251090803E20A0EA25F38
:1063A000A12BA651A127A151090803E20A0EA15F62
:1063B000A02BA551A027A051630803E2640EA05FA3
:1063C0009F2BA4519F279F51630803E2640E9F5F98
:1063D0009E2BA3519E2712000101A751A25FA2513B
:1063E0000A0803E20A0EA227A107A651A15FA15144
:1063F0000A0803E20A0EA127A007A551A05FA05139
:10640000640803E2640EA0279F07A4519F5F9F5179
:10641000640803E2640E9F279E07A3519E5F12004B
:106420000101E6A536D0E5A902D0310E01D05E0EFD
:106430009E2701ECD0F015DDE8ECCDF0030E45EC25
:10644000D8F031ECD9F037ECD9F03BC09EF13AEC02
:10645000D1F0CEECCBF0100E406E270E416E426AAA
:10646000436A2FECFDF03BC09FF137C00EF038C0FF
:106470000FF000ECD5F053ECD6F03DC0A0F18CEC61
:10648000CAF039C03EF05AECFEF03EC0A1F13AC06D
:10649000A2F1120063ECD5F02BBC03D01AD82F9ECA
:1064A00010D02CAA07D02050400B0AE01F50020B3E
:1064B00008E106D02050400B04E01F50020B01E021
:1064C00008D8020EE15C02E2E16AE552E16EE3EF18
:1064D000C9F063ECD5F00101E851010BDE6EDD6A15
:1064E0001F50020B06E02050400B03E0F6ECCFF00B
:1064F00002D0EBECCCF0A76BA7C1A6F1A7C1A5F128
:10650000A7C1A4F1A7C1A3F120ACE8912050400B92
:1065100010E1D4510EE1C6ECD9F001E0010E95EC8A
:10652000CDF002E0000E01D0010E491801E081D04B
:106530007CD02050400B12E03450400B0FE0C6ECF2
:10654000D9F001E0010E496E020ED45D02E0000EAA
:1065500001D0010E491801E189D06BD02050400BC9
:1065600019E1D40503E0020ED45D14E187ECD4F008
:1065700011E201010F0EA56FE651040B01E0010EBF
:10658000496E020ED45D02E0000E01D0010E4918E2
:106590004CE04FD010ECD3F014E00101090EA56FD0
:1065A000010EA66F050EA76FE651040B01E0010E68
:1065B00095ECCDF002E0000E01D0010E491835E057
:1065C00038D02050400B13E1C5ECD0F010E00101B1
:1065D0000A0EA56FE651040B01E0010E95ECCDF01B
:1065E00002E0000E01D0010E49181FE022D0205019
:1065F000400B21E1BDECCAF003E0040ED45D1BE1C9
:10660000010EA46F140EA56F040ED45D03E1E6A580
:1066100010D00BD0E651040B01E0010E496EE5519C
:10662000800B01E0010E491804E0D6DE0101E8818B
:106630001ED0AEDE1CD02050400B19E0BDECCAF0DD
:1066400016E1A46BA4C1A3F1A56B5751080B0AE195
:10665000E651040B07E002018951040B03E001013C
:10666000140EA56F0101A76BA7C1A6F1B5DE01014C
:10667000E651010B2DE02050400B2AE1020114519C
:106680001DE00101E851010B496E4A6ADF504918CB
:1066900013E1DE52DD504A180FE10201A051010161
:1066A000A45D0AE10201A1510101A55D05E102011C
:1066B000A2510101A65D02E005014785A3C19FF239
:1066C000A4C1A0F2A5C1A1F2A6C1A2F2A7C1A3F2E2
:1066D00049ECD2F015E02050400B12E1050ED45DDC
:1066E0000FE0040ED45D0CE0A36BA46B500EA56FFD
:1066F000A76BA7C1A6F1E6A502D04ADE01D06CDEE9
:106700000101E6B58DDE73ECCEF01BE2100E2B5DC1
:106710002EECCFF00101A46BA4C1A3F1CAECD9F017
:10672000A56FCFECD9F0A66FA76BE651040B01E083
:10673000010E496ED4ECD9F0491802E04DDE01D0CB
:1067400027DE010196B374D057A943D057AB70D060
:10675000D2C70EF0D3C70FF0260ED8800E54020E0B
:106760000F5406E20480260E0E5E020E0F5A06D06B
:106770000490260ED8800E56020E0F569F51496E79
:106780004A6A9E51640DF3504924D86FF4504A2050
:10679000D96FD8C14DF0D9C14EF0A9ECCBF037C0BC
:1067A0003BF038C03CF039C03DF03AC03EF0880EB6
:1067B000406E130E416E426A436A2FECFDF03BC0FF
:1067C0000EF03CC00FF043ECCDF004A030D004DE5E
:1067D0002FD09EC100F0000405E19F51310802E274
:1067E000020E006E030E005C05E19F51310802E2CB
:1067F000040E006E98514F6E506A00504D6E4E6AF6
:106800000A0E4B6E4C6AB2C23DF0B3C23EF0BAEC17
:10681000DAF000ECFEF052ECDBF0A8ECCFF04FC069
:1068200042F050C043F010ECCDF043ECCDF0B0DDC1
:1068300081ECCCF003E1F8ECD2F019E00601F05164
:106840000101A05D14E10601EF5101019F5D0FE11F
:106850000601F1510101A15D0AE10601F2510101B8
:10686000A25D05E10601EE5101019E5D0CE09EC1B5
:10687000EEF69FC1EFF6A0C1F0F6A1C1F1F6A2C1FC
:10688000F2F6F4ECC5F0020EE15C02E2E16AE552D8
:10689000E16EE3EFC9F0D9CFE6FFE1CFD9FFBAC18E
:1068A0009EF1BBC19FF1BCC1A0F1BDC1A1F1BEC1B0
:1068B000A2F10101A86BFE0EDB500A0807E229963F
:1068C000FE0EDBCFE6FFF3EC2CF0E5520101006B8E
:1068D000800E01011315036E800E01011015026E6A
:1068E000010EEA6E9E5105D89F5103D8A05101D8E0
:1068F00014D0076B066F0A0E065DD8A003D0066F92
:10690000072BF9D700510E0FE96E0751EF6EE92AF8
:106910000651EF6E002B002B000CA1C114F1A2C197
:1069200015F10101A85107E10A0E01019E5D03E284
:106930000101100E0E6F0701BEBB03D00101100E46
:10694000156F0701BEAD05D00101100E146F14C103
:1069500015F11DBC03D00101108F03D002500101BD
:1069600010130101138F0101A85109081AE2020155
:10697000365117E08EECDBF00101020E006F9EC174
:1069800000F080ECE1F0A8C100F00101006B80ECA8
:10699000E1F0010EE66EE66A29EC09F0E552E552F7
:1069A00023D00101A8511FE007010701BE51200BB0
:1069B0001AE1288C14C115F113C114F112C113F19D
:1069C00011C112F110C111F10FC110F10EC10FF17F
:1069D0000A0E496E49C043F0A8C13EF05AECFEF0E1
:1069E0003AC00EF101D0289CE552E7CFD9FF120042
:1069F000D9CFE6FFE1CFD9FF020EE126010EA8C1F3
:106A0000DBFF2BC1DFFF0101D551EA6AB80FE96E48
:106A1000070EEA22EFCFBFF7BFC19EF1C0C19FF1C1
:106A2000C1C1A0F1C2C1A1F1C3C1A2F10101A86B12
:106A3000DF500A0806E22996DFCFE6FFF3EC2CF0E0
:106A4000E5520101016B800E01011B15026E010E62
:106A5000EA6E9E5105D89F5103D8A05101D816D097
:106A6000076B066F0A0E065DD8A003D0066F072BD2
:106A7000F9D70151160FE96E0751300FEF6EE92A71
:106A80000651300FEF6E012B012B000C300E01016F
:106A9000A12501011C6F0101A85107E10A0E0101A6
:106AA0009E5D03E20101200E166F0701BFAD03D00A
:106AB0000101200E1C6F0101188F01011B8F0101C4
:106AC000A8511DE007010701BF51200B18E11BC1B0
:106AD0001CF11AC11BF119C11AF118C119F117C122
:106AE00018F116C117F10A0E496E49C043F0A8C14A
:106AF0003EF05AECFEF03A50300F0101166FA8C17B
:106B0000A9F1010EDBCFA8F1020EE15C02E2E16A1D
:106B1000E552E16EE552E7CFD9FF12005FECD5F008
:106B2000830E096E0A0EE66E01010D03F350E66E48
:106B30005E0EE66E020E55ECCAF0DE0EECECCBF00B
:106B40000050DF6EFE0E73ECDBF00101E59D2E9E22
:106B5000B90E005C16E1FF0E02015E5D12E02E8EA2
:106B6000020E01012B5D0DE1050E0201635D09E1DD
:106B7000210E5F5D01E1606B280E645D02E13C0E59
:106B8000656FA30EDF5C02E10101E58DE552E3EFE5
:106B9000C9F08C0E02018D1909E10A0E8E1906E169
:106BA0008C0E8F1902E10A0E901907E0800E8E15E7
:106BB00004E1800E901501E1000C010C02019151DD
:106BC00002E1925107E0FF0E915D04E0FF0E925D3D
:106BD00001E0000C010C2B50080B0DE000ECD6F08E
:106BE0000AE12B5106E1010EE66E56EC31F0E5525A
:106BF00012008DECD3F0120018B03DD00DC1E6FFAD
:106C0000CCEC5AF0E552C5DF000902E0E7ECD0F029
:106C10000DC1E6FFE8EC5AF0E552D0DF000903E0D1
:106C20000201916B926BF8EC15F078DF010156517F
:106C3000080B03E12B51090809E2FF0E02018A5DEE
:106C400002E1320E8A6F8AC248F108D0FF0E8C5DD5
:106C500003E1320E8C6F02D08CC148F1C1EC41F0DF
:106C600001015F8DE6B55F9D07ECC4F06EECCCF0E2
:106C700001ECD2F0B0DF15EFD2F05FECD5F0FD0EF5
:106C8000DB50100DF350DF6E010E096E0201680E2D
:106C9000986FFD0EDB500A080AE2020E096E690EBB
:106CA000986FFD0EDB50F00F100DF350DF6EFE0EEF
:106CB000DB50FF0802E064ECD7F0DF50E552E3EF71
:106CC000C9F00201875103E08751330802E20D0E3B
:106CD000876F885158ECCBF007E24950FA08000E54
:106CE0004A5402E21E0E886F89BF896B93510E08C9
:106CF00003E2936B0101D09B1200A5ECD6F0FF08D4
:106D00001BE064ECD7F00F0E72ECD8F00A0E005CBA
:106D100007E10101E351010B03E0096A000EB9D15B
:106D200000C02BF101018A51100B06E00A0E6DEC38
:106D3000CAF002E2FE0EDB682BC10DF10201756B99
:106D40000101E695E5992B510A0838E2100E2B5DFA
:106D5000006E005014ECD7F029E03BECD8F00101B4
:106D60000D6F1BECCAF0EF380F0B0201756FAEEC24
:106D7000D6F024E01B50020B0EE02B50080B03E171
:106D80002250080B08E00101E68532ECD7F04608F6
:106D900015E1E58913D00701020E266F1BA202D070
:106DA000050E266F180E20ECCBF008D0FE0EDB6827
:106DB0000101090E0D6F0DC12BF1258E0101E6A514
:106DC0000FD02BA605D007011397140E8CECD4F02E
:106DD00022A603D0010E8CECD4F00701149F0FD033
:106DE0002BA605D007011387140E1EECD2F022A6A5
:106DF00003D0010E1EECD2F00701148F149377EC30
:106E0000D5F0010191ECD4F001E0098FE1ECDAF06A
:106E100007010B890101E6A502D007010B99BCEC23
:106E2000C4F00201D86BBBECCBF0100E9DECD7F098
:106E300029A403D07CEC04F029940F0E0101CE1597
:106E4000D46FCE390F0BD56FD551060802E2D4C1ED
:106E5000D5F1D40501E1CF91020ED45D01E1CF81DE
:106E600026ECDAF00A6E040EE66E0B0EDF24E66EF8
:106E7000DC0EE66E010E55ECCAF0BBECCBF0FE0E5C
:106E8000DB50FF0803E198C209F002D0100EDF26A4
:106E9000100EFBECDAF09DECD8F0FE0EDB50FF0894
:106EA00052E004ECCFF0DF6E0B0E72ECD8F03AEC4F
:106EB000CCF008E01F0ECF17E00E0014CF1326EC25
:106EC000DAF00A6E0C0E72ECD8F0440E0101D01705
:106ED000BB0E0014D01329ECDAF0470E0101D117D4
:106EE000B80E0014D11329ECDAF09E0E0101D2176E
:106EF000610E0014D21398C209F00A0EE66E030E5A
:106F0000DF24E66E8A0EE66E020E55ECCAF004EC43
:106F1000CFF0DF6E0C0E72ECD8F0440E0101DD17DD
:106F2000BB0E0014DD1329ECDAF0470E0101DE1769
:106F3000B80E0014DE1329ECDAF09E0E0101DF1703
:106F4000610E0014DF13096AC4C119F5C5C11AF531
:106F5000C6C11BF5C7C11CF5C8C11DF5C9C11EF5C9
:106F6000CAC11FF5CBC120F5CCC121F5CDC122F599
:106F700018B41CD012941296129A1F92010138A3D1
:106F80000CD0D1A102D0128A1F821296D1B31286E0
:106F90001294D1A509D0128407D040ECD3F001019E
:106FA000DE95DE93D195D193A4EC9AF073ECCEF0FC
:106FB0003DE25C0E0D259CECCBF0006E0050010113
:106FC000C45D016E01AE03D0C451005C016EE65198
:106FD000040B03E10150030803E3015019080AE21E
:106FE000050E17ECD1F0C40EE66E010EB3ECCAF03C
:106FF00000C0C4F100500101C95D016E01AE03D0B3
:10700000C951005C016EE651040B03E10150030815
:1070100003E3015014080AE2050E17ECD1F0C90E83
:10702000E66E010EB3ECCAF000C0C9F123ECD2F059
:1070300080EC25F04FEC0DF0129C01013BB1128C5D
:10704000129E3BB3128E92EC64F0129801013BB990
:107050001288B5EC20F00101D09F1190118267ECED
:1070600009F09CEC4EF057EC4EF0096A010137A78D
:1070700002D038EC48F0E0ECCFF0EBECCFF0BCDD28
:107080000101246B1DBC04D00701A16B87ECD3F078
:10709000010EE552E3EFC9F05FECD5F00B0E0101F4
:1070A0002B5D11E2C5C1E6FFC4C1E6FF67EC21F02C
:1070B000E552E552005001012B5D05E00701020E8B
:1070C0001FECD7F06ED00A0E2B5D02E248C18CF1A6
:1070D000BBECCBF0ADEC20F00101D09F38A30DD07C
:1070E000F80ED117D1911FB2D181D19312B6D183AD
:1070F000D19512B4D185F3EC40F02BC1D3F16DECF6
:10710000D7F0050E9DECD0F0FBECDAF04DECCAF0B8
:107110000A0EDF24016E0101D539F00BD411CDEC3C
:10712000D0F0050EE66ECF0EE66E010EE66E0B0E8B
:10713000DF2481ECD6F0050E19ECD2F0E66E050ED8
:10714000DF2481ECD6F01CBA24D0BBECCBF00101DB
:107150005651080B03E12B51090802E248C18AF29B
:107160005AECBCF03AC18BF2FE0EDB50FF0803E193
:1071700098C209F002D0100EDF26100EE66E870EC0
:10718000E66E020EFBECDAF04DECCAF0096A03EC95
:1071900014F0010137A702D076ECCFF0096A0201A2
:1071A000206BE552E3EFC9F05FECD5F00F0EDF6E18
:1071B000F40E06010017F00E0517DF500617E55212
:1071C000E3EFC9F00601069100950191029901993A
:1071D00014991399049903911200E7ECC9F000EC9B
:1071E000D6F001E0010E496EFE0EDB5002E0000E0B
:1071F00001D0010E491803E00601058502D0060101
:10720000058701018AA102D00601068DE3EFC9F0CE
:107210000050050A4FE0010A4AE0070A22E0010A8D
:107220001BE0030A17E0010A01E0120006010583D2
:1072300000ECD6F001E0010E496ED051400B01E0A8
:10724000010E491802E0060105810601EA5146E0F7
:10725000068B1200E66A02D0010EE66EBEDFE55232
:1072600012000601008100ECD6F001E0010EF1EC05
:10727000D0F002E0060105810A5003E0030E0A5C2B
:1072800002E1060105711FECD5F002E00601068B54
:1072900032A024D000ECD6F001E0010EF1ECD0F0E9
:1072A00003E00601058712000601058512000601AC
:1072B000008312000601008702018951040B04E0DB
:1072C0003A5102E10601068B020189A102D00601B2
:1072D000068D020189A302D00601068F1200800EDE
:1072E000071406E02050010B03E1D4C100F003D0E5
:1072F0006EEC20F0006E58DF08EF39F01200E7EC7A
:10730000C9F03AECCCF00DE10A0403E0020E0A5C8D
:1073100004E1D051040B16E10BD0CF51040B08E06F
:1073200011D0D40507E187ECD4F002E2420E21D05F
:10733000450E1FD0020ED45D07E187ECD4F002E2C7
:10734000400E17D0440E15D0050ED45D07E1E5516F
:10735000800B02E0480E0DD0470E0BD0040ED45D1A
:1073600002E1460E06D0D051400B02E1430E01D09F
:10737000410E52ECCAF0B2ECCDF0030E005C12E10B
:107380000A0403E0020E0A5C05E10101D051040B7E
:1073900005E106D00101CF51040B02E0540E1CD0D0
:1073A000550E1AD0000402E1520E16D0020E005CF7
:1073B00002E1500E11D0050E005C02E1570E0CD018
:1073C000040E005C02E1560E07D00101D051400BC3
:1073D00002E1530E01D0510E52ECCAF0E3EFC9F0B6
:1073E000A9ECD6F0BDECCAF00CE12A50020B01E08A
:1073F000010EE66ED950010F4FECCCF02A92AEECA4
:1074000016F033B842D02050800B12E11450100B0C
:107410000FE01450200B0CE10101D45106E0030EE3
:10742000D45D03E0050ED45D03E11498DFEC4FF06A
:107430002050800B0AE11450200B07E0BDECCAF08D
:1074400004E1149A1498DFEC4FF03AECCCF003E02E
:10745000050ED45D01E1D29D1390D45103E1139048
:107460008AB51380030ED45D05E10A5003E0139042
:107470008EB51380139A13A0138A67EC0CF092EC6C
:1074800064F025EC19F080EC25F025824AEC32F00E
:10749000010EE66E34DFE552FEEC16F029EC1EF02C
:1074A00033B85FD0D5CAE6FFAB0E42ECCAF037EC7A
:1074B00019F0DFEC4FF09AEC0FF0B9EC1FF0DAECBA
:1074C0001EF028B24ED01C9834902450010B05E1D8
:1074D0002750200B02E0DDEC08F00E6A0F6A51EC39
:1074E000D2F004E1100E0E6E270E0CD0050ED45D06
:1074F00004E1240E0E6E2C0E05D0D2A104D0400E55
:107500000E6E1F0E0F6E06ECCCF0A40E0DECCAF042
:10751000BDECCAF003E0050ED55D02E14BEC0CF0CA
:10752000CFEC1EF06F0E52ECCAF043EC53F046EC79
:107530001FF0B7EC1DF044EC19F09BEC15F0A4EC37
:10754000CAF002E03AEC1EF0C3EC15F0050E005C48
:1075500002E113EC09F0C3EC23F0F5EC64F0F6EC77
:10756000C4F0BDECCAF00AE1010EDB502A92E8B08B
:107570002A822AB203D02A82B5EC16F03398030E81
:10758000E15C02E2E16AE552E16EE3EFC9F08C985A
:1075900000000000030EE66EA2EC5CF0E552040E63
:1075A000095CE66EA2EC5CF0E5520150E66EA2ECDE
:1075B0005CF0E552D3ECFDF0006E00008C88120008
:1075C000D9CFE6FFE1CFD9FF8C9800000000060E6E
:1075D000E66EA2EC5CF0E5528C8800000000000032
:1075E0008C9800000000020EE66EA2EC5CF0E55202
:1075F000040E095CE66EA2EC5CF0E5520150E66E0A
:10760000A2EC5CF0E552FE0EDBCFE6FFA2EC5CF0F4
:10761000E5528C88040EE66EA5ECFDF0E552E552CD
:10762000E7CFD9FF120063ECD5F00050DF6E010EFA
:10763000DB6A3CD8DF50005C31E0680E095C02E197
:10764000012A0106040E095C16E2F29EA698095072
:10765000636E0150626EDF50616E7F9E7F9C7F84FF
:10766000550E7E6EAA0E7E6E7F82F28E040E23EC85
:10767000D7F07F9413D0010EDB2ADFCFE6FFA0DF27
:10768000E55285DFDF50005C02E03DEC0DF0DF509D
:10769000005C04E0050E65ECCCF0EDE3020EE15C6D
:1076A00002E2E16AE552E16EE3EFC9F063ECD5F086
:1076B000010EDB6A040E095C0AE20950636E015098
:1076C000626E7F9E7F9C7F806150006E12D0010EA3
:1076D000DB2A5DDF0050DF6E5ADF0050DF5C02E026
:1076E0003DEC0DF00050DF5C04E0050E65ECCCF0E5
:1076F000EEE3020EE15C02E2E16AE552E16EE3EFE5
:10770000C9F0E7ECC9F02DECD0F012E0FC0EDBCFB5
:10771000F3FFDB2AF350ECECCBF0FD0E2CECDAF0AF
:10772000FE0EDBCFEAFF01E3DB2A00C0EFFFEBD761
:10773000E3EFC9F0E7ECC9F02DECD0F01AE0F7EC7C
:10774000D1F017E3EFECD8F005E24950A408000EA1
:107750004A540FE37EECD1F0016EFC0E2CECDAF013
:10776000FD0EDBCFEAFF01E3DB2AEF50CDECD0F0DA
:10777000E3D7E3EFC9F0E7ECC9F01F0E0501235D85
:107780000DE2232B2551EA6A270FE96E050E29EC3D
:10779000D8F0252B25511F0801E2256BE3EFC9F036
:1077A000E7ECC9F0030E0A5C54E10E6A0F6AFE0EA4
:1077B000DB500D0803E11F0E0E6E0F6AFE0EDB504C
:1077C0000A0803E11D0E0E6E0F6AFE0EDB5009085B
:1077D00003E1EF0E0E6E0F6A23ECD5F003E10E68A5
:1077E000020E0F6EFE0EDB507F0804E1B50E0E6E2A
:1077F000030E0F6EFE0EDB501F0821E27F0E6DECB4
:10780000CAF01DE2410E6DECCAF00CE3FE0EDB5037
:107810005A0808E3200E496EFE0E4AECD8F0FE0E20
:10782000E7CFDBFF4A0E496ECD0E4A6E010E4B6E5E
:10783000FE0EDB50E00F87ECDAF03DECD9F00E5095
:107840000F1049E00FC0E6FF96DFE5520EC0E6FFDD
:107850003DD0FE0EDB50090803E1200E1BECCFF0FB
:10786000016A400E015C37E2290E4A6EDB0E4B6E58
:10787000010E4C6E0150EFECCAF0FE0EDB50495C7D
:1078800028E1030E066E01B0068C01B2068A01B42F
:10789000068801B6068601B806842350040B09E168
:1078A000200E011406E06F0EE66E65DFE5522384BC
:1078B0000BD02350040B08E0200E011405E17F0ECD
:1078C000E66E59DFE55223940650E66E54DFE5522A
:1078D00002D0012AC6D7E3EFC9F05FECD5F0800EE5
:1078E0006DECCAF003E3200E1BECCFF00201050E95
:1078F0002D6FFE0EDB50740810E1010E2D6F030E8C
:107900000A5C07E105012351F2ECD8F0020F0201F5
:107910002D6F0501106B1D822BD0FE0EDB5028E071
:10792000DF6A150EDF5C11E244ECD9F00BE1DF2ACF
:107930006BECCDF096ECD4F0DF2A6BECCDF096EC4E
:10794000D4F003D0030EDF26ECD7150EDF5C04E184
:1079500095ECD5F025DFE552200E6DECCAF003E280
:10796000200E1BECCFF095ECD5F002EC70F0E55258
:10797000E552E3EFC9F063ECD5F023A01CD01DB0B5
:1079800013D02750200B06E00AECCBF003E00201F5
:10799000050E2D6F020E0201535D1FE30701016BFF
:1079A000026B53C254F219D00201532B5351800879
:1079B0001EE2800E1BD01DA013D0070E0701015D33
:1079C0000AE2012B02910243020E0201535D05E31C
:1079D0000701028F02D0070E016F0201010E06D0CF
:1079E0000201532B5351800802E2800E536F1D9009
:1079F00023B01D802350010B03E1020E535D04E010
:107A00001D50020B01E18AD01DA204D00701CC0E4B
:107A1000026F0FD0070102910243028F070ED88038
:107A20000155016E01500106000903E00291024375
:107A3000F9D700C709F00101B5A7E88B020154513D
:107A400007081DE254513F0802E23F0E546F10EC4C
:107A5000D2F006E0200E32ECCDF0200E96ECD4F001
:107A6000D0ECD0F00CE00701035109E0800E0201D8
:107A70005425006E03C701F007010307D4DD780E1B
:107A80000701025D18E2298A02C7E6FF3CEC04F018
:107A9000E552DF6EDF500EE010ECD2F00BE02D511E
:107AA00004E0DFCFE6FF19DF04D0DFCFE6FF02EC12
:107AB00070F0E552299A0101E89BB5A72FD0070184
:107AC000035105E002C700F003C701F0ACDD070178
:107AD000035106E01D50020B03E11C0E025D1BE189
:107AE00003510AE01C0E025D07E1CC0E006E030795
:107AF00003C701F098DD1D820101B5978CEC65F09C
:107B0000230E155C03E1410E9FECCAF0249223ACD6
:107B100003D0248201D003070701026B096A020E19
:107B2000E15C02E2E16AE552E16EE3EFC9F081EC6B
:107B3000CCF00CE11C0E0101B95D08E11850400BBE
:107B400005E084848C808D8A8D8C12000601505152
:107B5000040B02E08D8C01D08D9C5051080B02E08B
:107B60008D8A01D08D9A5051010B02E08C8001D09A
:107B70008C905051020B02E0848412008494120015
:107B8000000012000601D99D8850800B01E0D98DBC
:107B9000D99F8850400B01E0D98FD9918850100BA4
:107BA00001E0D981D9938850200B01E0D983D9997C
:107BB0008850080B01E0D989D99B8850040B01E05B
:107BC000D98B1200E7ECC9F0FD0EDB506DECCAF06A
:107BD00008E3FE0EDBCFE6FFFD0E8CECD2F00AE2EE
:107BE00007D0FD0EDBCFE6FFFE0E8CECD2F002E2FA
:107BF000010E01D0000EE3EFC9F0A9ECD6F02EB2D1
:107C000054D082B003D00701290E76D082B203D0BF
:107C100007012C0E71D0DF6A060EDF5C43E2DF50F5
:107C2000040DF350830985ECD0F0050EDF5C03E111
:107C3000DE52BB0EDD6ED9ECD9F000C047F7005024
:107C40001A082EE2F00E005C2BE2FE0EDB5002E181
:107C5000010E56D0D9ECD9F000C048F700501A08F0
:107C60001FE2F00E005C1CE2D9ECD9F000C049F72D
:107C700000501A0815E2F00E005C12E2080EE66EE3
:107C800048C7E6FF47C7E6FF0EECCEF009E0080E56
:107C9000E66E49C7E6FF48C7E6FF0EECCEF002E10C
:107CA000DF2ABAD7060EDF5C02E1000E29D0010EF2
:107CB0007EECD4F094ECD2F010E20C0EE66E020EE4
:107CC000DB50370F78ECCCF0E66E48C7E6FF0EECE1
:107CD000CEF003E1020EDB2AEDD794ECD2F00FE2F6
:107CE00047C74AF748C74BF749C74CF7020EDB5066
:107CF000080DF350DF1007014D6F4D5101D0800E7C
:107D0000496E030EE15C02E2E16AE552E16E495020
:107D1000E3EFC9F037ECCFF0DCECD2F006E1BDECDC
:107D2000D0F003E001011E0EAC6F01012D0E176FA4
:107D30001FA402D02B0E176F0201405107E13F51E3
:107D400005E13E5103E10101200E176F8CECCAF0F2
:107D500040C23EF0B3ECCCF00101186F300E3A2473
:107D6000196F300E02013F2501011A6F0701BEABEA
:107D700005D0300E02013E2501011B6F0101198F54
:107D80001200A5ECD6F04DECCBF0EFCFDFFF0101F8
:107D9000A36BA46BA56BA66BA76B1DAE03D0050EE2
:107DA000A56F32D05AECCEF0EF50400B03E12750D4
:107DB000040B1DE095ECD5F056EC0DF0E55200C03B
:107DC000A5F1005063081BE20101A56BA42B7D0EF9
:107DD000005C02E1190EA56F76ECDAF0FA0E491894
:107DE0000EE14A500CE1A42B320EA56F08D05AECDC
:107DF000CEF0EF50200B02E0A72B01D0A62B2AAE2D
:107E000003D0020E16ECCAF0E552E3EFC9F0AC0E57
:107E1000006E0050B6ECCEF035C100F02BECD5F082
:107E200001011A5D05E14FECD8F002E1200E1B6F55
:107E30000201060E3D6F80EF25F0E7ECC9F0D40E8D
:107E4000496EDD0E4A6E010E4B6E050E4F6E4FC031
:107E500043F0FE0EDBCF3EF05AECFEF03EC04CF09D
:107E600057ECDBF0006E8EECDBF00101020E2EEC25
:107E7000D4F0128F0C0E6DECCAF003E20E0E0F6FF1
:107E80000ED00E0E106FFE0EDB50630802E2100ED5
:107E9000106F0F0E6DECCAF002E2090E116F140E96
:107EA000146F120E156FE3EFC9F0E7ECC9F09EEC0A
:107EB000DBF00101012BFE0EDB50006E9DECE1F0CA
:107EC0002B50100B07E1640E6DECCAF003E20101C8
:107ED000200E176F2BA807D001014D0E1B6F570EF8
:107EE0001C6F188F16D0FD0EDB5003E10101198FB6
:107EF00007D00A0E6DECCAF003E20101200E186FE4
:107F00000101570E1B6F33B602D02A0E1C6F5FB3F0
:107F10001C8FE3EFC9F0E7ECC9F080EC25F0FE0E12
:107F2000DB5003E004ECD5F003D00068E9EC26F068
:107F300085ECCBF01AE0020E0101395D0FE1A50ED0
:107F4000485D0CE19EECDBF0470EE66EE40EE66E5B
:107F5000010EE66E44ECE2F0E5520BD0010EE66E47
:107F60006FEC05F0A60FE66E03D0E66A48C1E6FFA7
:107F70009CDFE552E5522BA807D00068DDEC26F027
:107F800048C1E6FF5ADFE552E3EFC9F05FECD5F0F8
:107F900080EC25F0B40E61ECD2F034C1DFFFF0ECE0
:107FA000D2F003E0E4ECD2F001E1DF6ADF50006ED2
:107FB0009DECE1F0640EDF5C03E20101200E1A6F1C
:107FC0000A0EDF5C03E20101200E1B6FE552E3EFB6
:107FD000C9F037ECCFF0DCECD2F008E1BDECD0F02A
:107FE00005E00101D45102E0AC91AC4349C100F07D
:107FF0009DECE1F0640E0101495D02E2200E166F76
:108000000A0E495D02E2200E176F8F0E006E25EFFB
:1080100026F0270E9FECCAF00101500EAC6F3B51C9
:10802000200B06E1BDECD0F003E001011E0EAC6FA9
:108030001200EB0E006EA4ECCAF002E0EE0E006E31
:10804000D2EC26F032C100F0A4ECCAF002E053C139
:1080500000F00101040E016F9DECE1F001011B8FA6
:108060001200E7ECC9F0A4ECCAF003E00AECCBF094
:1080700003E028C100F008D01BECD5F003E058C1A4
:1080800000F002D054C100F0E3EFC9F0CD0E61EC76
:10809000D2F0010EE66EE5DFE5522BECD5F00101E2
:1080A0001A5D05E14FECD8F002E1200E1B6F1200C3
:1080B000E7ECC9F0DEECCBF0EF50400B03E12750CA
:1080C000040B04E001018E51020B6BE0DEECCBF0FF
:1080D000EF50200B03E02750040B02E00101A26BDC
:1080E000DEECCBF0EF50400B03E12750040B59E0DE
:1080F0000101A4510EE0A5510CE1FE0EDB5005E19B
:10810000A05102E1A15101E0A46BA06BA0C1A1F1BB
:1081100048D05A0EA55D16E18CECCAF0A0C13EF025
:108120000BECD5F0006EFE0EDB5007E1005003E1D2
:108130000101A15102E00101A56B0101A16B0050F9
:10814000A05F2FD0A05102E1A1512BE0A151496EB7
:108150004A6AA0510A0D17ECCDF0A5510A0D56EC54
:10816000D4F0E2ECCBF0D8C142F0D9C143F000EC3E
:10817000FEF039C0D6F13AC0D7F10101D651D7117E
:1081800010E0D6510E5ED7510F5AFE0EDB5001E1C2
:10819000A56B45ECD2F053ECD6F03DC0A0F139C050
:1081A000A1F1E3EFC9F0E7ECC9F095ECD5F0E66A90
:1081B0007FDFE552E55201ECD0F0ECEC31F001014B
:1081C0009E510DE11F0E9F5D0AE29AC29EF19BC275
:1081D0009FF19CC2A0F19DC2A1F19EC2A2F1020139
:1081E0006F2BE3EFC9F00101DE93D1B3DE83DE959F
:1081F000D1B5DE851200010138A306D0D19312B6A5
:10820000D183D19512B4D185EEDF04B083DDA4EC27
:108210009AF0ABEF2EF00A0E02013F03F3504B6EC3
:108220004C6A4051640D79ECD3F03E510101492470
:10823000DA6F000E4A20DB6F0A0E006E0701BEAB3C
:1082400002D0010E006E1FB403D0010127ECD2F062
:1082500028AA1AD076ECDAF0100ED8804956270EEC
:108260004A560101DB514A18E8AE02D04A3404D024
:108270004950DA5D4A50DB591FE2005006ECD7F056
:10828000DA274A50DB2318D000504A6AF00F496EB3
:10829000D80E4A2201014A50DB19E8AE02D0DB3584
:1082A00004D0DA51495CDB514A5806E2005006EC32
:1082B000D7F0DA5F4A50DB5B1F84800EDB1503E0EA
:1082C0001F9427ECD2F076ECDAF0DAC13DF0DBC196
:1082D0003EF062ECD3F04AAE04D0396C3A1E000E88
:1082E0003A2239500101DA5F3A50DB5B00ECD5F0FD
:1082F0004BECD9F03DC040F239500101DA6FDB6B35
:1083000045ECD2F04BECD9F03DC03FF239C03EF223
:108310008AEF41F02F8E0480FBEF40F00A01DA9FD4
:1083200067EC0CF0016A0101D4510EE10701BEBFF8
:1083300011D00A0E016ED8ECCDF03E50006E015007
:10834000005C18E2005015D0030ED45D11E1070166
:10835000BEAF02D0160E0DD0030E0A5C02E1140E61
:1083600008D00A5002E11E0E04D0E8ECD7F001D08C
:10837000160E016E0150160802E2160E016E120072
:10838000000CFEDF000903E00101500E486F1200EF
:10839000E7ECC9F000AE14D0FF0E0002F3CF6FF28D
:1083A0006F0EE96E020EEA6EEFCF3EF0FE0EDBCFEF
:1083B00043F05AECFEF03EC0EFFF02016F6D09D0B2
:1083C00000C03EF0FE0EDBCF43F05AECFEF03EC0A4
:1083D0006FF2E3EFC9F05FECD5F02F50200B56E1C0
:1083E0002350800B53E13050400B50E12450010BDF
:1083F0004DE11FA618D099ECD2F001012699020197
:108400006F5102E0010126890101269B02016FAF35
:1084100002D00101268B010126A938D01DAC36D02F
:108420001EEC0CF033D024C100F00101269900505D
:1084300001E02689269B00BE268B26BB006C81ECC2
:10844000CCF016E12E50100B0DE01E50040B0AE18B
:108450001B50080B07E1005002E0F5EC08F0006A41
:108460000101246BF8ECD2F006E0450EB95D03E0A3
:1084700000380F0B006E005007E00101268D269F8B
:1084800026BB268F246B02D001012699010126A963
:1084900002D08CEC04F001012651100B06E02B50A9
:1084A000200B40E01D50400B3DE11F50080B16E033
:1084B0003B51200B13E13BB332D0A1ECD2F00101D0
:1084C000279902016F5102E0010127890101279BD1
:1084D00002016FAF27D00101278B24D025C100F006
:1084E0002799005001E02789279B00BE278B2799F9
:1084F00027BB006C32A005D00038E8461F0B006E89
:1085000004D0D8900032D890003200500AE0070121
:10851000460EA66F0101278D279F27BB278F256B4E
:1085200001D027992B50200B03E01D50400B10E089
:1085300001012651100B02E0E2EF46F02751100B2B
:1085400002E0E2EF46F02050200B02E1E2EF46F0BD
:10855000D7CADCFAD6CADDFA0601D551D595010B8A
:1085600001E0D585D551D597020B01E0D587D5918E
:108570008650040B01E0D581D5938650020B01E0B3
:10858000D5830F0ED51521ECCCF000A019D08CECC2
:1085900004F006015051040B0CE03250010B09E1CC
:1085A0003050040B06E100AE02D0DA0709D0DA2B16
:1085B00007D000AE03D00101250702D00101252B11
:1085C000DAC600F00601D599005001E0D589D59BA7
:1085D00000BED58BD5A92ED0D5BB006C0090004233
:1085E000005028E0DA6B50A525D001013751010B6E
:1085F00006E01250080B03E11250040B0FE0288A2A
:108600000601D5BB289A07DE1EAC03D002010987FC
:1086100002D0020106810501478D0CD0AAC224F1C7
:108620000601D5AB04D0AAC224F10101246D0101D9
:10863000268927840601D651D695010B01E0D685FF
:10864000D651D697020B01E0D687D951D691020BAD
:1086500001E0D681D951D693010B01E0D6830F0EEC
:10866000D61521ECCCF000A009D0A1ECD1F000AEE1
:1086700003D00601DB0702D00601DB2BDBC600F0CE
:10868000D699005001E0D689D69B00BED68BD6A9DC
:10869000CBD0D6BB006C30BC02D000900042005062
:1086A00001E1C2D0DB6B010E0D6ED6BB0D68A1ECF3
:1086B000CBF001E1B0D027ECD5F0BDECCAF003E17E
:1086C000D9EC0BF0A8D031BCA6D030AC0ED0D00E77
:1086D000E66E0F0EE66E840EE66E070E25ECCAF00F
:1086E000F5EC04F014EC50F096D0D4510BE0030EEE
:1086F000D45D08E08D51100B3EE0020ED45D02E027
:10870000D40539E114BC1CD03484ECEC0FF05CECE3
:10871000D6F007E249501408000E4A5402E2ECEC8D
:108720000FF05CECD6F009E249503D08000E4A54C7
:1087300004E2ECEC0FF0ECEC0FF0F5EC0FF06BD08A
:1087400034844DECD2F008E0C80EE66E280EE66EDA
:10875000B80EE66E030E0AD0E1DD190E0124E66EB6
:10876000F4ECD2F0E66ED70EE66E0A0E25ECCAF0F7
:108770000A01030E49D014BC25D03484CFDD0D048A
:108780000BE193ECD3F008E2190E0124D75D04E26B
:10879000020ED65FD72B11D0800E0D140EE0DCEC4C
:1087A0000FF0FF0F0A01D65D08E2F4ECD2F0D8809A
:1087B000D75503E2020ED627D7070A01010ED46F60
:1087C000338825D03484AADD800E0D140CE093ECA0
:1087D000D3F009E2F4ECD2F0D880D75504E2020ECF
:1087E000D65FD7070FD00D040DE1DCEC0FF0FF0FC3
:1087F0000A01D65D07E2190E0124D75D03E2020EDD
:10880000D627D72B0A01020ED46F3388010EE66EED
:108810008CEC1BF0E5521EAC03D00201098902D09A
:108820000201068B050147850601D751D795010B3B
:1088300001E0D785D751D797020B01E0D787D951EF
:10884000D791200B01E0D781D951D793100B01E0CC
:10885000D7830F0ED71521ECCCF000A009D0A1ECE6
:10886000D1F000AE03D00601DD0702D00601DD2BFA
:10887000DDC600F0D799005001E0D789D79B00BE34
:10888000D78BD7A9C8D1D7BB006C0090004200504D
:1088900001E1C1D1DD6B010E0D6ED7BB0D68195022
:1088A000100B04E12050800B01E1E4D001018DB5F3
:1088B00095D133B635D020BE04D0740E006EDDECF9
:1088C00026F0FF0E0D5C0CE10201050ED88000556C
:1088D000000E015522E2060E005F000E015B1DD066
:1088E00071C201F02B50100B0BE10201715158ECD9
:1088F000CBF006E220ECD4F003E25A0E015C016EEC
:1089000001500B5C0AE20201880E005D130E015952
:1089100004E2060E0027000E0123E7EC0BF077D1EE
:1089200002011D6B960E016E026A2FECD5F002E07B
:10893000C80E016E2BA804D0960E016E0A0E026EB0
:108940000150E66E0250E66E480EE66E010E25EC12
:10895000CAF085ECCBF00CE1010148510A0808E2AD
:10896000010E481505E00D0402E1482B01D048072F
:108970002A840901ED6BEE6BE9EC04F0C3EC23F003
:108980009BECD4F0E5520201320E046F48C15BF259
:1089900064ECD2F002E248C18CF1E783E795E797F7
:1089A00048C102F085ECCBF004E00101E7935A0ED8
:1089B000025E0250E66E14ECD3F02FECD5F015E019
:1089C0002B50100B12E10D0404E1650E0101485D0E
:1089D00007E0800E0D1409E0640E0101485D05E119
:1089E000318EA1ECCBF001E01C94B2ECCDF0315013
:1089F000800B11E12050800B0EE1A1ECCBF00BE1DC
:108A000000500BE0050E005C08E0030E005C03E183
:108A1000020E0A5C02E00D5001D0020E2CECD2F0E6
:108A200031AE25D0319E049819A006D0048843ECBD
:108A30000BF0050E16ECCAF00101395111E085EC7E
:108A4000CBF006E0410EE66EE40EE66E010E02D0BB
:108A5000A7ECD1F077ECD7F003E1FA0E16ECCAF0F0
:108A600004A802D03EEC0BF00D502CECD2F0020129
:108A7000078BCDD00101E6AF28D08DB5AFD034C182
:108A8000A8F23AEC19F01E0EE66E340EE66E010EF8
:108A900020ECCAF0C6EC3FF09FECD4F034C1E6FF06
:108AA00014ECD3F0B7EC1DF00201A85103E0010172
:108AB000345106E00201A85105E10101345102E000
:108AC000F5EC17F002010885A1D02CA426D0E7858B
:108AD000E793E797A4ECCAF00EE1C80EE66E320EFB
:108AE000E66E010E20ECCAF032C1E6FF14ECD3F0C2
:108AF00092EC64F00FD0C80EE66E010EE66E530ED7
:108B0000E66E010E25ECCAF053C1E6FF14ECD3F07B
:108B100025EC19F019EC40F07AD024A035D0D451CE
:108B200011E1460EE66E280EE66E290EE66E010E87
:108B300025ECCAF001012951E8240301B86F18ECB3
:108B4000CFF016D0AEECCDF007E0E66A2E0EE66E62
:108B5000010E20ECCAF00ED0BDECCAF00BE1330ED2
:108B6000E66E010EE66E870EE66E020E25ECCAF08A
:108B7000F5EC04F049EC4FF073ECCCF0F5EC17F0A9
:108B800005014785478F43D0A4ECCAF006E00AEC04
:108B9000CBF003E12750020B1CE0320E006E0050B8
:108BA000E66E080EE66E490EE66E010E25ECCAF082
:108BB000E9EC3FF00101E793E795E78749C1E6FF5C
:108BC00014ECD3F049C113F52FEC65F002010687D0
:108BD0001ED0B2ECCDF001018DA503D0EEEC08F073
:108BE00016D03AEC19F0500EE66E350EE66E010E18
:108BF00020ECCAF09BEC15F007EC3FF09FECD4F0B2
:108C000035C1E6FF14ECD3F0020108832A842D8ECF
:108C100002011E0E206F0601D851D895010B01E00C
:108C2000D885D851D897020B01E0D887D951D8916F
:108C3000800B01E0D881D951D893400B01E0D88353
:108C40000F0ED81521ECCCF000A009D0A1ECD1F08A
:108C500000AE03D00601DC0702D00601DC2BDCC627
:108C600000F0D899005001E0D889D89B00BED88B7D
:108C7000D8A9A8D0D8BB006C00900042005001E1F8
:108C8000A1D0DC6B010E0D6ED8BB0D682CA631D0C7
:108C9000A4ECCAF003E00AECCBF00AE0280EE66E82
:108CA000280EE66E010E20ECCAF0A7ECCCF01ED028
:108CB000F0ECD2F00BE11E0EE66E580EE66E010EE1
:108CC000E66E59EC7AF0E552E5520DD01E0EE66ED6
:108CD000540EE66E010E20ECCAF09FECD4F054C1A5
:108CE000E6FF45EC0AF0E55244EC19F046EC40F0A2
:108CF00065D023AE23D021B661D0016A0101D451E1
:108D000002E0010E016E71ECD6F00AE1FFECD6F044
:108D100004E6E20E495C000E4A5802E2190E0026F3
:108D2000FF0E0D5C05E10050180802E2190E005E0E
:108D3000015087ECCAF000C0EFFF0BD02FAA0DD076
:108D400021B63CD00E0EE66E930EE66E020E20ECBF
:108D5000CAF0F5EC04F0238A31D021B00ED021B650
:108D60002DD03C0EE66E660EE66E010E20ECCAF0CB
:108D700022EC53F01BEC05F021D021B61FD0BDEC46
:108D8000CAF00CE1280EE66E680EE66E010E20ECCD
:108D9000CAF04BEC0CF059EC05F010D0800E0D141D
:108DA00004E03C0E675D01E2672B0D0403E16751AF
:108DB00001E0670743EC53F035EC05F02D8E02011E
:108DC0001E0E206F1DAC66D00701BE837EEC09F03D
:108DD00001013B91129C3B51010B01E0128CE66AB0
:108DE00004EC2CF0E552006E00500F0802E20F0E6A
:108DF000006E100E0002F3CF0EF26FEC27F01D9AFA
:108E0000050E0701A1250201D8800E5501E21D8A39
:108E10002A50800B13E10D5111E0050E0701A15DF1
:108E200002010E5D03E2DDEC08F01D881D50100B01
:108E300031E01D50200B2EE0020109D02A50800B9A
:108E40000AE11D50800B07E11D50200B04E0FA0ED3
:108E50000D6F1D981FD02ABE02D0DAEC08F02BBA95
:108E600017D01E0EE66E050E9DECD0F0E66E5DECA2
:108E7000CDF00AE019C5C4F11AC5C5F11BC5C6F18C
:108E80001CC5C7F11DC5C8F1AAC224F10101269B6A
:108E9000010126891D50800B0DE101012651100BA7
:108EA00001E17ED01F50080B01E17AD02050200B49
:108EB00001E176D002011E0E206F1DAC02D0140E0F
:108EC000206F2BAA2FD01DBC16D00101445163087E
:108ED00001E2446B800E241506E0FB0E245D03E2E4
:108EE000246B000E12D0800E241559E12451030882
:108EF00056E2246B09D00101246B2AAE09D005018A
:108F000016514DE1320E166F010E9AECD3F047D098
:108F1000AD51030844E3010E9AECD3F00101140EA5
:108F2000AD6F3DD01E50400B03E00951010B37E1FE
:108F30001EAC02D0098101D00683050147812B8C2C
:108F40002C8A15ECCBF0D4C1E6FFC1EC3EF0E55223
:108F500099ECD2F01D50800B06E00101245103E191
:108F6000C8EC31F016D002016FAF0AD0BEC7E6FFE1
:108F7000D3EC40F0E5520201AA510101242709D0A7
:108F80006F5107E0BEC7E6FF0CECD0F0AA5101011B
:108F9000245F02016F51DCE12D827CEC04F01D9E08
:108FA00001012751100B4BE01F50080B48E02050E7
:108FB000200B45E002011E0E206F1DAC02D0140EE6
:108FC000206F1EAC02D0098301D0068305014783C0
:108FD0002B8CD5C1DFFF2C9AE0ECCCF0DFCFE6FF85
:108FE000C1EC3EF0E552A1ECD2F002016FAF0DD022
:108FF000DF504DECCBF0EF50E66ED3EC40F0E55295
:109000000201AB51010125270CD06F510AE0DF505E
:109010004DECCBF0EF50E66E0CECD0F0AB51010113
:10902000255F02016F51DFE12D82F6ECCCF024A622
:1090300006D00101010EAC6F0701140E556F2BAC69
:1090400006D083ECD4F02B9C25822CAA238A010124
:10905000279926992794E552E3EFC9F03B0E00ECDF
:10906000CBF00101320EAC6F2F8833C119F2120020
:10907000010137A70AD04D0E096E0F0EE66E100ED5
:109080000D03F35031ECD2F010D0030E096E0F0E29
:10909000E66E140E31ECD2F055ECCAF0030EE66E1B
:1090A000230EE66E230EE66E0A0E55ECCAF0096A30
:1090B0001200E7ECC9F0030E096E140EE66E000E06
:1090C000E66E0A0EB5ECD9F0040EE66E260EE66EDC
:1090D0000A0EE66E260E81ECD6F0FE0EDB501EE088
:1090E000010137A70AD04D0E096E0F0E31ECD2F0F8
:1090F000E66E100E0D03F3500ED00F0E31ECD2F0D1
:10910000E66E140E81ECD6F0030EE66E230EE66ECC
:109110000A0EE66E230EE66E4DECCAF0096AE3EF26
:10912000C9F0030E096EAA0EE66E2A0EE66E0A0E4E
:10913000E66E300E5CEFDBF07AEFDAF000ECD6F0A2
:1091400003E10201D8511CE0010191ECD4F001E0EF
:10915000098FE1ECDAF00601EE6B69EC32F0070101
:109160000B99BCECC4F0B5EC20F00701149F77EC30
:10917000D5F0070115817EECD5F0B5EC16F02D8603
:109180000201D96BD9C2D8F21200010121A17BEFF3
:109190004DF0219102010F070F5101E01AD1640E29
:1091A0000F6FBDECCAF016E12050400B13E1080E22
:1091B00097ECCBF0046E04AC0DD00101E5BF02D0FA
:1091C000E58F02D0E5BFE59FE66A7FEC39F0E55216
:1091D0004AEC32F002013D510CE03D51010803E33D
:1091E000A1ECCBF006E002013D073D5102E180EC2D
:1091F00025F03196150E0101555D0BE00201165167
:10920000171103E01607000E175B1651171101E145
:109210002F8C0201145101E0140701018B5104E06D
:109220008B078B5101E13196020120510CE01F5058
:10923000080B09E02007205106E11DAC02D01D8E6D
:1092400002D02DBE2D9E300E0401F75D06E1020115
:10925000066B076B086B096B05D0340EF75D02E2F5
:10926000A4ECA1F0020119511BE00501105118E115
:109270002750400B15E159ECD2F012E119071951B2
:109280000FE10C50006E555106E07F0E5515006E33
:10929000189A55BF188A010EE66E00507CECD2F089
:1092A0000201580758510BE10101515102010B5DB8
:1092B00006E2410E00ECCBF00101AC69258EA1EC79
:1092C000CBF008E00101835105E0765103E169EC40
:1092D000E3F002D035ECE4F049ECD2F008E081ECA8
:1092E000CCF005E133ECD5F002E106011D7908EC84
:1092F000D3F011E01B50100B0EE12150020B09E0DE
:10930000050ED45D06E0040ED45D03E01E50200B74
:1093100002E10601047901013851100B06E11350F6
:10932000020B05E01950200B02E106010D752850D3
:10933000400B01E0010E020F016E2850400B01E0CE
:10934000010E050F026E03681DAC08D079ECD8F051
:10935000EF7E79ECD8F0EF50800B036E0101835162
:109360002BE0DAECE3F0000903E12E50200B24E0BF
:109370002E9AAEEC16F0016A030E015C12E2026A4C
:10938000040E025C08E2020EC1ECD6F0320E16ECBE
:10939000CAF0022AF5D7E668BFEC21F0E552012AAF
:1093A000EBD7B5EC16F001015F9925821EEC79F040
:1093B000C4ECE3F069ECE3F002012D5101E02D076C
:1093C0007A5104E02250100B01E17A07325101E09A
:1093D0003207D35109E0D307D35106E1D45102E15A
:1093E000010ED46F62ECC2F01EAC09D00201D107AD
:1093F000D15105E1A4ECA1F00201030ED16F59ECAB
:10940000D2F040E02050400B3DE01950400B3AE0D4
:10941000D0ECD0F003E11950200B34E00201370703
:10942000000E385B1950200B0AE00FECD1F009E177
:109430003FECCDF004E10101E451100B02E1000E1C
:1094400001D0010E0490E8B0048059ECD2F003E0A2
:109450000450010B17E0376B386B0101E49904A04D
:1094600006D00201196B19C255F28CEC65F00DECB7
:109470000BF00101B5A705D0249223BC2482FBEC9C
:10948000D0F0209402013C5101E03C07335101E04F
:109490003307315101E0310730510AE030073051D4
:1094A00007E144ECCEF001E14A5002E04FEC0DF050
:1094B0000201185109E01807185106E12AECCFF013
:1094C0000201D05101E11194100710513FE1280E23
:1094D000106F1AAC0FD0D4EC38F0D4C100F008EC07
:1094E00039F00601017901A931D0D5C100F008ECAD
:1094F00039F02CD01BA803D00601047927D01CA278
:1095000006D00101E6B522D0060114711FD0195012
:10951000200B06E001013851100B02E106010D7528
:109520002450020B03E1E0ECD2F010E002013051D4
:109530000DE144ECCEF001E14A5008E02C50800BE4
:1095400005E12C50400B02E10601017102012B5193
:1095500001E02B070701A65105E0A607A65102E18D
:10956000FCECD1F002012A5116E02A072A5113E13E
:10957000A4ECCAF003E194ECE2F00DD00701A35192
:10958000A41109E0A35101E0A307A45101E0A4073D
:109590000201020E2A6F020129510CE0290729510C
:1095A00009E1178E17901788080E156E2CAC02D0A3
:1095B000290E156E0101AE5169E0AE07AE5166E1AC
:1095C00043ECD1F0006E0201A95107E0830E096E51
:1095D000A9C201F056EC3BF0096AFF0E0201845D5E
:1095E00028E084C24FF0506A516A050E496ED90EC8
:1095F0004A6E010E4B6EB9C14CF04D6A4E6A4BEC8F
:10960000D5F00900F5504F24F36E0900F5505020B5
:10961000F46E0900F55051204DECD6F00800F550DD
:10962000006E0201842B005004E18469010151ECB9
:10963000D9F0005013E00101190EAE6F0050E66E34
:109640000DEC70F0E5520201A95102E0A92B1ED0E9
:109650000101B22B000EB323B42318D02850080BFD
:1096600003E13050080B04E028960101E8970ED082
:109670000201A95105E0A96B0101FA0EAC6F05D0FA
:109680000101D890AC33D890AC33E897020128514F
:1096900004E02807285101E1259E275107E027070C
:1096A000275104E10601416941C640F60101AA5172
:1096B0000DE0AA07AA510AE1090E155C07E181EC49
:1096C000CCF004E10101FA0EAB6F1A8A0101AB5133
:1096D00001E0AB070701555101E0550702012F5189
:1096E00023E02F072F5120E1000E0601E76EBE197F
:1096F000E8AE02D0BE3503D0E750D880BE5502E2B6
:10970000BE0701D0BE2B000EE76EBF19E8AE02D037
:10971000BF3503D0E750D880BF5502E2BF0701D064
:10972000BF2B0201050E2F6F155105E015071551CE
:1097300002E11CEC6AF00201215124E0210727AA72
:1097400021D020BC1AD01A50800B17E0800E0714CD
:1097500014E02050010B11E1216B1A9E0A01DA8FEF
:1097600067EC0CF04AEC75F01EAC03D002010989DD
:1097700002D00201068B050147850201215102E159
:10978000238A25820D5107E01D50400B04E00D0790
:109790000D5101E11D8E0501165101E01607020170
:1097A000355105E03507355102E1C6EC0AF00201FA
:1097B000B05101E0B007D0510DE0D007D0510AE11F
:1097C00007010A83BEECC4F043EC53F002011851C8
:1097D00001E111942C5101E02C070101AC5101E190
:1097E000A3D0AC07AC5101E09FD0B59DB59F2F9899
:1097F000E4951C921B9830AC02D033EC50F02FBA99
:1098000005DB23BE96DA24B05ADB2582238A27980B
:1098100020BA02D01FEC27F0208A0C0E155C29E13B
:109820002150200B26E00101AA5123E1156881ECAB
:10983000CCF002E11E8417D001013B71129C3B5118
:10984000010B01E0128C6DEC99F0540E9FECCAF004
:1098500001013BA108D04B0EE66ECC0EE66E26EC65
:109860000AF0E55204D0550EE66EFFEC26F0E55204
:109870001A861D50400B11E02A50800B0EE121503A
:10988000200B0BE02A8E130EB6ECCEF0460EE66EE1
:10989000410EADECD1F0DDEC08F00101E8A909D0F2
:1098A000E899E887710EE66ED40EE66E010EF6ECCE
:1098B000CDF02550040B38E00B0E155C35E121503E
:1098C000200B32E00101AA512FE120982594B59B8D
:1098D000B599E67DE6AD1AD0E8A30AD0330EE66E60
:1098E000E40EE66E010E12ECCAF00101198F09D0E8
:1098F000800EE66ED40EE66E010EF6ECCDF00101A0
:10990000E887E883500EE66EC60E0CD02B0EE66E8E
:10991000E40EE66E010E12ECCAF00101198F500E32
:10992000E66E4E0E78ECCAF002011D5101E01D07F3
:10993000045101E004071E5101E01E071F5101E020
:109940001F07345101E034070101AD5101E0AD07BB
:109950000201235101E02307395101E03907D851B1
:1099600008E0D807D85105E19EEC48F002010E0E40
:10997000D96FD95101E0D9073A511CE02150200B91
:109980000AE1110E28ECD6F03AC23EF00BECD5F00D
:1099900002E10601067B02013A072150200B05E097
:1099A0002050400B02E085EC05F002013A5102E143
:1099B000ABEC04F0060143510AE04307435102E1D6
:1099C0005A0E436F25860F0E435D01E22596020174
:1099D000225108E02207225102E1B2EC69F00201B3
:1099E0001E0E216F3B5110E001012651400B0CE18E
:1099F00002013B073B5108E144C100F01886C9EC65
:109A000096F00201010E246F0201245141E0240767
:109A100024513EE10101395103E00901010EEB6FD0
:109A20000901ED6B27ECD5F00101E78F7FECC5F064
:109A30000201186BD05101E111942AECCFF020A261
:109A400004D02092ABEC2EF014D0A4ECD4F0B5EC02
:109A500016F0640E16ECCAF069ECE3F00BECD1F0F2
:109A600008E02050200B05E0010EE66E02EC9AF0B3
:109A7000E55218B002D058ECD9F0189002010689CE
:109A80001EAC02D0098709850501BF0E476F4881CA
:109A90000201365104E03607365101E12582255195
:109AA00001E02507D25109E00501105106E102014C
:109AB000D207D25102E152EC0AF002011B5106E03A
:109AC0001B071B5103E1630E52ECCAF002011C514B
:109AD00006E01C071C5103E1B10E52ECCAF0020172
:109AE0001A5105E01A071A0502E132EC10F00201E2
:109AF0002E5101E02E07120006014F6B4FC64EF6A5
:109B00004FC64DF64FC64CF64FC64BF6120063ECEF
:109B1000D5F0DE52010EDD6EFE0EDB501AE125ECB3
:109B2000D9F0050EE66E200EDF24E66E4B0EE66ED3
:109B3000060E55ECCAF0050EFBECDAF0BA0EE66E36
:109B4000010E55ECCAF00F0E72ECD8F00050DF6E2B
:109B5000096A0101BA51630805E3BA510EE11F0E0B
:109B6000BB5D0BE2360E006EC7EC26F0FE0EDB503E
:109B700001E1C2DF010EDB6A22D0FE0EDB501FE1E5
:109B80002C50800B07E0DF500A0804E20701BE9B5F
:109B90007EEC09F0DFCFE6FF4BEC34F0E55201013B
:109BA0008A51100B0CE00A0E445D09E28EECDBF0EA
:109BB0007CECD8F0DFCFE6FF8BEC80F0E5520201C1
:109BC000295115E1640E0101445D0BE28CECCAF0F1
:109BD00044C13EF0B3ECCCF00101166F300E3A24D4
:109BE00005D04D0E166F030E4415310F176F016A25
:109BF000050E015C2EE2A10E496EDB0E4A6E010ECF
:109C00004B6E0150EA6A4B0FE96E060EEA22EFCF67
:109C10004CF057ECDBF0026E2D0E025C05E1010109
:109C2000B65102E1200E026E0201295110E1020E2E
:109C3000012489ECCBF002C0EFFF015008E12B9A20
:109C40002A0E025C04E12C50800B01E02B8A012AD1
:109C5000CFD70201295102E10101188F010EDB501B
:109C6000FCECD2F002E2E16AE552E16E4950E3EF2A
:109C7000C9F06AECD4F0016E44512BECCCF0050E27
:109C8000E66E4B0EE66E060EE66E200E01245CEFCD
:109C9000DBF00201050EB86FF00EB96FFA0EBA6F65
:109CA000140EBB6FF00EBC6FFA0EBD6F1200016A8E
:109CB0000101D45102E0010E016E015014ECD6F006
:109CC000EF50006ED2AD006A015087ECCAF0EF5041
:109CD000E66E015014ECD6F0010EF3ECDAF0E66E0D
:109CE0000050E66E250E49ECCCF001011496D251DD
:109CF000400B01E014861200026A0101D45102E017
:109D0000010E026E025087ECCAF0EFCF49F0190E37
:109D1000E1ECCAF09AECCEF002E1200E1B6F4E0E81
:109D2000186F520E196F57EF4EF0238E1F967CEF6F
:109D30004EF0239E4CEFD1F0020EE66EBD0E42ECCB
:109D4000CAF00101D0BB0FD0BB0E52ECCAF0010E1D
:109D5000E66E200EE66EE66A2F0EE66E78EC16F0E2
:109D600064ECDAF03AD0070E0201935D18E29351E9
:109D7000E824496E4A6AFF0EE2ECD7F0E66E060E62
:109D8000D8809355070DF3500A0FE66EBC0E0DEC0C
:109D9000CAF0010EE66E200EE66EE66A17D0F30EEC
:109DA000E66E0A0EE66EBC0E0DECCAF0020193518F
:109DB0000A0802E2030E01D0010EE66E0F0ED880F3
:109DC00093550C0DF350E66E800EE66E2F0E49ECA7
:109DD000CCF0B90EE66E39EC16F0E55201011494A0
:109DE000D051200B01E014841200020193299AEC57
:109DF000CEF002E1200E1B6F4E0E186F420E196F4F
:109E00009CEF4EF02F8A1F96F5EF4EF02F9A4CEFF5
:109E1000D1F09EECDBF0BDECCAF017E1020E016F51
:109E20000201872911ECD4F037ECD8F0030EE66E6E
:109E3000020EE66E3EEC09F0E552E55201011C8F80
:109E4000500E166F4C0E176F1200030ED45D10E10A
:109E5000AEECCDF006E0230EE66EE40EE66E010EEB
:109E600005D01B0EE66EE40EE66E010E8FEFD7F006
:109E7000016B29C100F02BECD5F00101165D02E168
:109E8000200E166F300E196F480E1B6F5A0E1C6F86
:109E900012002450010B09E1BDECCAF006E0AEEC63
:109EA00016F0030E006E7CEC75F02480BDECCAF059
:109EB00003E00068D2EC26F01F9609EF4FF0BDECEE
:109EC000CAF005E113EC09F046EC1FF004D0C6EC33
:109ED0000AF0B5EC16F024901A940101AC6BB59F12
:109EE00023980FEC0DF03BEF0EF08EECDBF00A50F8
:109EF00018E01F0E006E010196BB02D03F0E006EEF
:109F0000030E0A5C02E02D0E006E80ECE1F0010110
:109F10000E5102E1100E0E6F002B8B0E006E10EC36
:109F200026F09EECDBF0300E496ECE0E4A6E010E2E
:109F30004B6E0A5019ECDBF017C1E6FF16C1E6FFC5
:109F40000EEC0AF0E552E552010136AD02D090EC7C
:109F5000DFF0120032800068C7EC26F004ECD5F088
:109F60001F96C3DF6FEF39F032900FEC0DF001DA7E
:109F70002F98120085ECD5F0140DB8ECCAF017EC50
:109F8000D5F005E006ECCCF0230E0DECCAF04FEC5A
:109F900015F0140E16ECCAF0E3EFC9F0E7ECC9F0C7
:109FA000B6C200F0FE0EDB5001E1006AB7C2E6FF68
:109FB0000050E66E240E0DECCAF0E3EFC9F0070185
:109FC0008B51845D15E11450100B01E0010E496EB8
:109FD0003350010B495C0CE11450200B01E0010EE1
:109FE0004A6E3350020B01E0010E4A5C01E112009F
:109FF00084C78BF7339014B83380339214BA33820A
:10A0000014A80BD014AA03D084C7E6FF07D0E66AD1
:10A01000B1DFE552010EE66E04D0E66AABDFE55231
:10A02000E66ABCDFE552120007018451140D37ECDB
:10A03000D8F019C116F11AC117F11BC118F11CC1D2
:10A0400019F10101200E1A6F480E1B6F5A0E1C6F7A
:10A05000300E165D02E1200E166FDFEF4FF0308CF0
:10A060001F9614EF50F0309C2F980101AC6B239891
:10A07000B59F0FEF0DF00101AC5103E02450080B28
:10A0800003E0B551200B01E02F88005032ECCDF0F9
:10A090000101AC5106E02F50100B03E1FA0EAC6F3A
:10A0A00024861200010E0701D89056375737E8066C
:10A0B000FBE121AC02D0070156810D0E0701585D6E
:10A0C00001E2582B1200219C8450020B01E0218CEC
:10A0D00007014E5111E121AC78D04E2B010E566F85
:10A0E000576B586F3098596F5151FE0BE84251250C
:10A0F000506F010121931200010121A366D0219329
:10A1000007014E0562E121BC52D030A84DD00C0EA3
:10A11000585D47E2D89057335633006A5F0E005CB3
:10A120001BE24A0E4B6ECD0E4C6E010E4D6E005072
:10A130004E6EEFECCBF0565149180CE157514A18CE
:10A1400009E1200E0026610E005C02E3200E005E95
:10A1500092DF02D0002AE2D75F0E005C22E1070105
:10A160001F0E561901E157510AE01D0E561901E163
:10A17000575105E0EF0E561905E1575103E1200E46
:10A18000006E79DFFF0E0701561902E1020E571922
:10A1900006E0B50E561905E1030E571902E1CAECA7
:10A1A0006FF007014E6B1200308852EF50F07ADFEB
:10A1B00030A804D00701010E596F06D00701592BB2
:10A1C00059510C0801E24E6B3098120007AE06D0D0
:10A1D0008450020B02E0219C01D0218C07014E51DA
:10A1E00010E121BC75D00101219307014F6B07AE2F
:10A1F0006FD0020E4E275151FE0BE8425125506F91
:10A2000012004E050BE14E2B51C750F7010121936F
:10A2100021AC5ED00701080E4E6F1200010121A390
:10A2200057D02193070E07014E5D46E14E6B21ACDE
:10A2300040D00101AC5103E02450080B03E0B551BC
:10A24000200B01E02F88290E496EDB0E4A6E010EAD
:10A250004B6E07014F51522570ECD5F0006E810E08
:10A26000005C02E1526B1BD0800E005C03E1200E0B
:10A27000526F15D00D0E005C03E00A0E005C02E187
:10A28000200E0BD00B0E005C02E12A0E06D00A0E47
:10A29000005C05E0005003E0005032ECCDF001011D
:10A2A000AC5109E02F50100B06E1FA0EAC6F24867A
:10A2B0001200080E4E6F1200080E4E5D04E121AC34
:10A2C00007D04E6B12004F914F4321BC4F894E2B4C
:10A2D00012009EECDBF03AECCCF013E11FECD5F071
:10A2E00006E0140E496EE40E4A6E010E05D09F0E74
:10A2F000496EF20E4A6E010EFDECD7F07EECCAF00C
:10A3000018D0EAC600F00050020802E2020E006E09
:10A31000080E496ECE0E4A6E010E4B6E005019ECBF
:10A32000DBF00601EA51020804E2EA05300F010100
:10A330001C6FB9EC1FF0C4EC0FF0006E00500A0166
:10A34000D65D04E200C0D6FA73ECCCF01200010135
:10A35000D45105E1308404ECD5F01F9603D0006899
:10A36000E9EC26F069EF51F030940FEC0DF0B9EF05
:10A3700051F0040EE66EEA0EE66E060EE66EA00ED4
:10A3800081ECD6F0140E016E3CC100F013EF3BF0EF
:10A390005FECD5F0E0C649F0E1C64AF0D890493606
:10A3A0004A360601A8ECD4F00CE3DEC64BF0DFC65B
:10A3B0004CF0D8904B364C36E0514B5CE1514C5848
:10A3C00020E2DE51E0250E6EDF51E1210F6E55ECEB
:10A3D000D2F0E2C649F0E3C64AF0030E7CECD0F0BE
:10A3E000FDE149500601E25F4A50E35B57ECD6F0CD
:10A3F000030E7CECD0F0FDE149500601E2274A5003
:10A40000E323DEC6E0F6DFC6E1F6B3ECD1F0493671
:10A410004A36D89049364A36A8ECD4F00BE3B3EC70
:10A42000D1F04A32493230ECDAF04950DE5D4A5020
:10A43000DF5902E2DF6A09D0E251DE5DE351DF5904
:10A4400002E2010E01D0020EDF6EB3ECD1F049360C
:10A450004A364950E225E46F4A50E321E56FDF5068
:10A46000E552E3EFC9F01DBC1200219C8450020BA1
:10A4700001E0218C21AC03D002016C2B02D002013F
:10A480006D2B1F9E0601E65109E121AC4BD0010E58
:10A49000E66FDE6BDF6BE76BE86B44D0E60515E13A
:10A4A00021BC40D0020EE66F73DF006E00500BE05F
:10A4B000070E0601E85D07E2E82BE791E74300504D
:10A4C000010801E2E78F06011FD0020EE65D2AE1D6
:10A4D00021AC1DD0E2C64BF0E3C64CF0030E0F0BCF
:10A4E00005E0D8904C324B32E806FBE106014B50B8
:10A4F000E25D496E4C50E3594A6E4950DE5D4A5068
:10A50000DF590EE2010EE66FDE6BDF6B0BD0E4511C
:10A51000E425496EE551E5214A6EA8ECD4F002E24B
:10A52000030EE66F030EE65D43E1E791E743E78F35
:10A53000070ED880E855016E01500106000903E0BE
:10A54000E791E743F9D7780EE75D30E20101AC51BE
:10A5500003E02450080B03E0B551200B01E02F88E5
:10A56000E7C6E6FF3CEC04F0E552006E200E005C0E
:10A5700003E300506E0802E22A0E0BD0298A005035
:10A5800032ECCDF00601DE51E45DDF51E55903E226
:10A59000200E32ECCDF0299A0101AC5107E02F508A
:10A5A000100B04E12486FA0EAC6F30860601E66BD0
:10A5B0001F8E12000101E583D45102E154DF07D060
:10A5C0001F9EC5ECD0F002E07EDD01D0FFDD010171
:10A5D000E5931200800E071420E02A50020B1DE1C3
:10A5E0002050200B1AE00201A95117E10101D451BA
:10A5F00004E10601EA51010806E33AECCCF00DE172
:10A600001FECD5F00AE02A0E0101B51506E10C0E8B
:10A61000155C10E12150200B0DE0800E071409E1BC
:10A620000AECCBF006E00601EC5103E002012D51EB
:10A6300001E0000C010C0201395103E1120E9FEC04
:10A64000CAF012005FECD5F066C1DFFF0101665170
:10A65000140804E26651E824EC0FDF6E21A204D056
:10A660006651F2ECD8F0DF5E1EBCDF6ADFCFE6FF9A
:10A67000720E42ECCAF030800201078334B0DBDF97
:10A68000E552E3EFC9F05FECD5F067C1DFFFBDEC49
:10A69000CAF002E1DF6A05D007010AB302D00F0E4B
:10A6A000DF5EDFCFE6FF710E42ECCAF002010787E2
:10A6B000E552E3EFC9F063ECD5F0D00EDE6E070E85
:10A6C000DD6E01014851320804E28C0EDE6E0A0E86
:10A6D000DD6EE6A510D0D00EDE6E070EDD6E6EECE0
:10A6E00020F0010804E06EEC20F0020820E1340EB6
:10A6F000DE6E080E1BD0090E2B5D0DE25F51020BC2
:10A700000AE02250100B07E13450800B04E10201F3
:10A710000B517D080CE2B80EDE6E0B0EDD6E0101F2
:10A720004851780804E2800EDE6E0C0EDD6E5CECA3
:10A73000CBF002E3000E01D0010EFCECD2F002E2FD
:10A74000E16AE552E16E4950E3EFC9F063ECD5F000
:10A7500039EC11F0C5EC48F0BDECD0F002E02ADF96
:10A7600002D01FBE1F9E2450200B06E00201245180
:10A7700003E1F6ECC4F0249A02012B5102E0C2EC92
:10A780003DF00101B75111E1E66A04EC2CF0E5520D
:10A79000006E1DAC9FEF5AF00701A151F00BE83A93
:10A7A000A15D0024A16F9FEF5AF0B7050DE15AECAF
:10A7B00071F06FEC27F077EC18F01E92E8A09FEF95
:10A7C0005AF01E829FEF5AF0020EB75D04E1C4EC0E
:10A7D000DBF09FEF5AF0030EB75D07E12EB49FEF59
:10A7E0005AF0EFECE0F09FEF5AF0040EB75D01E095
:10A7F000B4D00201255102E09FEF5AF01750100B20
:10A8000006E11750010B03E11750200B02E0000E88
:10A8100001D0010E2290E8B0228021AA45D09BEC05
:10A82000D1F0166E22A036D00101AA512AE1090EFC
:10A83000155C17E181ECCCF014E10101AB510BE1A7
:10A84000A00E176E99EC09F000093CE00BECD1F07A
:10A8500039E11A8637D0165035E1AB6B900E176E82
:10A860001FD0165002E1010E01D0100E8009176EA4
:10A8700099EC09F0000926E00BECD1F023E11A84F1
:10A8800021D016501FE1AB6BABC1AAF1810E176E40
:10A89000219A06D0165016E12250010B13E1219A9D
:10A8A0000201020E256F0ED031B40CD0E66AFDEC29
:10A8B0003DF0E552000906E031840201020E256FE9
:10A8C00007AE256B3150040B02E19FEF5AF00201F5
:10A8D000255102E09FEF5AF031949BECD1F0166EB7
:10A8E000165002E19FEF5AF08CEC04F00201A96BC4
:10A8F0000101280EAA6F150E165C05E12050400BD1
:10A9000002E01E0EAA6F080E165C06E0290E165C09
:10A9100003E0100E165C02E12D0EAA6F0201020E7A
:10A92000256F218A176A1650156E99EC09F00009F7
:10A930000BE001013651800B07E00201355104E1C3
:10A94000040E006E7CEC75F028B602D00101AE6BEF
:10A95000BCEC0CF02A849FEF5AF0050EB75D21E1A4
:10A96000A1ECCBF00FE01B50080B0CE1A5ECCEF0F6
:10A9700009E2A5ECCEF006E202011E0E186F2AECE9
:10A98000CFF0118401012651100B02E09FEF5AF025
:10A990002751100B02E09FEF5AF0C2EC3DF09FEF01
:10A9A0005AF0060EB75D07E120AA9FEF5AF0D8ECE7
:10A9B00007F09FEF5AF0070EB75D02E19FEF5AF0E4
:10A9C000080EB75D01E089D32550800B0AE0020133
:10A9D000285107E1020EC1ECD6F002011E0E286FCD
:10A9E000259E25AC03D018ECCFF0259C25AA03D0DA
:10A9F000C6EC0AF0259A01013651800B1BE00201DA
:10AA0000355118E11AA404D0040EC1ECD6F01A9402
:10AA10001AA604D0070EC1ECD6F01A961AA804D0D4
:10AA2000060EC1ECD6F01A981AAA04D0050EC1EC95
:10AA3000D6F01A9A0101B5BDA7D0B5A967D020AE4E
:10AA40000FD0AD5101E07BD02BA805D00B50E66EA6
:10AA50001DEC3FF003D0E66AE3ECBDF0E5526FD0A9
:10AA600024A003D049EC4FF06AD032A012D026AD1A
:10AA70000DD0C5ECD0F002E00101967BBCEC0CF0EF
:10AA800046EC1FF0B9EC1FF075EC4FF00101269D6C
:10AA900034D02C50400B03E12C50800B30E026AD1D
:10AAA0004ED0CEEC08F00101B6511AE1630EE66E0D
:10AAB000440EE66E010E1EECCDF044C10CF2020114
:10AAC0003B6BA7ECD0F0000917E02C50800B14E092
:10AAD00001018E51100B10E10201100E3B6F0CD0E2
:10AAE000290EE66EB6054A6A4B0F496E060EA3ECB8
:10AAF000D7F0ADECD4F0E5520101AD6B20D021B61A
:10AB00001ED059C200F0C7EC26F019D0B5A305D06D
:10AB100025A215D02592228212D0B5A110D025A24F
:10AB200006D025922BC1E6FF4BEC34F0E552020132
:10AB3000215105E11A50400B02E16FEC39F0E5ECD0
:10AB400014F0006EFF0820E0570E005C07E18EEC69
:10AB5000DBF0220E006EC7EC26F016D01B0E005C58
:10AB600003E195ECC3F010D0FF0E015C0DE08EEC1C
:10AB7000DBF00101140E116F0D0E126F050E006F48
:10AB80000150006E80ECE1F00101B5BF8ED2B5AB93
:10AB9000F6D02CA603D046EC40F071D230AC03D0F6
:10ABA00014EC50F06CD22FAA05D023AA68D2F5EC91
:10ABB0004EF006D023AE06D023AA61D27CEC4EF034
:10ABC000239AA8D024A003D009EC4FF058D22CA48B
:10ABD00003D019EC40F053D2E6AF03D0C6EC3FF0FF
:10ABE0004ED219A803D09BECD4F0B1D03050040B56
:10ABF0001BE0D45119E127AD0DD0010E0D6E27BF1A
:10AC00000D680A0EE66EEA0EE66E060E20ECCAF03D
:10AC100073ECCCF02350200B04E101012751400BD1
:10AC20003FE069EC51F03CD032A03ED027AD16D0C9
:10AC3000010E0D6E27BF0D680AC006F1030EE5EC8C
:10AC4000D5F01EECCDF006C10AF06DECD7F00A503D
:10AC50009DECD6F0B9EC51F0050147852350200B4F
:10AC600003E00BECD1F004E001012751400B18E0A8
:10AC7000BCEC0CF05EECD9F075EC4FF002010881F1
:10AC8000050147871EAC02D0020109851F50020B47
:10AC900005E0C5ECD0F002E0B9ECD1F0F0EC39F011
:10ACA0000101279D239A37D02C50400B03E12C50F3
:10ACB000800B33E023AA04D0239AADECD4F047D024
:10ACC00027ADDDD1279D010E0D6E27BF0D68006AEF
:10ACD000050EE66E0050E66EB60EE66E010E25EC31
:10ACE000CAF00601030E426F0101B6510EE0B6290B
:10ACF000496E010E495204E0E846FE0B4906FCE1AC
:10AD00000601426F1E0E436F02D039EC4EF0ADECDF
:10AD1000D4F0E5520101AD6BB2D120AE1AD0AD51E5
:10AD200001E0ADD185ECCBF001E0A9D10B50016E73
:10AD30002250100B03E13450800B02E01FEC68F04E
:10AD4000006A0050B6ECCDF055EC3FF0E552E5520C
:10AD500096D121B694D15AC200F0D2EC26F0A30EBF
:10AD600002015A5D01E08BD1A4ECCAF001E187D168
:10AD70000AECCBF001E083D10101320E20D0B5B353
:10AD80007ED1B5A71ED01950400B04E01950040B1A
:10AD900001E075D19EECDBF00A0E006E25EC26F08A
:10ADA0000101040E016F03C700F019AC02D094EC4E
:10ADB00004F09DECE1F019AC62D10101200E1A6F94
:10ADC0005ED13BAB46D1070E006E0050D880765561
:10ADD00001E2766B27AD10D0279D010E0D6E27BFC7
:10ADE0000D680050E66E760EE66E010E20ECCAF09D
:10ADF0000601426B0101AD6BAD5101E040D1205025
:10AE0000200B01E13CD10201A95101E038D1070E2C
:10AE10000101765D40E19EECDBF0A7EC16F001014C
:10AE20002B0E166F00010FAE0BD001012D0E166F09
:10AE3000FF0ED8800E560F56010E0E26000E0F2262
:10AE4000E70E80ECD0F002E2B1ECD4F00E500F101F
:10AE500003E10101200E166F57ECD6F0640E43ECAF
:10AE6000D6F039C049F03AC04AF04950006E0101AD
:10AE7000012B9DECE1F082EC04F0300F0101176F23
:10AE8000300E175D02E1200E176F198F640E1A6FD6
:10AE9000420E1B6FD0D0060E765D1EE19EECDBF0FD
:10AEA000A4EC16F0A1ECCCF00101410E166F460E99
:10AEB000176F560E186F300E195D01E0E0D0200EAE
:10AEC000196F300E1A5D01E0DAD04FECD8F001E0D6
:10AED000D6D0200E1B6FD3D0040E765D03E0050E96
:10AEE000765D6CE19EECDBF00498050E0101765D69
:10AEF00009E14F0E166F530E176F430E186F64EC77
:10AF0000D9F026D0500E166F410E176F048885ECCD
:10AF1000CBF006E00101580E186FEAC900F01AD014
:10AF20000101E6A50DD0320E186FE5A902D0340E4E
:10AF3000186F45ECD2F0ABC73DF0ACC73EF008D07F
:10AF4000490E186F45ECD2F0A9C73DF0AAC73EF0F4
:10AF5000B5ECDAF0049000AE02D0006C0480010180
:10AF6000030E016F5EECCFF004A002D02D0E196F1E
:10AF7000430E1C6F04B8188F050E765D0FE196A383
:10AF800002D0230E09D05751100B01E178D0575150
:10AF9000200B01E174D02A0E196F71D0E651040B19
:10AFA0006EE08A51400B6BE0A1ECCBF068E101014F
:10AFB0004E0E1A6F2F0E1B6F410E3ED0760514E118
:10AFC0009EECDBF0100EE66EE40EE66E010E8FECEA
:10AFD000D7F00BC200F02BECD5F00101195D02E1B6
:10AFE000200E196F1B8F27D0020E765D27E19EEC95
:10AFF000DBF0080EE66EE40EE66E010E8FECD7F085
:10B00000010183513CE033AC02D02A0E186F060ECA
:10B01000E66E820EA1ECD3F0005002010B5D006ED3
:10B020000101030E016F2BECD5F00101195D02E166
:10B03000200E196F1B8F560E1C6F21D0030E765DEC
:10B0400003E1A6EC10F01BD0765119E109ECE4F015
:10B0500016D0020119510BE02750400B10E1140EDD
:10B060000101AC5D0CE23B0E00ECCBF008D001011D
:10B07000B5A105D023AA03D0239AF8EC34F0E5EC6F
:10B0800014F0006EFF0811E0570E005C0AE104ECBA
:10B09000D5F0000EE66EE40EE66E010E8FECD7F0F2
:10B0A00004D00050006ED2EC26F00101AD5101E059
:10B0B00046D2140EAD6F0201565101E05607020E42
:10B0C000685D01E03CD2330E0101B95D04E00E0E73
:10B0D000B95D01E034D2258232D2090EB75D0AE1B2
:10B0E00006015051515D01E12AD250C651F697EC4C
:10B0F0003DF025D20A0EB75D05E1C9ECDFF094EC16
:10B10000DFF01DD20B0EB75D01E019D2B85124E17A
:10B11000E5EC11F000ECD6F001E10BD28A51400BC6
:10B1200009E0A1ECCBF001E104D2040E0101765D4F
:10B1300001E0FFD153EC13F00701BC0ED880AB55F2
:10B14000020EAC5501E3F5D101018A51400B01E03B
:10B15000F0D10AECD7F007D1B8053EE154ECD1F0BC
:10B1600001E3E7D154ECD1F001E3E3D11B50080B2C
:10B1700001E0DFD10101485132080FE2770E00EC07
:10B18000CBF090ECDFF0B6ECD4F034ECDAF0E30E78
:10B19000E66EE30EE66E010EDED0C80EBFECDAF00E
:10B1A00034EC13F00701A80EDDECD9F00DE2D20E5D
:10B1B000E66EE30EE66E010EE5ECCAF0CA0EE66E30
:10B1C000E30EE66E010E9BD0760EDDECD9F001E3C6
:10B1D000B0D10AECD7F0E8D0020EB85D01E0EAD0B9
:10B1E0005CEC10F0A1ECCBF001E195D02050040B09
:10B1F00001E091D02050400B01E08DD05E0EDE6E5C
:10B20000010EDD6E01012B51090804E2900EDE6E85
:10B21000010EDD6EE6A504D0F40EDE6E010EDD6ECD
:10B2200021B204D0640EDE26000EDD225CECCBF0F1
:10B2300001E37FD11B50080B01E07BD15CEC10F0E7
:10B24000ECECD8F05CECCBF001E373D15CEC10F0EB
:10B25000050E16ECCAF05CECCBF001E36AD12CA62B
:10B2600009D0A4ECCAF003E00AECCBF00AE0A4ECAD
:10B27000D8F007D001016651ACECD0F0665F22EC4B
:10B2800053F0460EBFECDAF05CECCBF001E351D1A9
:10B29000170E9FECCAF02CA609D0A4ECCAF003E06C
:10B2A0000AECCBF011E0A4ECD8F00ED0B20EE66EB2
:10B2B000E30EE66E010EE5ECCAF001016651F2EC18
:10B2C000D8F0665F22EC53F0960EBFECDAF024EC77
:10B2D000D8F0320E1CECD3F00201CD51495CCE51B6
:10B2E0004A5801E326D19F0EE66EE30EE66E010E8C
:10B2F000E5ECCAF0970EE66EE30EE66E010E47EC43
:10B30000D3F0CCEC10F0010EE66EE1EC10F0E5525B
:10B3100012EC11F00ED15BEC53F0000901E109D100
:10B320001B50080B01E005D15CEC10F05BEC53F016
:10B33000000901E1FED0170EE2ECD9F00101E6A50B
:10B3400014D048510EE0480537ECCDF0890EE66E7A
:10B35000E30EE66E010EE66E91EC14F0E552E55256
:10B36000E7D0ABECD8F0209422D04851320809E263
:10B37000680EE66EE30EE66E010EE5ECCAF0320EE4
:10B380000BD048511E080EE25A0EE66EE30EE66E32
:10B39000010EE5ECCAF01E0E37ECCDF0B6ECD4F0A1
:10B3A000640E83D0ABECD8F02094B6ECD4F055EC1E
:10B3B000CEF0BFD0030EB85D34E1060150932450A7
:10B3C000020B12E11F50020B04E00FEC2AF00009FF
:10B3D00009E01250080B03E11250040B05E029ECC0
:10B3E000D4F002E0060150832450020B01E0A1D00A
:10B3F000E0ECD2F001E09DD00201305101E099D0A3
:10B4000044ECCEF001E14A5001E193D02C50800B86
:10B4100001E08FD02C50400B01E08BD00601018160
:10B4200088D0040EB85D4DE11F50080B48E0A1EC38
:10B43000CBF045E01BECD5F042E1D0ECD0F03FE1A1
:10B4400056A53DD0D70E3CECCDF02ABC24D0FFEC65
:10B45000D6F004E68F0E495C000E4A586AE2140EDC
:10B4600016ECCAF0D70E1CECDAF0016E050E16ECE5
:10B47000CAF0D70E3CECCDF0040EB6ECCDF0005087
:10B48000E66E0EECCEF055E02A8C35EC0CF00201A5
:10B49000090E336F4ED0EFECD8F00BE249508F0815
:10B4A000000E4A5406E22A9C140EE66EBFEC21F010
:10B4B0003FD0020133513DE135EC0CF03AD02A9CEB
:10B4C00038D0050EB85D35E1A30E3CECCDF001019E
:10B4D000E5A105D00050E66ED7EC75F0E55204907A
:10B4E0002150020B01E00480C00E005C02E22192B8
:10B4F00004D00050F00801E221822150020B02E04A
:10B500008F9001D08F800450010B496E2150020BA7
:10B5100001E0010E495C0DE08CEC04F0FEEC16F04D
:10B5200022EC53F073ECCCF0010EE66EE4EC1DF06F
:10B53000E5520101B82BB851050801E2B86B0101D1
:10B54000B72BB7510B0801E2B76B020EE15C02E2C8
:10B55000E16AE552E16EE3EFC9F0016A750E015C44
:10B560000DE2E60E496ED90E4A6E010E4B6E015089
:10B5700070ECD5F0CDECD0F0012AF0D71200026AC1
:10B58000400E025C08E2B00E0224016E320ECDECD9
:10B59000D0F0022AF5D7120054ECD8F0060F016E55
:10B5A000040EB6ECCDF08D0EE66E020E55ECCAF030
:10B5B000096AE3EFC9F054ECD8F0060F016E040EEF
:10B5C000E66E8D0EE66E020EDCECD7F0E3EFC9F00E
:10B5D00054ECD8F00A0F016E020EB6ECCDF0910ECD
:10B5E000E66E020E55ECCAF0096AE3EFC9F054ECBE
:10B5F000D8F00A0F016E020EE66E910EE66E020E94
:10B60000DCECD7F0E3EFC9F05FECD5F0340EA8EC3A
:10B61000D3F0010E096EDF6A100EDF5C42E2026AAF
:10B62000100E025C3CE2C4ECD6F003E0050E025CB6
:10B6300006E1DF50E824820F78ECCCF0006E0204C3
:10B6400003E0060E025C07E1DF50E824820F010FE1
:10B6500078ECCCF0006E020EDF5C03E3030EDF5CDF
:10B660000AE10A0E025C02E1110E006E0B0E025C92
:10B6700002E1240E006E0C0E025C05E10A0EDF5C96
:10B6800002E11B0E006E0D0E025C05E10A0EDF5C8E
:10B6900002E1200E006E13EC3BF0022AC1D7DF2A34
:10B6A000BBD7020E096EDF6A090EDF5C12E2026A86
:10B6B000100E025C0CE2C4ECD6F003E0050E025C56
:10B6C00002E11C0E006E13EC3BF0022AF1D7DF2AD8
:10B6D000EBD7096A42DFDF6A200EDF5C09E2100E59
:10B6E000006E800EDF24016E13EC3BF0DF2AF4D7EE
:10B6F000DF6A0B0EDF5C03E242DFDF2AFAD7DF6A84
:10B70000090EDF5C35E2DF28006E0038F00B006EBA
:10B71000090E0012DFCFE6FF27EC0CF0E5526BECD0
:10B72000D9F0EE52090EEF6E1BECCAF0020E7DEC62
:10B73000D6F02C0EEF6E1BECCAF0030E7DECD6F0AB
:10B74000010EEF6E1BECCAF0040E37ECD7F0050EBD
:10B7500037ECD7F0070E37ECD7F0080E37ECD7F000
:10B76000060E37ECD7F0090E33ECCFF0DF2AC8D73E
:10B770001FD829D8DF6A060EDF5C0DE2DF5002E138
:10B78000030E01D0010EE66EDF504DECCBF07DECE8
:10B79000CCF0DF2AF0D77AECDAF0FD0E016EDB0E8A
:10B7A000CDECD0F00101010EB56FE552E3EFC9F029
:10B7B000020E096E5A0EE66E000EE66E030EE66E7F
:10B7C000A20E5CEFDBF0F7ECDAF0030E096EFE0E72
:10B7D00073ECDBF0850E005C02E0010EDF6E2D0ED7
:10B7E000A8ECD3F0140E17ECD1F0000EE66E0A0EA2
:10B7F000B3ECCAF00A0E17ECD1F0CA0EE66E0A0ED0
:10B80000B3ECCAF0040E17ECD1F0260EE66E0A0E69
:10B81000B3ECCAF0DF501DE00F0E17ECD1F0140EA0
:10B82000E66E0A0EB3ECCAF0030E17ECD1F0230E4D
:10B83000E66E0A0EB3ECCAF00A012D0E1B6F1BCA8E
:10B840001AFA1BCA19FA410E206F20CA1FFA20CA21
:10B850001EFA0A01D46BDA6BDA81D56B380ED66F1B
:10B86000040ED86F3C0ED96F190ED76F016A020E05
:10B87000015C0CE20150050D60ECDBF0000EE926E6
:10B880000A0EEA22360EEF6E012AF1D70101D46BBF
:10B89000050ED45D18E20701010EB16FFF0EB15D18
:10B8A0000FE003EC14F0D2ECDAF0F2ECD7F0070181
:10B8B000B151A5ECDAF009ECCDF00701B107EED7F4
:10B8C0000101D42BE5D70701B16B0101D46BDFCFA8
:10B8D000E6FF59EC48F0E55291EC48F0030E096E92
:10B8E000FE0E016E850ECDECD0F0096AE552E3EF55
:10B8F000C9F00490049201013EB104803EB3048279
:10B900000450010B02E08E8E01D08E9E0450020B7B
:10B9100002E08F8801D08F984051E8240A0FE66E2C
:10B92000E66A86ECFCF0E552E5520C0EBB6E006A4E
:10B9300001013E5104E1100E3F03F350006E005030
:10B94000BC6E1200E7ECC9F095ECD5F053ECFDF0BD
:10B95000E552000902E0C69EF7D7E3EFC9F0C79EA3
:10B96000C698C78C1200C78EC688C78C1200F29E7C
:10B97000AFECD0F0480EE6ECD9F0480E3BECD7F037
:10B98000480EF6ECC9F00701800E146FF90E156F22
:10B9900077ECD5F07EECD5F0F28E1200D9CFE6FF31
:10B9A000E1CFD9FF030EE12613EC10F0E668930E09
:10B9B000E66EDFECFCF0E552E552AA9EC26A00009A
:10B9C00000000000000000008A8A209A3386278A3F
:10B9D0001AEC14F00601B66BB76B3DEC0DF057ECAA
:10B9E000C4F0F6ECC4F092688F0EE66EE66800ECE8
:10B9F000FBF0E552E552CF0EE66EE66851ECFCF046
:10BA0000E552E552050EE66E71ECFDF0E5520101DE
:10BA1000010E3E6F0101030E3F6F0101020E406FE8
:10BA200068DFE668870EE66EB5ECFCF0E552E5529D
:10BA3000B09E0201320E116F000EA56EA26E9F6EB7
:10BA4000A282D08E010EC26EC16A0A0EC06E0F01B4
:10BA5000DF0E256F0F01F70E246F0F01E00E236F2D
:10BA6000DB0E006EDFEC25F000C04AF5010EDB6A4C
:10BA7000100EF36E010EDBCFF4FFF350F45C28E2FE
:10BA8000CC0E496EDB0E4A6E010E4B6E010EDBCF03
:10BA90004CF04D6A4E6A49504C24F36E4A504D208A
:10BAA000F46E4B504E20F86EF4CFF7FFF3CFF6FF55
:10BAB0000800F550E66E010EDB50EA6AC50FE96E2C
:10BAC000060EEA22E552E750EF6E010EDB2AD0D7D0
:10BAD0000101266B010126918850010B01E02681AE
:10BAE000010126938850020B01E02683F28E0601A5
:10BAF000506997EC3DF04FECE1F00101CC0EB26FD4
:10BB0000D30EB36F010EB46F020184690601506B4E
:10BB100097EC3DF00101010EB56F8EECDBF09EEC71
:10BB2000DBF0AFEC6FF0060117810601416941C6F9
:10BB300040F60601426B138A128011881182138627
:10BB400013880A01380ED66F0A01010ED76F91ECE7
:10BB500019F094ECDFF049EC20F0010EE66EFDECFC
:10BB60003DF0E552166E200E165C02E101013889A7
:10BB7000010EE66EFDEC3DF0E552000901E0F8D75C
:10BB8000640EE66EA5ECFDF0E5521C9EF6ECC4F0EA
:10BB9000096AFC0E016E56EC3BF0001CDF6EFC0ED9
:10BBA000016EDF50006E13EC3BF0FC0E016E56ECA4
:10BBB0003BF0DF50005C06E0210EE66EA6EC14F0D0
:10BBC000E5524ED0830E096EFC0E016E56EC3BF032
:10BBD000001CDF6EFC0E016EDF50006E13EC3BF0BC
:10BBE000FC0E016E56EC3BF0096ADF50005C06E08B
:10BBF000240EE66EA6EC14F0E55232D0FD0E016E76
:10BC000056EC3BF0DB0E005C03E1210E165C02E11A
:10BC1000FBDC1ED0020E016E56EC3BF000C02AF198
:10BC2000370E016E56EC3BF000C05FF1110E016E55
:10BC300056EC3BF000C039F1120E016E56EC3BF0B1
:10BC400000C03AF10F0E016E56EC3BF000C037F128
:10BC5000E00E016E56EC3BF00050800801E28FDCF4
:10BC60000701580E626F020E636F07018B69BCEC0F
:10BC70000CF0F6ECC4F0C2EC3DF01F860001116A36
:10BC8000126A136A146A800E076E176A219A750E7B
:10BC9000E66EE66A280EE66E010EE66E81EC3BF07B
:10BCA000E552E552E552E552020E096E5A0EE66E75
:10BCB000A20EE66E000EE66E030EE66E81EC3BF021
:10BCC000E552E552E552E552030E096E2A0EE66E84
:10BCD000E66A000EE66E0A0EE66E81EC3BF0E55277
:10BCE000E552E552E552AA0EE66E300EE66E2A0ED9
:10BCF000E66E0A0EE66E81EC3BF0E552E552E55247
:10BD0000E552FE0E016E56EC3BF0096A850E005CB2
:10BD100001E059DD060EE66EF00EE66EB80EE66E38
:10BD2000070EE66E81EC3BF0E552E552E552E55236
:10BD3000040EE66EA00EE66EEA0EE66E060EE66EE7
:10BD400081EC3BF0E552E552E552E5520601EA513D
:10BD50000A0802E20601EA6B0601EC51010802E260
:10BD60000601EC6B200EE66E800EE66E640EE66E4B
:10BD7000070EE66E81EC3BF0E552E552E552E552E6
:10BD8000830E096EF90E016E56EC3BF000C071F2A5
:10BD900002017151C80803E20201C80E716FF80E6A
:10BDA000016E56EC3BF0339A6E0E005C01E1338A73
:10BDB000DF0E016E56EC3BF00101E391720E005C68
:10BDC00002E10101E3817E0E096E080EE66EE66A6D
:10BDD000B60EE66E020EE66E81EC3BF0E552E552E1
:10BDE000E552E552096A01019C51040802E2010191
:10BDF0009C6B1C0E165C10E10101368F0101368D23
:10BE00000101369136833695010EE66EFDEC3DF06C
:10BE1000E552000901E0F8D7090E165C09E11B861E
:10BE2000010EE66EFDEC3DF0E552000901E0F8D7A9
:10BE300001018051060802E20101806BCFEC04F0A1
:10BE4000E1EC0CF001018DAB06D001013C9F01013A
:10BE50003C9D01013B9F0A0E0101985D04E3010135
:10BE60009851640803E201011E0E986F010101015F
:10BE70005751200B07E0010101015751100B02E15E
:10BE80000101579BB6C201F0BDC202F0FF0E015C7A
:10BE900007E0015005E0FF0E025C02E0025008E1FD
:10BEA00002017C0EB66F0201FA0EB76F49EC4EF03C
:10BEB00001018351050802E20101836B01018451F4
:10BEC000020802E20101846B0101425104E0010118
:10BED0004251020803E20101020E426F01016D515D
:10BEE000230803E201010A0E6D6F01015F8D01015C
:10BEF000505104E0010150510D0803E20101010E0F
:10BF0000506F0601EA510A0804E20601EA6B0601D5
:10BF1000EB6B01018E9D0101578301012E6B460ED3
:10BF20000101525D04E301015251730803E2010172
:10BF3000540E526F640E01014A5D0BE301014A5138
:10BF4000496E4A6A4A3404E24950B408000E4A5421
:10BF500003E201018C0E4A6F01015551150804E3FB
:10BF6000030E0101555D03E20101150E556F040E2C
:10BF70000101475D04E301014751080803E20101A3
:10BF8000050E476F01017D51496E4A6AD8904A50AB
:10BF900004E6C80E495C000E4A5803E20101CF0EC8
:10BFA0007D6F01014D51496E4A6A4A3404E249509D
:10BFB0009608000E4A5403E201018C0E4D6F0101F8
:10BFC0004C51320803E20101280E4C6F01014B5124
:10BFD000496E4A6A4A3404E24950C808000E4A547D
:10BFE00002E201014B6B0A0E0101415D04E3010114
:10BFF00041510F0803E201010F0E416F010135515C
:10C00000500803E20101010E356F01012851280893
:10C0100003E20101280E286F550E01014E5D07E075
:10C02000680E01014E5D03E00101680E4E6FFF0EC8
:10C030000101695D03E00101695109E10101C80ED7
:10C04000696FD90E6A6FCF0E6B6F060E6C6F0101B0
:10C050007751010802E20101776B010166513C084A
:10C0600002E20101666B010167513C0802E2010135
:10C07000676B01016851280802E20101686B010148
:10C0800001018D51020B05E101013A5102E001016C
:10C090008D8301016151030802E20101616BFF0E12
:10C0A00001015F5D02E101015F6B01017151496EA8
:10C0B0004A6A4A3404E24950C808000E4A5403E26E
:10C0C0000101C80E716F01017351496E4A6A4A3409
:10C0D00004E24950C808000E4A5403E20101280E48
:10C0E000736F01017251496E4A6A4A3404E2495041
:10C0F000C808000E4A5403E201010C0E726F0101E0
:10C100007551496E4A6A4A3404E24950C808000E23
:10C110004A5403E201011E0E756F010131510208FC
:10C1200003E20101010E316F3C0E0101E76E7C1943
:10C13000E8AE02D07C3503D0E750D8807C550BE3C5
:10C14000C40E0101E76E7C19E8AE02D0E73402D0DC
:10C15000E7507C5D02E201017C6B010186510F0812
:10C1600002E20101866B01017B510F0802E201012D
:10C170007B6B01016E513C0802E201016E6B010113
:10C180006F513C0802E201016F6B0601EB511E0882
:10C1900002E20601EB6B0601ED511E0802E2060108
:10C1A000ED6B01017F51640803E201011E0E7F6FF8
:10C1B00001012951496E4A6AD8904A5004E6280E76
:10C1C000495C000E4A580BE3010129514B6E4C6A41
:10C1D0004C3404E24B504608000E4C5403E201017B
:10C1E000370E296F01018551C80802E20101856BF4
:10C1F00001018551496E4A6A4A3404E24950960861
:10C20000000E4A5403E20101960E856F0201875128
:10C2100004E002018751330803E202010D0E876F2B
:10C2200001018751780803E20101640E876F010163
:10C2300093510C0803E20101060E936F0101955121
:10C240000C0803E20101060E956F010188511E08DA
:10C2500002E20101886B01018AAF02D001018A6B01
:10C2600001018DAF02D001018D6B01018EAF03D0B2
:10C2700001010A0E8E6F010196AF03D00101600E1D
:10C28000966F1E0E0101895D04E3010189512808A2
:10C2900005E201011E0E896F01018A9101018B5196
:10C2A0000A0802E201018B6B01017A51190804E2CC
:10C2B00001017A6B01018A930101705104E00101CF
:10C2C00070511E0803E201011E0E706F01013E5104
:10C2D000010803E20101010E3E6F210EE66E27EC1C
:10C2E00014F0E552000909E00101010E3E6F010161
:10C2F000030E3F6F0101020E406F79EC5CF0318854
:10C3000005014B69C6EC0AF00101E38301012951E3
:10C31000E8240301B86F87EC21F0300E0101842579
:10C320000401F76F020E0101845D03E10401340E84
:10C33000F76FC8ECA7F004013B0EFE6F0501106B10
:10C3400010C512F510C511F50501800E156F95EC9D
:10C35000C7F0B3ECC7F0BCECC7F0000905E12D0E47
:10C36000E66EA6EC14F0E55207013C0E846F010165
:10C37000D56BD5C1D4F10701B16B4AEC75F007015B
:10C38000BE81BCEC0CF072EC1EF022EC53F043ECDE
:10C3900053F00101010138510701099F040B01E02D
:10C3A000098FB5EC20F007ECC4F01FDBF6ECC4F00D
:10C3B000E5EC11F0F3CF0EF0F4CF0FF0430E0E5C6E
:10C3C000010E0F5806E3D30ED8800E54020E0F5400
:10C3D00011E20EC049F00FC04AF0040ED8904A3264
:10C3E0004932E804FBE149C026F75A0EE66EA6EC96
:10C3F00014F0E55234EC13F0F3CF0EF0F4CF0FF05D
:10C400001F0E0E5C010E0F5806E3D30ED8800E549B
:10C41000020E0F5411E20EC049F00FC04AF0040E94
:10C42000D8904A324932E804FBE149C026F75D0E54
:10C43000E66EA6EC14F0E552550EE66E020EE66EC0
:10C44000400EE66E2DECC4F0E552E552E552020EC8
:10C45000E66E400EE66E79ECC4F0E552E552006EF1
:10C46000550E005C07E000C026F7600EE66EA6ECF5
:10C4700014F0E552E66A020EE66E400EE66E2DEC12
:10C48000C4F0E552E552E552AA0EE66E020EE66EE3
:10C49000420EE66E2DECC4F0E552E552E552020E76
:10C4A000E66E420EE66E79ECC4F0E552E552006E9F
:10C4B000AA0E005C07E000C026F7630EE66EA6EC4D
:10C4C00014F0E552E66A020EE66E420EE66E2DECC0
:10C4D000C4F0E552E552E5520201440E976F120E88
:10C4E000E66E420EE66E79ECC4F0E552E552046E5B
:10C4F000026E0450800B01E0010E496E0450400BA7
:10C5000001E0010E495C23E1047C0450E66E120E4A
:10C51000E66E420EE66E2DECC4F0E552E552E552B1
:10C52000120EE66E420EE66E79ECC4F0E552E5526C
:10C53000046E0450800B01E0010E496E0450400B64
:10C5400001E0010E495C03E10201450E976F0250C4
:10C55000E66E120EE66E420EE66E2DECC4F0E5526B
:10C56000E552E5520101835116E07DECE4F000094B
:10C570000AE00AECE3F069ECE3F001018351010801
:10C5800001E2338C08D00701050E266F1E0EE66E01
:10C59000A6EC14F0E5527DECBDF02B96229601013D
:10C5A0003A510101941101E17CD0150EE66E020EA4
:10C5B000E66E440EE66E2DECC4F0E552E552E5520F
:10C5C0002A0EE66E020EE66E460EE66E2DECC4F006
:10C5D000E552E552E552020EE66E440EE66E79EC47
:10C5E000C4F0E552E552150802E1000E01D0010E3B
:10C5F000006E005014E001013A5108E000C026F737
:10C60000660EE66EA6EC14F0E55208D00701030EA4
:10C61000266F180EE66EA6EC14F0E55242D001012A
:10C620003A5118E0020EE66E460EE66E79ECC4F062
:10C63000E552E5522A0802E1000E01D0010E006E1B
:10C64000005008E000C026F7690EE66EA6EC14F074
:10C65000E55227D0120EE66E440EE66E79ECC4F079
:10C66000E552E552006EC00E001601013A510CE091
:10C67000005008E000C026F7840EE66EA6EC14F029
:10C68000E55201D02B860DD0C00E005C09E00701F9
:10C69000040E266F180EE66EA6EC14F0E55201D0DB
:10C6A0002286B7EC5CF01B92010194511FE0370E1B
:10C6B000E66E020EE66E480EE66E2DECC4F0E55214
:10C6C000E552E552020EE66E480EE66E79ECC4F0D5
:10C6D000E552E552370809E00701010E266F180EF2
:10C6E000E66EA6EC14F0E55201D01B822580E668C8
:10C6F0007DEC36F0E55239C1E6FF42ECC3F0E5527D
:10C700000101B581219401013BBB06D00601509582
:10C710000601508797EC3DF00101D45104E0030E6F
:10C720000101D45D04E10A01D46B149C04D00A0118
:10C73000020ED46F148C93D901012ABD0CD0D6EC13
:10C74000C8F0C6C269F1C7C26AF1C8C26BF1C9C2FA
:10C750006CF101012A8DABEC2EF00201320E246F38
:10C760000101100EB96F0501010E176F0901020ECC
:10C77000E56F0201582B0201320E226FA8EC96F0F1
:10C780008CEC04F00201CF5108080AE21AEC14F014
:10C79000CFC226F72A0EE66EA6EC14F0E5521B86F1
:10C7A0000D0EE66E21EC15F0E552870B006E005081
:10C7B00008E000C026F73C0EE66EA6EC14F0E55249
:10C7C00014D076EC20F03B0E0E5C000E0F5806E302
:10C7D000E60ED8800E54030E0F5407E20EC026F763
:10C7E000570EE66EA6EC14F0E552030EE15C02E291
:10C7F000E16AE552E16EE552E7CFD9FF1200440E3F
:10C800000101B95D03E3B951490801E2000C010CD3
:10C8100001013B7B279D256B1DD8238A25820101C1
:10C820003BBB13D009014F0EE66F460EE76F0601C2
:10C8300050A707D00901560EE66F420EE76F0101BF
:10C8400036890601436B43C642F601013BBB0480B7
:10C85000D1EF09F006015097509501013BBB07D07D
:10C8600021B403D006015085120006015087120042
:10C870000A01D65177EFDBF0D4C100F0005003E09D
:10C88000030E005C33E100500EE10101D07D09018F
:10C89000430EE66F0101D0AD02D0BEECD1F0010134
:10C8A000D0AD20D010D0AEECCDF00FE00101D075AE
:10C8B0000901440EE66F0101D0A502D0BEECD1F013
:10C8C0000101D0A50FD004800DD00101CF75090161
:10C8D000440EE66F0101CFA502D0BEECD1F00101FC
:10C8E000CFB50480D1EC09F025EFD4F0000403E0CB
:10C8F000020E005C16E103EC14F0000402E1020EEB
:10C9000001D0010E006E09014C0EE66F020E005CB4
:10C9100003E10480550EE66FD1EC09F000C0D4F1BC
:10C9200066D812000101325103E1A4ECCAF002E022
:10C93000000E01D0010E1492E8B01482A4ECCAF0EB
:10C9400003E137ECD5F00CE1A4ECCAF007E00AEC07
:10C95000CBF004E101013B51800B02E1000E01D05C
:10C96000010E1490E8B014801200A4ECCAF00AE0A2
:10C9700010ECD3F007E1E4ECD2F004E000ECD6F0E8
:10C9800001E1000C010C0CECD3F003E0010181513A
:10C9900012000101785112000CECD3F003E0010108
:10C9A00082511200010179511200E7ECC9F00CEC40
:10C9B000D3F005E0FE0EDB500101816F04D0FE0EC6
:10C9C000DB500101786FE3EFC9F0E7ECC9F00CEC44
:10C9D000D3F005E0FE0EDB500101826F04D0FE0EA5
:10C9E000DB500101796FE3EFC9F0AAEFD7F0219096
:10C9F0002792D4C100F00050800802E2050E006EBC
:10CA0000060E005C01E3006A000402E10101CF911F
:10CA1000020E005C02E10101CF8100C0D4F1248A42
:10CA200020BE03D0A4ECD4F002D0F0EC39F080EFBB
:10CA300025F05FECD5F0030EDF6E01014951496E20
:10CA40004A6AB00E3D6E040E3E6E69ECCAF03D506F
:10CA5000D880DF540201506FE552E3EFC9F05FEC7C
:10CA6000D5F026B00ED0320EDF6E080E0101495D02
:10CA700002E2080E496FDF50D880495502E2DFCF4D
:10CA800049F1D7DFE552E3EFC9F050C2B0F122AE71
:10CA900034D0006A01013D510C0803E3070E3D5DEF
:10CAA00002E20C0E3D6F070E3D5D4D6E4E6A0201B7
:10CAB00050518FECCBF0006E76ECDAF00101B05102
:10CAC0004B6E4C6AFF0ED8804B56000E4C564A50A7
:10CAD0004C18E8AE02D04C3404D04B50495C4C505A
:10CAE0004A580BE20050D880B05507E223A003D08B
:10CAF0000050B02702D00050B05FD0ECD0F008E179
:10CB000002012D510601EA1106E02750400B03E116
:10CB10001D92BBEC3CF01200050EB6ECCEF0580EA8
:10CB200025EFCFF0F9DF258E1200180E9FECCAF02A
:10CB3000010136AD03D0580E25EFCFF0258E12003F
:10CB4000E7ECC9F0050EE1261FA20FD0BFC1DFFF41
:10CB5000010EC0C1DBFF020EC1C1DBFF030EC2C16B
:10CB6000DBFF040EC3C1DBFF0ED0BAC1DFFF010E35
:10CB7000BBC1DBFF020EBCC1DBFF030EBDC1DBFF8F
:10CB8000040EBEC1DBFF00ECD6F022E0E551100B35
:10CB90001FE13851010B03E19651040B06E0320E00
:10CBA000DF5C62E3DF5033085FE32E50800B06E06A
:10CBB000320EDF5C59E3DF50350856E32E50800B10
:10CBC0003BE12F0EDF5C50E3DF50380835E24CD0FC
:10CBD000DF504AE0DF0404E1460E65ECCCF044E3AC
:10CBE000DF50180806E21C0EDF5C03E29651010BD1
:10CBF00023E1E5BD07D0DF50180815E21C0EDF5C0D
:10CC000012E232D0190EDF5C2FE01A0EDF5C04E175
:10CC1000010EDB505F0828E31B0EDF5C04E1290EE8
:10CC200065ECCCF021E32B50100B06E12E50800B6D
:10CC300003E02B510A0802E2F36A1BD0630EE66E92
:10CC4000020EE66ED9CFE6FFDACFE6FF5DECCDF05F
:10CC50000BE1D9CFE6FFDACFE6FF5E0EE66E020EFD
:10CC6000E66E5DECCDF004E060DF010EF36E01D006
:10CC7000F36AF46A050EE15C02E2E16AE552E16EF4
:10CC8000E3EFC9F065C301F022A802D078C301F038
:10CC90000E0E015C01E2010C100E015C01E2020CBF
:10CCA000120E015C01E2030C140E015C01E2040CA3
:10CCB000160E015C01E2050C1B0E015C01E2060C84
:10CCC000220E015C01E2070C080C85ECD5F01CEC8F
:10CCD000DAF0F00801E2006A0050E3EFC9F0E7EC97
:10CCE000C9F095ECD5F0F1DFE552FE0EDB509B0864
:10CCF00005E1030E28ECD6F01BECCEF0FFECD6F0ED
:10CD000004E6DC0E495C000E4A580AE24D0E496EFC
:10CD1000D50E4A6E010E4B6E005070ECD5F001D06E
:10CD2000D20E0E6E0F6AFFECD6F004E6AA0E495C36
:10CD3000000E4A580CE2A30E496ED40E4A6E010E44
:10CD40004B6E005070ECD5F00101D86F02D001019C
:10CD5000D869D96BE3EFC9F05FECD5F0049034B833
:10CD60000480B30E016E0101E6A539D01BB62AD0AE
:10CD7000B30E3FECD7F0D8C1D7F26EEC20F0026EC4
:10CD8000300EDF6E020403E0020E025C02E1380E98
:10CD9000DF6EDF500201D880D75509E26AEC0EF051
:10CDA000530EE66EE30EE66E010E12ECCAF0DF5093
:10CDB000496E4A6A0101D851495CD9514A5802E288
:10CDC0004851D6E1070114B108D0148177ECD5F0B1
:10CDD0007D0E976E080E87ECD8F09B0E016E015009
:10CDE0003FECD7F085ECCBF012E00E500101D66F8E
:10CDF000D76BB30E3FECD7F00E5006ECD7F0010125
:10CE0000D6274A50D723D6C10EF0D7C10FF0010163
:10CE1000E6A502D0D86BD96BD8C161F3D9C162F352
:10CE200034B80AD113A64DD00B50016E2250100B0E
:10CE300003E13450800B02E002D913D085ECCBF033
:10CE400010E00701C1514D6E4E6A0B508FECCBF0D4
:10CE5000016E2050800B05E00901EC5102E0ECC9A5
:10CE600001F0050E0124496E0A0EE1ECCAF0016ED4
:10CE7000015005E12250400B02E0010E016EA4ECCE
:10CE8000CAF003E03450400B05E001C0A3F70201F3
:10CE90000A0E08D00701A351015C05E301C0A3F706
:10CEA00002010C0E2A6FEEDE0701A46F2B50100B4F
:10CEB00003E1040E0B5C01E2A46B34ECD0F040EC17
:10CEC000CEF0B2ECCDF00480005009E03450400BBD
:10CED00006E1030E005C04E1020E0A5C01E104902D
:10CEE000070E016E04A004D0090E97ECCBF0016E82
:10CEF0000F0E01140201736F070E731701380F0B29
:10CF0000016E04A0016A13A408D0020EE66E73C27B
:10CF1000E6FF0150E66E40ECCEF052C100F0010198
:10CF2000E6A502D04AC100F076ECDAF0E2ECCBF0F4
:10CF3000B7ECD6F018ECD7F0640E71ECD9F00E50C7
:10CF40000B6EB2ECCDF0040E005C0BE0000409E0C7
:10CF5000020E005C06E0030E005C0AE1020E0A5CB1
:10CF600007E00201AF51D8800B5402E20BC0AFF2D0
:10CF70000101E6A507D00301636B646B676B686B07
:10CF8000656B5AD0B70E3FECD7F0D8C163F3D9C167
:10CF900064F303016151635D6251645906E3010E5C
:10CFA0006325616F000E6421626F61516325676FB5
:10CFB00062516421686F67516725496E6851682125
:10CFC0004A6E67C34BF068C34CF0030ED8904B36E3
:10CFD0004C36E804FBE149504B240301676F4A508B
:10CFE0004C20686F6351615D496E625164554A6EB1
:10CFF000B7ECD6F067C33DF068C33EF000ECFEF03E
:10D000003DC067F33EC068F367C365F367C349F08B
:10D0100068C34AF04B6A4C6A4C34000E4C1809E65F
:10D02000D880FF0E4954000E4A54000E4B54000E97
:10D030004C5402E203016569E552E3EFC9F048C1CF
:10D0400001F02B50100B05E185ECCBF002E0D5C2CE
:10D0500001F01200B2ECCDF000500DE03450400B66
:10D060000AE1050E005C07E0030E005C03E1020E1E
:10D070000A5C01E0000C010C0482ECDF000901E015
:10D080000492348604A23496349866DE34B81200D2
:10D09000B2ECCDF004980496030E005C01E1048626
:10D0A000000403E0020E005C01E104882250400B02
:10D0B00001E1F8D02250100B01E0F4D03450800B85
:10D0C00001E0F0D03350080B01E1ECD002011D511A
:10D0D00001E0E8D01950010B01E1E4D0048204948E
:10D0E000B9DF000901E00492040E005C01E1048450
:10D0F000A6DF0150F2ECD8F0026E8CECCAF001C051
:10D100003EF05AECFEF03EC007F1020E0101075D51
:10D1100002E2020E076F07510A0802E20A0E076FC9
:10D120000450040B07E00201735104E1D89001326E
:10D13000D890013204902050800B33E00901ED516A
:10D1400030E085ECCBF02DE00901EE51020829E238
:10D15000030E006EEE51190802E2020E006EEE514F
:10D16000280802E2010E006EEDA104D00050A9ECE7
:10D17000D2F00480020E0901ED150FE076ECDAF032
:10D1800002010051495C01514A5807E2005006EC87
:10D19000D7F0005F4A50015B0480040E0901ED17CF
:10D1A00072D001500B5C42E20201880E005D130E4A
:10D1B000015969E203016C0E635D000E645963E27C
:10D1C00004B20AD00B50015C0E6E0F6A0E500201C1
:10D1D00000270F50012356D002011E5154E10A0EC0
:10D1E0001E6F0150AF5D20E2AF5103E173510108A2
:10D1F0001BE204A802D0020E1E6F0450080B0FE0C1
:10D20000030E0A5C03E07351010809E201010751B2
:10D21000A9ECD2F01F5107E01E911E4304D0020E6C
:10D220000027000E01230480AF6B2DD00150D88061
:10D230000B5429E2010E036E04A208D007C103F0CB
:10D2400004A804D0030E0302F3CF03F003500E6EC4
:10D250000F6A0450020B06E00450080B09E00201BB
:10D260001F5106E001500B5C1FECDBF018ECD7F00F
:10D27000020100510E5C01510F5805E20E50005F93
:10D280000F50015B048004A00DD00201025100196F
:10D2900002E10351011906E0E7EC0BF000C202F2D3
:10D2A00001C203F20201205102E00F0E206F1200B2
:10D2B000F7ECDAF01750100B0CE0200E155C4CE088
:10D2C000210E155C49E0150E155C03E1E4ECD2F08B
:10D2D00043E01750010B09E0150E155C3DE0220EEE
:10D2E000155C3AE01D0E155C37E00A0E155C03E193
:10D2F000BDECCAF031E01950200B12E102011951C6
:10D300000FE1230E155C28E00B0E155C25E0090EDD
:10D31000155C22E0090E155C1FE0220E155C1CE076
:10D320003BECD5F004E0B1EC96F0000915E11D0EE0
:10D33000155C07E11750100B04E019EC19F0000917
:10D340000BE12050800B06E10201685103E03250EE
:10D35000200B02E0000E01D0010EDF6EDF50E5521F
:10D36000E3EFC9F00101E6A509D0070115817EECC4
:10D37000D5F00701149F149377ECD5F0030EE66EF9
:10D38000CAEC16F0E5528A8607010B91BCECC4F09A
:10D3900037EC19F0A4ECCAF003E03450400B11E074
:10D3A00063EC0BF000090DE0DAEC08F0C3EC16F0CA
:10D3B0006F0E52ECCAF0C80EA9ECCDF0DDEC08F00F
:10D3C00002D0C3EC16F00601509197EF3DF05BC21E
:10D3D00048F15CC200F25DC201F2E7EC0BF0C3EC75
:10D3E00023F001ECD2F0239612000101B05103E1C9
:10D3F0002B820850076E2050010B12E0A4ECCAF0FB
:10D400000FE11750800B03E05DECD2F006E02050F6
:10D41000040B06E13FECCDF003E06AD9BEEC71F0FD
:10D4200012000101050EAF6F2050010B04E01950EE
:10D43000020B01E0AF6B1200B2ECD6F001013951E2
:10D440002BE105C2DFFF50ECBEF0DF500201055DAD
:10D4500023E0010E69C3DBFF020E6AC3DBFF030E8C
:10D460006BC3DBFF010EE66EF5ECBEF0E552010E7C
:10D47000DB500301695D08E1020EDB506A5D04E1E7
:10D48000030EDB506B5D08E09FECBDF0F6ECC4F0E2
:10D490001C820101960EAC6F040EE15C02E2E16AAF
:10D4A000E552E16EE3EFC9F00201185107E0186B95
:10D4B0002AECCFF00201D05101E11194A4ECCAF0A2
:10D4C00009E12050010B06E137ECD5F003E12050D3
:10D4D000800B0FE0D0ECD0F00CE11E50400B09E1C6
:10D4E00081ECCCF004E1020E0101B95D02E0228C76
:10D4F000D18022BC06D0E66AE66A740E0DECCAF052
:10D5000017D0E4ECD2F012E13350080B0FE000C268
:10D5100049F001C24AF0030E0F0B03E094ECD0F087
:10D52000FDE149500201005F4A50015BE7EC0BF05E
:10D5300002010A0E1E6FAF6B20AE1C84C80E1F6F57
:10D54000BCEC16F0780E006E0050A9ECCDF074EC37
:10D5500018F00201226B0101E6A509D00701148F22
:10D5600001012AA102D00701148377ECD5F08A9635
:10D57000320EA9ECCDF034ECCBF014E12B50080BBB
:10D5800011E02250100B0EE101013A050BE0A4EC72
:10D59000CAF007E12050800B04E102011E0E156F56
:10D5A00001D04ADF2050800B0EE12050010B0BE12F
:10D5B000A4ECCAF008E03450400B05E102012D5103
:10D5C00002E0050110511DAC02D01EEC0CF0208CC5
:10D5D0003182D5CA85F2B2ECCDF0360E026E380E2D
:10D5E000036EBAC17DF277ECD9F03EC07EF27CECDE
:10D5F0002FF0BAC17BF277ECD9F03EC07CF21FA2CB
:10D600000AD0BFC17BF28CECCAF0C0C13EF05AEC2C
:10D61000FEF03EC07CF222AC26D007010B8F0B81BE
:10D62000BCECC4F064ECD2F008E15751010B05E00A
:10D630000701088F089DC9ECD5F0030E01012B5D91
:10D6400004E102017B51070808E3040E01012B5D90
:10D650000AE10A0E02017B5D06E20701088F0897C6
:10D660000895C9ECD5F02F8E4AEC32F00201FA0E83
:10D67000236F238A2582319222AC02D0BBECD4F0F6
:10D680006FEC39F021AE12D0219E1AEC0BF080EC39
:10D69000D7F099ECD5F00AE099ECD5F007E099ECD9
:10D6A000D5F004E00DEC0BF078EF6BF002011451B3
:10D6B00009E00101E551080B05E1140E93ECCAF0F5
:10D6C0000101E58712005FECD5F005012307245125
:10D6D000EA6A270FE96E050EEA22EFCFDFFF242B5F
:10D6E00024511F0801E2246BDF50E552E3EFC9F03B
:10D6F000F1EC21F00201196B19C255F210ECD2F0D5
:10D7000007E0200E01011C5D03E0200E32ECCDF09D
:10D710000101B06B006A7CEF75F04B0E026E140EC7
:10D720000301655D07E364ECD2F01EE11E0E030108
:10D73000655D1AE2100E01012B5D16E22B50100BF5
:10D7400003E0640E485D11E02B50100B0DE1280E34
:10D75000485D0BE03C0E485D08E0020E395D04E1D7
:10D760005A0E0224485D01E0000C010CF7ECDAF0DF
:10D770001B50080B0AE181ECCCF009E13C0E0101E1
:10D78000B95D03E0430EB95D02E1000E36D0010140
:10D79000815102E0825104E1480E20ECCBF0DF2AF7
:10D7A0000101785102E0795104E14B0E20ECCBF0FD
:10D7B000DF2AB3DF00091CE1C9EC35F0000906E0FF
:10D7C0003F0E20ECCBF0E7ECD0F0DF2ADEEC35F0BA
:10D7D000000907E0420E20ECCBF00201916B926B46
:10D7E000DF2A0701C05104E1450E20ECCBF0DF2A0F
:10D7F000DF5002E07DDF2094DF50E552E3EFC9F017
:10D8000073ECCEF002E27B511200865112005FEC05
:10D81000D5F00750DF6E27AA03D002011E0E216F3C
:10D82000050110510201191103E13751381109E0C6
:10D830001D50040B0FE01D50080B0CE01E50010B97
:10D8400009E01750800B08E02750200B05E1050187
:10D85000105102E04DDFB4D2075049E127BA04D09D
:10D8600018ECCFF0020E87D081DF000901E0A8D2CA
:10D870000201245101E0A4D220B002D015DE0AD06A
:10D880002D5108E00501105105E1E0ECD2F002E174
:10D8900018ECCFF0E4ECD2F019E1020189A514D024
:10D8A000330E875D0EE10101E451800B03E12D5041
:10D8B000080B0CE02D96A7EC04F00201330E3A6F32
:10D8C00005D0A7EC04F002D0ABEC04F099DF050D15
:10D8D000F3CFAFF10101E6A512D10A0EAF5D02E26E
:10D8E0000A0EAF6F070115917EECD5F008D1070441
:10D8F00020E10101AF5101E05FD21F9C34ECCBF07D
:10D9000002E01F8C05D0E0ECD2F002E13EEC0BF01F
:10D910000101280EAF6FE6A505D007011585158317
:10D920007EECD5F020AE03D00101050EB06F072AC2
:10D9300017D0020E075C16E10201155102E01E0E1F
:10D94000156F27BA06D00101B05101E035D2085059
:10D950005DD10101AF5102E13CEC68F048EC0BF005
:10D9600044DD2AD2030E075C3CE127BA06D0006AE8
:10D970007CEC75F0070E076E23D22BA218D05BC18A
:10D98000AFF10101B05105E03BDF050DF35001019E
:10D99000AF272B922050010B04E01950020B01E03D
:10D9A000AF6B02012D5103E0006A7CEC75F00101C0
:10D9B000AF5106E0A4ECCAF00FE03450400B0CE18C
:10D9C0001F50400B05E102012D5102E143EC0BF029
:10D9D0000101280EAF6F19D126B8EED13CEC68F0EA
:10D9E000EBD1050E075C62E10101AF5101E0E4D12A
:10D9F000072A269820B0E0D11C0E016E01DFE82432
:10DA00000124006E0201765107E00050765D04E2C9
:10DA1000090E076E2688D0D1318207010B9FBCEC1E
:10DA2000C4F064ECD2F008E15751010B05E00701A6
:10DA3000089F088DC9ECD5F0030E01012B5D04E1B0
:10DA400002017B51070808E3040E01012B5D11E17F
:10DA50000A0E02017B5D0DE20701089F030E010122
:10DA60002B5D03E10701088502D007010887C9EC97
:10DA7000D5F00101E6A508D00701159515937EECB8
:10DA8000D5F001010A0EAF6F209C85C2D5FAA7EC34
:10DA9000C4F083ECD4F0A4ECCAF003E03450400BA3
:10DAA00003E00101050EAF6F319286D1060E075CCF
:10DAB00028E10101AF5101E07FD120B01ED02650F6
:10DAC000100B0DE1325109E0A4ECCAF003E0345030
:10DAD000400B03E037ECD5F002E144DC0ED032C15C
:10DAE00022F226A80AD08CDE33ECD8F0006E00506B
:10DAF0000201225D02E200C022F20201566B072AF7
:10DB00005BD1070E075C24E10101B0510FE117AEB4
:10DB10000BD05DECD2F003E06EEC97F005D093EC07
:10DB20000BF0000901E0179E0850076E02012D510D
:10DB300001E042D12A5106E03450400B03E134ECBD
:10DB4000D0F003D0E66AE66AE66AD5EC28F047D062
:10DB5000080E075C4BE10101B05106E01D50040BBB
:10DB600003E01D50080B02E10850076E02012D5121
:10DB700001E122D13CEC68F048EC0BF002012E519F
:10DB800001E01AD182EC0EF0000901E115D1050186
:10DB9000020E266F235111E096DD006E020E0A5C24
:10DBA00002E1005010D0016A0501235102E08BDD33
:10DBB000016E0050B6ECCDF00ED0105114E1020E03
:10DBC0000A5C07E1030EE66E150EE66E69EC16F0D0
:10DBD00007D0E66AE66A160EE66E6FEC16F0E552BE
:10DBE000E552E552E9D002012D6BE6D0090E075C43
:10DBF00028E1020176417F0B76250101D880B155DD
:10DC000007E20201766B76C2B1F1050E076ED4D041
:10DC10001EB0D2D0010EB16F320EAF6F010E076E83
:10DC2000A4ECCAF003E002012D5108E0E0ECD2F0D0
:10DC300005E12750200B02E118ECCFF00B0E086E27
:10DC4000BBD00A0E075C06E121BAA9D0179E0B0EC5
:10DC5000076EA7D00B0E075C01E0A6D01750800B13
:10DC600039E12050010B06E02050040B03E13FECAA
:10DC7000CDF030E1A4ECCAF003E03450400B0CE0EE
:10DC80002050800B09E11E50010B06E01D50040BD3
:10DC900003E01D50080B1EE1A4ECCAF00CE0345068
:10DCA000400B09E12050040B06E13FECCDF003E00E
:10DCB0000FECD1F00FE02050800B09E01D50040B59
:10DCC00009E01D50080B06E03FECCDF003E034EC1A
:10DCD000CBF05BE017AE18D01950800B07E00A0EAE
:10DCE000155C04E061EC2DF000096AD05DECD2F027
:10DCF00005E06EEC97F0000907E162D093EC0BF0C1
:10DD0000000902E0179E5CD0A4ECCAF023E0345076
:10DD1000400B20E10AECCBF01DE119AA06D00DEC76
:10DD20000BF0B6EC08F0B7EC1DF0D0ECD0F00AE048
:10DD30001950400B07E0249223BC24820DEC0BF019
:10DD4000FBECD0F00101885105E088C1E6FFBFEC93
:10DD500021F0E552B1C176F20101B15102E0010EAC
:10DD6000B16F26A802D03CEC68F00701A16B030E4E
:10DD7000076E800E086E2050800B03E11750800B59
:10DD800008E020940C0E086E04D022A802D0BCEC4F
:10DD9000BFF00101AF5105E12650100B02E13CEC50
:10DDA00068F048EC0BF008D00C0E075C05E121BAD6
:10DDB00003D01EEC99F007D8DF50075C01E01C8C03
:10DDC000E552E3EFC9F020AEABD01D50040BFDE0EF
:10DDD0001D50080BFAE02A840101B59B238AB599EE
:10DDE00025829D510BE01FA203D09DC1D5F102D029
:10DDF0009DC1D4F17CEC2FF0F7EC64F02250100BB5
:10DE000003E13450800B04E0E7EC69F0349E63D00A
:10DE100084DC000950E085ECCBF04DE15BECD4F004
:10DE200000C20EF001C20FF00EC04DF00FC04EF058
:10DE3000A9ECCBF03AECD1F08CECCAF00BC23EF07E
:10DE40006EECD8F0006E00505BECCAF0C40E406E71
:10DE5000160E416E020E426E436A31ECD9F000504C
:10DE60005BECCAF048C149F0B3ECD5F02FECFDF003
:10DE70003EC0EDFF3DC0EDFF3CC0EDFF3BC0EFFFFE
:10DE8000070130513111321133110CE0DC0E305DDD
:10DE9000000E3159000E3259000E335903E230C7DB
:10DEA00000F007D030C726F74E0E20ECCBF0DC0E8A
:10DEB000006E13EC3BF018A804D0E7EC69F018985A
:10DEC0000AD00901EC5107E085ECCBF004E00BC06F
:10DED000D5F20901ED6B209E33A403D0F0EC39F0AC
:10DEE00005D0010EE66E7FEC39F0E5522298A7ECE2
:10DEF000CCF080EC25F0010136BF04D0050EC1EC5A
:10DF0000D6F00ED036AD0CD0E385E783E795E797E2
:10DF10000601FB29FC6F65C3E6FF45EC0AF0E552FC
:10DF2000800E076E12002F50100B04E00101E85123
:10DF3000080B13E00701555110E10101B551200B09
:10DF40000CE13B51200B0AE081ECCCF007E0A95139
:10DF500005E10101E851080B01E1000C010C070E7D
:10DF6000E66EE66A200EE66E440EE66E060EE66E7D
:10DF7000E6ECFAF0050EE15E120045C644F646C630
:10DF800045F647C646F648C647F649C648F64AC665
:10DF900049F6120049C64AF648C649F647C648F649
:10DFA00046C647F645C646F644C645F60601200E67
:10DFB000446F1200E7ECC9F031AA02D04BECD3F069
:10DFC0000101E551020B0CE0280E0901BB5D08E2DE
:10DFD000BB51BB2BEA6A930FE96E090E29ECD8F00E
:10DFE0000101E851200B0CE0280E0901E45D08E274
:10DFF000E451E42BEA6ABC0FE96E090E29ECD8F073
:10E00000E3EFC9F0E7ECC9F00101E8B704D095EC03
:10E01000D5F003D8E552E3EFC9F063ECD5F0010E7B
:10E02000DB6A1A50010B0AE0800E6DECCAF004E2C4
:10E03000FE0EDB50200802E11A905CD09EDFFE0E3F
:10E04000DBCF4AF6DB50800804E0850E6DECCAF0A9
:10E0500003E30601200E21D0FE0EDB50300803E161
:10E060000601630E1AD02950200B1CE02850080B23
:10E0700019E1DF6A150EDF5C15E244ECD9F00FE11F
:10E08000DE52010EDD6EDF2A6BECCDF006014A6F29
:10E0900074DFDF2A6BECCDF006014A6F03D0030E6C
:10E0A000DF26E8D781ECCCF012E0010EDB5004E073
:10E0B00049C6E6FF7FDFE5524AC600F0630E005C0A
:10E0C00002E1300E006E0050E66E74DFE5522BDF89
:10E0D000000910E037ECCFF044C616F145C617F141
:10E0E00046C618F147C619F148C61AF149C61BF1D0
:10E0F0004AC61CF1020EE15C02E2E16AE552E16E01
:10E10000E3EFC9F05FECD5F00750DF6E2392100EFD
:10E11000075C13E11C0E076E02015151010B03E174
:10E120001D50040B02E1110E92D05151040B27E156
:10E130001D50080B01E0B3D022D0110E075C09E19D
:10E140002380228E0201080E516F2382076A120E6D
:10E15000A5D0120E075C06E123902382030E076E02
:10E16000130E9CD0130E075C0CE11C0E076E02010F
:10E170005151040B04E11D50080B01E090D0140E26
:10E1800066D0140E075C10E12380228E180E076EF5
:10E190001D50040B01E083D01D50080B01E07FD01F
:10E1A0002382076A150E7AD0150E075C0CE1010177
:10E1B0002AAF03D00201020E516F229E2382020E6B
:10E1C000076E160E6BD0160E075C05E12382020E59
:10E1D000076E170E63D0180E075C07E10201020EEE
:10E1E000516F2382076A190E59D0190E075C06E198
:10E1F000229E2382020E076E1A0E50D01A0E075C62
:10E2000005E12382020E076E1B0E48D0170E075C35
:10E2100008E101012ABF03D00201020E516F1B0E5B
:10E2200016D01B0E075C05E12390228E2382030E7D
:10E2300033D01C0E075C33E12390800E076E020181
:10E240005151010B03E11D50040B03E1110E076E48
:10E2500026D034AC0BD06EEC20F0010802E1520E57
:10E2600001D0500E52ECCAF0349C19D01750800BDC
:10E2700016E1D0ECD0F004E0090E0201535D0AE390
:10E280000601EA5104E0080E0201535D03E30201B6
:10E290002D5105E02382080E076E100E086E23A292
:10E2A00002D045EC65F0DF50075C01E01C8CE552C4
:10E2B000E3EFC9F01C9612000201566BE66AE66AAB
:10E2C000E66A40ECCEF002012A6B0701A36B0B6AF1
:10E2D00020B003D0208054EC6AF012005FECD5F03F
:10E2E0000201050E2D6F280E2E6FE6DF020E0A5C6E
:10E2F00005E189ECD1F0140E0DECCAF00501040E15
:10E30000266FE552E3EFC9F0348C0101D051400B88
:10E3100002E1530E01D0510E52EFCAF00101E35158
:10E32000020B18E03C51800B15E12050010B12E16B
:10E330002550040B0FE12450020B0CE1E3932F88CE
:10E34000670EE66EF20EE66E010E12ECCAF00101E7
:10E35000AA0EAC6F120037ECD5F004E12050010B8F
:10E3600001E1000C010C01015651800B05E0020E89
:10E37000005C03E0000401E0000C010C5FECD5F050
:10E3800010ECD3F005E089ECD1F0140E0DECCAF0DE
:10E39000209020940701A16B55ECCEF0E552E3EFFD
:10E3A000C9F075ECD8F0800E491843E14A5041E1BC
:10E3B0000101E39B199ED190FF0E05014B5D04E026
:10E3C0004BC507F04B6912000101E5A503D0E595A7
:10E3D00044EC19F00101E551080B08E02050400B16
:10E3E00005E1120E93ECCAF00101E59734AC0AD0B6
:10E3F0006EEC20F0010802E1520E01D0500E52ECFA
:10E40000CAF0349C20B013D010ECD3F002E0006AC4
:10E4100073DB2196020168510AE13250010B07E1DA
:10E420002C50800B04E12C50400B01E11F86072A81
:10E43000120084ECD1F001E00FD24A5001E00CD27E
:10E4400020A0229CE5EC14F0FF0801E005D120504B
:10E45000200B01E101D11850800B01E0FDD0020139
:10E46000766B76C2B1F11992B2ECCDF0349C1C906F
:10E470001E50010B06E01D50040B03E01D50080B5D
:10E480000DE100500BE01F50020B08E06CDF0009AB
:10E4900005E0258E1F0E9FECCAF0DED01E50010B4A
:10E4A00018E1005006E01F50020B13E15CDF000989
:10E4B00010E00101010EB16F1982076A0B0E086EA0
:10E4C000005003E148DF000901E01C8000502CE10E
:10E4D0002DD01D50040B03E01D50080B29E1005006
:10E4E0000CE010ECD3F009E11F50020B21E10AEC23
:10E4F000CBF003E138DF00091BE01DB402D0110EA0
:10E5000005D01DB604D00201516B140E076E0050E9
:10E5100003E121DF000901E01C80005007E03AEC34
:10E52000CCF002E1DBDE98D0EFDE96D0F7DE94D0BF
:10E53000050110511EE027AA12D0005003E00AEC9A
:10E54000CBF010E0005003E106DF000901E01C8081
:10E55000005001E1E3DE0AECCBF001E0BFDE1E0E6D
:10E56000076E7AD0258E8A0EB6ECCEF0D4EC21F070
:10E5700073D020AE05D0076A0A0E086E1C806CD0DE
:10E58000005051E03FECCDF006E02050040B03E1D9
:10E590001E50020B48E00201195114E01E50020BFC
:10E5A00007E1E0EC08F000090DE13FECCDF00AE1F5
:10E5B0000201376B386B196B19C255F20DEC0BF079
:10E5C0008CEC65F034ECCBF00AE03FECCDF0FDE0F4
:10E5D0000FECD1F0FAE120941E928CEF04F01C8035
:10E5E000D0ECD0F013E01950400B10E01950040BA0
:10E5F0000DE020A40AD01994050EE66ED00EE66E4A
:10E60000E80E0C240DECCAF001D01C901CA024D004
:10E61000000E02012A6F0701A36F0B6E1E92076A9C
:10E620000B0E086E19D0005017E12050010B14E1B9
:10E630003FECCDF003E02050040B0EE00101E3932A
:10E640008CEC04F034ECCBF005E03FECCDF0FDE0D9
:10E65000209412001C8030DE2050200B04E1B0EC2E
:10E660000BF0000903E1020134514DE081ECCCF0E4
:10E670004AE00501106B20902094810E076EFBECA0
:10E6800004F0000906E14B0EE66EE30EE66E010EA5
:10E690000DD03FECCDF002E11B0E12D00FECD1F00B
:10E6A0000AE0430EE66EE30EE66E010E37ECDAF09A
:10E6B000E552E55208D0B0EC0BF0000905E01A0E67
:10E6C000E66EFFEC26F0E552B0EC0BF0000919E025
:10E6D000ACC134F2FBEC04F0000905E10101806BF0
:10E6E000CFEC04F00ED00FECD1F00BE01BECD5F02A
:10E6F00003E001013C9D02D001013B9F25EC19F094
:10E700001490D8EC07F084ECD1F001E14A5042E0DB
:10E710008CEC04F00201D95102E0DDEC08F00201BA
:10E72000D85102E09EEC48F027AA28D094ECE2F001
:10E7300002012A6B2FAA02D006EC4FF030A402D0BF
:10E74000B4EC51F030AC02D033EC50F024A002D045
:10E750005FEC4FF032A002D0B4EC4FF023AE02D009
:10E7600099EC4EF01FA802D032EC10F02C50800B28
:10E7700003E12C50400B02E08DEC0EF0259A1AAC10
:10E7800002D0C6EC09F028A203D02892F0EC39F0B0
:10E790001C8C12002050010B14E002012D5111E1DC
:10E7A0001750800B06E05DECD2F009E00B0E155C13
:10E7B00006E02050040B05E13FECCDF002E0BEEF97
:10E7C00071F002012A5104E034ECD0F040ECCEF0BC
:10E7D00017AE5BD06EEC97F0A1ECCBF017E02F50AA
:10E7E000200B14E13050040B11E12350800B0EE19B
:10E7F0003050400B0BE12450010B08E13250010B6B
:10E8000005E13250020B02E1ABEC2EF032921FAA6E
:10E810003CD01F9A01013BAB38D037ECCFF002015E
:10E82000315110E1F8EC34F0190E155C14E1175079
:10E83000010B11E00101D451D55D0DE10201C80EBB
:10E84000316F1200316B1C0EE66E4AECE2F0E552BD
:10E850000101960EAC6F120044ECCEF016E14A5066
:10E8600014E121BA12D0C9EC07F0000902E1C4ECAE
:10E87000D4F04FEC0DF0238A810E076EC9EC07F03F
:10E88000000903E0ABEC2EF0258212000C04040F0B
:10E890000701006F12000101B59B19AC27D00DECE8
:10E8A0000BF0138225A41CD09EECDBF03B0EE66E31
:10E8B000E30EE66E010E8FECD7F090ECDFF0E30E86
:10E8C0000C2452ECCAF01AEC0BF09EECDBF0330E89
:10E8D000E66EE30EE66E010E8FECD7F090ECDFF003
:10E8E00002010E0E376F060E386F1200CFDF0701E0
:10E8F000FA0E036F016B026B0201536B546B1D9098
:10E90000120000C709F00201555104E0800EEAEC44
:10E91000CAF01A800701035117E003510307ECEC1A
:10E92000CBF0CC0E005C10E0FF0E005C0DE0800E22
:10E93000005C06E20050E66E3CEC04F0E552006E2E
:10E940000050EAECCAF0E6D7096A120083ECDAF06C
:10E95000DBCF55F22F88006A2388E9EC26F001010D
:10E96000320EAC6F17A802D00201558F0201195167
:10E9700002E0010E196F179EE3EFC9F017A802D04D
:10E980002EEC48F019AC24D00DEC0BF0139280EC77
:10E99000D7F0D00ED8800E54050E0F5405E292EC3D
:10E9A00065F00201196B120013820101E683218ECA
:10E9B000EFEC0AF0198AE0EC08F000090FE120847E
:10E9C0000101E4993FECCDF009E00101E489120076
:10E9D000278A02012D5102E0010E2D6F1200E7EC93
:10E9E000C9F0198CA4ECCAF003E00AECCBF001E00A
:10E9F000199C25A410D0FE0EDB500C6E4CDF259424
:10EA00000101B587239C24B2238C248219AC32D017
:10EA1000198428802FD01950400B0EE0E0EC08F04C
:10EA200000090AE03FECCDF007E02050040B04E1C0
:10EA30001D0E9FECCAF01ED0FD0EDB500DE1020151
:10EA4000195103E12750400B07E095ECD5F07EDF2C
:10EA5000E5520201196B0ED0FE0EDB500C6E1BDF6F
:10EA600019BC07D04EDF0501105103E192EC65F0AF
:10EA700001D084DFE3EFC9F00601060E406F73ECAE
:10EA8000CEF004E2A85102E00601402B02011E0E66
:10EA9000276F120001012951E8240301B86F0A0110
:10EAA000190ED76F360ED66F0101D45103E0030E55
:10EAB000D45D03E10A01080ED66F51ECD2F003E1F8
:10EAC0000A013C0ED66F0A01DA8FD46B348473EFDF
:10EAD000CCF0E7ECC9F07EEC39F091EC19F033881A
:10EAE00095ECD5F08CEC1BF0E552E3EFC9F0010E8C
:10EAF000E66EEFDFE5521200000403E1EDECD7F023
:10EB00001BD0005045E0030E005C18E1EDECD7F09F
:10EB1000C5ECD0F004E0E80E0E6E030E0F6EAEEC06
:10EB2000CDF004E06AEC04F0B8ECCAF0BDECCAF039
:10EB300003E1640E0E6E0F6A7DEFD9F04FEC15F015
:10EB4000930E0E6E020E0F6E0050030819E2700E47
:10EB50000E6E030E0F6E050E005C04E1930E0E6E3A
:10EB6000020E0F6E060E005C04E1970E0E6E040E90
:10EB70000F6E070E005C04E1200E0E6E060E0F6E87
:10EB80007DECD9F0020E005C05E1500E16ECCAF0E7
:10EB9000C6EF0AF00050030803E20201040E356FCD
:10EBA000070E005C03E10201080E356F1200E7EC6E
:10EBB000C9F0280E04ECD6F0290E93ECCAF0E3EF6E
:10EBC000C9F0D9CFE6FFE1CFD9FFE6528C9E000015
:10EBD0000000000000008C9600000000060EE66EAB
:10EBE000A2EC5CF0E5528C860000000000008C96E0
:10EBF00000000000D80EE66EA2EC5CF0E552A5C75E
:10EC0000E6FFA2EC5CF0E552E66AA2EC5CF0E552AD
:10EC1000E66AA2EC5CF0E5528C868C8EDF6A1E0EF2
:10EC2000DF5C07E2640EE66EBFEC21F0E552DF2AFE
:10EC3000F6D7E552E552E7CFD9FF1200D9CFE6FF6C
:10EC4000E1CFD9FF8C9E00000000000000008C96F0
:10EC500000000000030EE66EA2EC5CF0E552A5C7D2
:10EC6000E6FFA2EC5CF0E552FC0EDBCFE6FFA2EC87
:10EC70005CF0E552FB0EDBCFE6FFA2EC5CF0E55268
:10EC8000FA0EDBCFF3FFDB06F35000090FE0D3EC05
:10EC9000FDF0006EFD0EDBCFE9FFDB2AFE0EDBCFC1
:10ECA000EAFF01E3DB2A00C0EFFFEAD700008C8611
:10ECB000C69E8C8EE552E7CFD9FF120063ECD5F0EB
:10ECC000DF6ADF2AFA0EDBCFE6FF3BECD0F022EC66
:10ECD000CEF042ECD0F0FA0EDBCFE6FF3BECD0F00A
:10ECE000A80EE66E030EE66E42ECD0F0010EDB6A73
:10ECF000FA0EDB5065ECCCF017E2010EDB50E76E4C
:10ED000046ECD0F0E7507DECD6F0EFCF49F0010EA5
:10ED1000DB50EA6AA80FE96E030EEA22EF50495C65
:10ED200003E1010EDB2AE4D7AEECD3F002E03DECC8
:10ED30000DF0AEECD3F003E00A0EDF5CC2E30A0E86
:10ED4000DF5C02E3000E01D0010EFCECD2F002E227
:10ED5000E16AE552E16E4950E3EFC9F0D9CFE6FF31
:10ED6000E1CFD9FF8C9E00000000000000008C96CF
:10ED700000000000060EE66EA2EC5CF0E5528C8608
:10ED80000000000000008C9600000000020EE66EFD
:10ED9000A2EC5CF0E552A5C7E6FFA2EC5CF0E55200
:10EDA000FE0EDBCFE6FFA2EC5CF0E552FD0EDBCF02
:10EDB000E6FFA2EC5CF0E552FA0EDBCFF3FFDB06D8
:10EDC000F350000911E0FB0EDBCFE9FFDB2AFC0E5C
:10EDD000DBCFEAFF01E3DB2AEF50006E0050E66E66
:10EDE000A2EC5CF0E552E8D700008C86C69E8C8EC3
:10EDF000050EE66EBFEC21F0E552E552E7CFD9FFF4
:10EE00001200D9CFE6FFE1CFD9FFE652CEEC5CF09D
:10EE10000101640EAC6F0400EBEC41F0020E07013F
:10EE20005A5D0FE00701945109E0A9EC05F00401D7
:10EE3000FD6FFDC4E6FFCCEC05F0E55203ECA8F055
:10EE400071D0070194516EE007019451496E4A6AEE
:10EE50004A3404E24950C008000E4A5408E207014F
:10EE6000040E266F270EE66EA6EC14F0E552A9EC10
:10EE700005F00401FD6F3B0E0401FD5D0CE1040192
:10EE80003B0EFE6F0601C46B309A0101379BBCEC50
:10EE90000CF007015A6B610E0401FD5D07E30401EC
:10EEA000FD51660803E3200E0401FD5F300E0401EE
:10EEB000FD5D22E30401FD5146081EE30601C42B5B
:10EEC000410E0401FD5D04E2300E0401FD5F06D039
:10EED000410E0401FD5D0A0F0401FD6F020E0601E3
:10EEE000C45D08E10601C339F00B0401FD250401EE
:10EEF000FD6F02D0FDC4C3F6020E0601C45D11E130
:10EF0000FDC4E6FF17EC0DF0E552006E010EE66E53
:10EF1000BFEC21F0E5520601C46B0050E66E47DEFF
:10EF2000E5528FD70201685102E077EC8EF01C9C0D
:10EF3000100E075C03E207EC6CF024D01E0E075C99
:10EF400003E282EC70F01ED00750496E4A6AD890F6
:10EF50004A5004E6800E495C000E4A5803E2FFEC7A
:10EF600021F010D00750496E4A6AD8904A5004E602
:10EF7000920E495C000E4A5803E2D1EC71F002D0C7
:10EF8000AAEC2DF01CBCD3D7A6EC53F0095008E036
:10EF90000701070E266F270EE66EA6EC14F0E55269
:10EFA00022A228D022922E98329AD8EC80F0DF68E4
:10EFB0002E50100B15E0010101012A51040B10E144
:10EFC0002950020B0DE1DF500BE00D5002E1010E64
:10EFD0000D6E2E9832EC8EF0D8EC80F0DF06E8D77C
:10EFE000DF5008E10701050E266F270EE66EA6EC3E
:10EFF00014F0E55210D7E552E552E7CFD9FF1200E1
:10F000000101E6A507D0D40501E1020C020ED45D92
:10F0100001E1010CD4511200080E016E0101D4511E
:10F0200002E1180E016E380EB95D09E1016A8BEC40
:10F030000BF0000902E0100E016E3AEC19F012001C
:10F04000200EE66E640EE66E070EE66E800E81EF11
:10F05000D6F0A5ECD6F07CECCFF0EFCFDFFFFF0EC3
:10F06000DF5C02E1100EDF6EDF50E552E3EFC9F026
:10F07000D3DF03015E510126015065ECD4F0046E2C
:10F08000120037ECCFF00101040E016F0450006E46
:10F0900000500F0803E2100E005E04D0100ED8805E
:10F0A0000054006E9DECE1F00101200E1A6F050E78
:10F0B000006E300E1B5D02E0040E006E04500F085F
:10F0C00005E2005089ECCBF02B0E04D0005089EC07
:10F0D000CBF02D0EEF6E010E016F6C0E496EF40E2B
:10F0E0004A6E010E4B6E5EC34CF04D6A4E6A4BEC9D
:10F0F000D5F01CECD6F00101188F12001D0E010195
:10F10000B95D01E1010C000C5FECD5F00050EF0897
:10F110005CE2F00E005CDF6EDF50080862E329500D
:10F12000010B05E10401F95102E1FA5108E0010186
:10F13000E4910201246B3C6B03ECA8F0F0D737ECB0
:10F14000CFF0C9ECD0F0DF50FE0BE842750F096E2E
:10F15000016ADFA002D0800E016E026A070E025C17
:10F160000CE256EC3BF0005008E0FF0E005C05E0BE
:10F170002EECE2F0012A022AF1D790ECDFF0010137
:10F18000E485080E016EDFA002D0800E0126026A1F
:10F19000780E025C10E256EC3BF000500CE0FF0EE3
:10F1A000005C09E00050036EE66ECCEC05F0E55221
:10F1B000012A022AEDD73B0E035C05E03B0EE66E0A
:10F1C000CCEC05F0E552096A16D0B5ECD3F000504E
:10F1D00070ECD5F0056EFF0E055C05E16C0E00ECE1
:10F1E000CBF0258E08D0B9C157F205C0B9F12982FC
:10F1F0000201010E686FE552E3EFC9F01D0E010137
:10F20000B95D04E1F00E03015D2513D00068016AC9
:10F21000015082ECCAF004E6960E495C000E4A5892
:10F220000CE2B5ECD3F0015070ECD5F0B95D03E120
:10F230000150006E1200012AEBD71200020E016E7F
:10F240002AC100F013EC3BF02F0E016E57C100F005
:10F2500013EC3BF0370E016E5FC100F013EC3BF096
:10F260000F0E016E37C100F013EC3BF0100E016E73
:10F2700038C100F013EC3BF02E0E016E56C100F0C9
:10F2800013EC3BF0620E016E8AC100F013EC3BF010
:10F29000650E016E8DC100F013EC3BF0660E016E41
:10F2A0008EC100F013EC3BF06E0E016E96C100F0C3
:10F2B00013EF3BF0130E016E3BC100F013EF3BF078
:10F2C0003F0E0101B95D02E119A6D17B0A0EB95DBD
:10F2D00005E119B603D05F77FCEC35F0170E01019C
:10F2E000B95D14E119A63B79DAEC1EF0ABEC2EF017
:10F2F00008ECD3F004E02150020B01E1E8893BB9AE
:10F3000003D01E9A73ECCCF0050147873E0E010135
:10F31000B95D09E119B607D0020E425D02E1010EA6
:10F3200001D0020E426F050EB95D03E0060EB95D15
:10F3300011E119B608D0050EB95D03E10701BE71F0
:10F3400002D00701BE7323ECD2F07EEC09F002017B
:10F3500007812D84290E0101B95D04E119A6777199
:10F36000B5EC20F0220E0101B95D02E119A68D79FC
:10F37000100EB95D04E119A63E7179EC5CF0280E1F
:10F380000101B95D0AE119A6387591ECD4F001E0EC
:10F39000098FBEECC4F0F0EC39F0110E0101B95D3B
:10F3A00002E119A6D27B190EB95D02E119A6387FD8
:10F3B000090EB95D02E119A6967DB95104E119A6BD
:10F3C000337446EC1FF0320E0101B95D02E119A65B
:10F3D0002A752D0EB95D02E119A62A731B0EB95DBF
:10F3E00001E12E74300EB95D01E12E72400EB95D5F
:10F3F00002E119A63771130EB95D02E119A62A7F41
:10F400002F0EB95D0CE119B608D05F9F2F0EE66E86
:10F41000E30EE66E010E12ECCAF0B5EC20F012001D
:10F420005FECD5F046ECD0F0EFCFDFFFFB0EDB500A
:10F43000D880DF5403E2FB0EDB50DF6EFC0EDB50A6
:10F44000DF5C03E2FC0EDB50DF6E0DAE0CD0FC0E79
:10F45000DB50D880DF5402E2DF0605D032B603D09D
:10F46000FB0EDB50DF6E0D040BE1FB0EDB50DF5CAF
:10F4700002E2DF2A05D032B603D0FC0EDB50DF6E8D
:10F4800046ECD0F0DFCFEFFFE552E3EFC9F0B2EC8E
:10F49000D7F04DECD0F0E3EFC9F0E7ECC9F03286DD
:10F4A0003BECD0F022ECCEF04DECD0F03296E3EF16
:10F4B000C9F0B2ECD7F086ECDBF0E3EFC9F0500E08
:10F4C000036E00ECD6F005E01B50080B02E11E0EA7
:10F4D000036E12005FECD5F0F3DE310E0101B95D71
:10F4E0002AE13651070B006E0D040EE136BF02D043
:10F4F000368F1AD036BD03D0368D006A15D0070E70
:10F50000005C12E2002A10D0FF0E0D5C0DE10050ED
:10F5100005E0000600AE08D0006A02D036AD02D089
:10F52000369D02D036BF369F0050070BF36EF80EA3
:10F530003615F310366F1F0EB95D13E10D0408E1A7
:10F5400056B102D056810DD056B50BD0568509D094
:10F55000FF0E0D5C06E156A502D0569502D056B1BD
:10F5600056910D0EB95D0BE1150EE66E030EE66EBB
:10F57000550EE66E010E25ECCAF08CEC04F00E0E72
:10F580000101B95D08E1050EE66E830EE66E010E1F
:10F5900020ECCAF0339C0C0E0101B95D15E1020E9E
:10F5A000E66E840EE66E010E20ECCAF0300E01010C
:10F5B00084250401F76F020E0101845D03E104015B
:10F5C000340EF76FC8ECA7F0230E0101B95D13E10B
:10F5D000030ED015066F065102E1010E066F030EF1
:10F5E00025ECDBF0FC0E0101D0170651D013B5EC71
:10F5F00020F0050147892C0E0101B95D07E119A62C
:10F60000D2711E9A73ECCCF0ABEC2EF0120E01010D
:10F61000B95D2EE10D0411E1080E505D02E10D0E01
:10F6200026D0050E505D1EE0030E505D16E050051D
:10F630000FE00D0E505D1CE006D0FF0E0D5C18E1D2
:10F64000030E505D02E1010E12D0050E505D02E185
:10F65000030E0DD0080E505D02E1050E08D00D0E10
:10F66000505D02E1080E03D0500502E0010E506F1C
:10F67000240EB95D2DE1E7AB03D0D9EC0BF028D017
:10F68000640E006E0701BEAB02D00A0E006E0D04C0
:10F6900009E10001005001016927000E6A236B2374
:10F6A0006C2310D0FF0E0D5C0DE176ECDAF04B6AA6
:10F6B0004C6A49500101695F4A506A5B4B506B5B71
:10F6C0004C506C5B95ECC7F024843388F0EC39F037
:10F6D000140E0101B95D0BE1030E4F15066F020E0A
:10F6E000C3ECDAF0FC0E01014F1706514F13150E53
:10F6F000B95D11E1300E4F15066F06390F0B066F1D
:10F70000020EC3ECDAF001010639F00B066FCF0EE2
:10F710004F1706514F130F0EB95D09E1820EE66EC9
:10F72000520EE66E510EE66E010E25ECCAF03D0E4D
:10F730000101B95D19E10701BE51E840E8403F0B06
:10F740000101066F030E0617C3ECDAF00101040E87
:10F750000603F3CF06F1F30E0701BE1701010651B0
:10F760000701BE137EEC09F0430E0101B95D13E100
:10F77000E6A508D0B40EE66E640EE66E4A0EE66E9E
:10F78000010E07D0730EE66E460EE66E520EE66E62
:10F79000010E25ECCAF020ECD3F036E12050040B2A
:10F7A00003E11B50080B30E00D0414E12B50040B57
:10F7B00002E0140E01D0010E496E4A6A49BE4A6841
:10F7C0002250040B01E0010E9FECCDF04950EE26D3
:10F7D0004A50ED22FF0E0D5C14E12B50040B02E0A9
:10F7E000140E01D0010E496E4A6A49BE4A68225081
:10F7F000040B01E0010E9FECCDF04950EE5E4A5043
:10F80000ED5AF8EC15F01E88350E0101B95D07E1DF
:10F81000110EE66ED40EE66E010EF6ECCDF03A0E49
:10F820000101B95D29E133A60BD0E90EE66ED30ED6
:10F83000E66E010EE66E0DEC27F0E552E55218D0AB
:10F840002B510A0817E307ECC3F0E66E7DEC13F0CA
:10F85000E55285ECCBF00EE100C006F1DC0E25ECA4
:10F86000DBF006C100F013EC3BF0E66AC3EC1CF0E1
:10F87000E55202D0D9EC0BF0180E0101B95D20E180
:10F88000E3AD12D00C0EE66E030EE66E07ECD5F07B
:10F8900004E1950E496E010E03D0930E496E010EE0
:10F8A0004A6E53ECCBF008D0780EE66E280EE66E6A
:10F8B000870EE66E010EE66E86ECDBF013EC09F0C7
:10F8C000250E0101B95D07E1FA0EE66E880EE66EBF
:10F8D000020E20ECCAF01A0E0101B95D07E1020E1A
:10F8E000E66E700EE66E020E20ECCAF0210E0101EB
:10F8F000B95D1CE1020EE66E390EE66E010E20ECDB
:10F90000CAF00101395104E134ECDAF080EC25F061
:10F9100082ECCFF0006A0101395102E0010E006E65
:10F9200000C0D4F200C0D3F200C0EBF9B90507E182
:10F93000050EE66E940EE66E010E20ECCAF00B0E7C
:10F940000101B95D01E085D039512CE030A227D00A
:10F950000901E85104E10D0401E079D016D0E80571
:10F9600011E10D0408E1010EE86F230EE66EE30ECF
:10F97000E66E010E11D0E86B1D0EE66EE30EE66E2C
:10F98000010E0AD0FF0E0D5C62E1010EE86F290E38
:10F99000E66EE30EE66E010E48ECCAF058D0D9ECE4
:10F9A0000BF057D01E862950020B0AE03A5108E0AE
:10F9B0003A51010802E2010E01D0020E3A6F07D05F
:10F9C000130EE66E3A0EE66E010E20ECCAF064EC01
:10F9D00009F001013A5102E08D8303D03A5101E16F
:10F9E0008D93030E3A5D33E33A51130830E3000E72
:10F9F000036E026E016E030E3A5D006E080E005C2F
:10FA00000BE2010E00C0E7FFE75204E0E846FE0B00
:10FA1000E706FCE1016E12D0100E005C0CE2080E4D
:10FA2000005C496E010E495204E0E846FE0B4906AF
:10FA3000FCE1026E03D0100E005C036E010EE66E58
:10FA40000350E66E20ECDAF009ECCEF002D09FEC29
:10FA5000BDF0030E0101B95D0BE11E0EE66E010E55
:10FA6000E66E700EE66E010E25ECCAF044EC1FF057
:10FA7000070E0101B95D51E1E95109E1080EE66E99
:10FA8000040EE66E470EE66E010E25ECCAF001018B
:10FA9000E90508E1E668C80EE66E7D0EE66E010E29
:10FAA00025ECCAF0020E0101E95D08E1C80EE66E20
:10FAB000E66A4B0EE66E010E25ECCAF0030E01015C
:10FAC000E95D14E10701BEA308D0960EE66E780E3C
:10FAD000E66E4D0EE66E010E07D0320EE66E0A0E91
:10FAE000E66E4C0EE66E010E25ECCAF0040E010126
:10FAF000E95D09E10F0EE66E0A0EE66E410EE66E56
:10FB0000010E25ECCAF0050E0101E95D04E119A61C
:10FB1000627354EC1EF044EC1FF02A0E0101B95D33
:10FB20003AE1016AD45102E0010E016E020E0901B0
:10FB3000E55D1BE171ECD6F00AE1FFECD6F004E6DE
:10FB4000E20E495C000E4A5802E2190E0026FF0E32
:10FB50000D5C05E10050180802E2190E005E01502C
:10FB600087ECCAF000C0EFFF14D0020EE55D11E291
:10FB7000FA0EE66E010EE66E0150030DB7ECCCF006
:10FB8000B80E4B26020E4C22E551BAECD7F086ECAB
:10FB9000DBF057EC4EF0340E0101B95D07E1640E65
:10FBA000E66E850EE66E010E20ECCAF0040E010131
:10FBB000B95D09E1020EE66E310EE66E010E20EC33
:10FBC000CAF0DAEC1EF0370E0101B95D10E12B51DD
:10FBD0000A0806E20F0EE66E7B0EE66E010E05D0F9
:10FBE0000F0EE66E860EE66E010E20ECCAF03B0E9E
:10FBF0000101B95D0CE13AEC19F0190EE66EE66A06
:10FC00007A0EE66E010E25ECCAF0C3EC15F0390E43
:10FC10000101B95D0BE1280EE66E1E0EE66E890E3F
:10FC2000E66E010E25ECCAF033ECD3F0410E010173
:10FC3000B95D09E13C0EE66E6E0EE66E010E20EC3B
:10FC4000CAF025EC19F0420E0101B95D09E13C0E44
:10FC5000E66E6F0EE66E010E20ECCAF025EC19F090
:10FC6000330E0101B95D28E181C306F13B0E016E3F
:10FC700003017F5104E180C306F1170E016E020EED
:10FC80007F5D02E182C306F10150E5ECD5F01EEC88
:10FC9000CDF003017F5102E106C180F37F0502E14F
:10FCA00006C181F3020E7F5D02E106C182F301010C
:10FCB000835102E09FECE3F0080E0101B95D16E10B
:10FCC00003017F5107E1170EE66E830EE66E030E09
:10FCD0001EECCDF003017F0507E13B0EE66E840EBE
:10FCE000E66E030E1EECCDF0A8ECE3F0020E01016F
:10FCF000B95D0EE11B50080B02E0060E01D0050EA7
:10FD0000E66E800EE66E010E20ECCAF0CFEC04F039
:10FD100033ECD5F02CE1016AD5CA03F0D251010BC6
:10FD200012E03751080B0FE0040E036E1BA00BD03E
:10FD3000030E036E010E016E0A011C5104E1280E30
:10FD4000216F21CA1CFAFE0EB6ECCDF00501175149
:10FD5000050DB7ECCCF0140E4B260A0E4C220350C6
:10FD6000BAECD7F04DECD0F02484BDEC0DF03C0E95
:10FD70000101B95D0FE1FA0EE66E2250040B01E0BD
:10FD8000010E4A6A910F496E020EA3ECD7F0F8EC0F
:10FD900015F01E88270E0101B95D03E0380EB95D2C
:10FDA0001BE1030ED45D03E1D9EC0BF015D027EC79
:10FDB000D5F038EC78F004C006F1200EC3ECDAF090
:10FDC00001507CECCFF006C1EFFF308E06C104F08D
:10FDD00041EC78F04CEC1EF01E0E0101B95D06E11D
:10FDE00019B602D002017879EDEC15F0260E01016A
:10FDF000B95D09E1030EE66E430EE66E010E20ECDE
:10FE0000CAF087EC21F01C0E0101B95D0FE13EC183
:10FE1000DFFF188C3E6B070EE66E3F0EE66E010E9E
:10FE200020ECCAF0C8ECD4F0DFCF3EF1200E010187
:10FE3000B95D02E10D503327160EB95D09E10C0ED4
:10FE4000E66E070EE66E3D0EE66E010E25ECCAF07C
:10FE50005CC3E6FF27EC0CF0E552440E0101B95DEE
:10FE600014E119B611D065ECDBF0040A01E0010ED3
:10FE7000496E1BECCAF04950010BF36EF346F34692
:10FE8000FB0EEF14F310EF6E2E86450EB95D32E1D6
:10FE900040ECD8F0016E32ECD7F0026E0D50022625
:10FEA00002AE0ED0630E026E0106015058ECCBF08C
:10FEB00007E24950F908000E4A5402E2F90E016EB9
:10FEC0000250630802E2026A012A015058ECCBF0AA
:10FED00006E24950F908000E4A5401E2016A1BEC9F
:10FEE000CAF0030E01C0EBFF1BECCAF0020E02C009
:10FEF000EBFF2E86460EB95D1BE13BECD8F0016EA0
:10FF00000D50E824012601500A0802E20A0E016E93
:10FF1000080E015C02E1090E016E030E015C02E2B3
:10FF2000030E016E1BECCAF0010E01C0EBFF2E8622
:10FF3000480EB95D50E1CFECD9F0496E4A6ACAEC7F
:10FF4000D9F00A0DF3504924DA6FF4504A20DB6FE0
:10FF5000D4ECD9F002E127ECD2F00D040CE1D890FA
:10FF6000DB5104E6E70EDA5D030EDB5911E2DA2B12
:10FF7000000EDB230DD0FF0E0D5C0AE1DB3504E340
:10FF8000DA511908FC0EDB5503E2DA07000EDB5BE1
:10FF90002888800EDB1503E0289827ECD2F0DAC120
:10FFA00049F0DBC14AF00A0E01ECCAF01BECCAF0C2
:10FFB000040E49C0EBFF1BECCAF0050E39C0EBFF85
:10FFC0001BECCAF02850100B02E0EF8001D0EF903C
:10FFD0002E86ABEC2EF0470E0101B95D3FE11BEC24
:10FFE000CAF0060EEB50006E1BECCAF00490EF5006
:10FFF000020B01E004800D500026005006E1047061
:020000040001F9
:1000000004805FEC7AF00350006E5FEC7AF00350EE
:10001000D880005404E204700480010E006EAEEC3F
:10002000D6F001E0049004801BECCAF00450010BF0
:1000300002E0EF8201D0EF921BECCAF0060E00C086
:10004000EBFF100E01012B5D03015C5D06E100C0BA
:1000500048F16EECCCF05CC300F02E86490E010135
:10006000B95D39E10490AEECD6F001E004801BEC00
:10007000CAF0EF50016E0F0E0114006E01380F0B25
:10008000016E0D50012604A00CD00150800803E23F
:10009000090E016E0490015009080CE2090E016E70
:1000A00009D0015002E1010E016E0150090802E27F
:1000B000016A04800138F00B016E015000126BECF4
:1000C000D9F0090E7DECD6F00450010B02E0EF8E62
:1000D00001D0EF9E2E86E552E3EFC9F05C0E0024BE
:1000E000EBECD9F00101100E136F145102E1100E68
:1000F000146F120032ECD7F0B9ECCEF040ECD8F02F
:10010000006E0101030E006F80ECE1F0060EE66E5A
:10011000030E88EFCFF085ECD5F00A0809E2FE0E59
:10012000DB50F00F006E00502EECCFF0E3DF23D059
:10013000FE0EDB50006ED2DF020E6DECCAF00DE257
:100140000101010E146F080E156FFE0EDB040DE1A8
:10015000030E146F050E156F08D013C112F114C1F0
:1001600013F115C114F10101156B23ECD5F002E177
:10017000090E156F158FE3EFC9F010EC26F02E80F5
:100180001200140E006E04A002D0110E006EBDEF1E
:1001900080F00E0E006E04A002D0080E006EBDEFBF
:1001A00080F0E5EC11F0D0C7F3FFD1C7F4FF1200E7
:1001B000B2ECD6F00101B551800B04E02F50100BCA
:1001C00001E1E3D09EECDBF048EC8DF00101395108
:1001D0000DE00B0EB95D0AE1016B150EE66EE30E44
:1001E000E66E010E8FECD7F00101198F0A0EB95D92
:1001F00001E1198F070EB95D49E1040E016F2A0E66
:10020000196FE95108E1110EE66EE30EE66E010E7C
:10021000E66E7EECCAF00101E90508E10D0EE66E1E
:10022000E30EE66E010EE66E7EECCAF0020E0101F0
:10023000E95D08E1090EE66EE30EE66E010EE66E7C
:100240007EECCAF0030E0101E95D08E1050EE66EE1
:10025000E30EE66E010EE66E7EECCAF0040E0101BE
:10026000E95D08E1010EE66EE30EE66E010EE66E54
:100270007EECCAF0050E0101E95D08E1FD0EE66EB7
:10028000E20EE66E010EE66E7EECCAF02A0E010169
:10029000B95D0FE1420E1C6F0901E50503E10101A3
:1002A000440E1C6F020E0901E55D03E101014D0ED4
:1002B0001C6F350E0101B95D11E10201B0510EE074
:1002C0009EECDBF0F60EE66EE20EE66E010E8FECB3
:1002D000D7F02CA203D00101370E1B6F33ECD5F001
:1002E00007E13751080B04E04C0E1B6F2A0E1C6F00
:1002F000240EB95D0CE196A302D0230E07D057A9B6
:1003000006D02A0E196F57BB02D03F0E196F1FA8D7
:1003100005D09EECDBF0006A25EC26F0FFEC63F0E4
:10032000000905E0310E03015C250101186F1D0E67
:100330000101B95D05E1310E03015D2501011C6F6D
:10034000270EB95D03E0380EB95D05E1310E0301FA
:100350005E2501011C6F430EB95D0CE1E651040BF3
:1003600009E0016BEE0EE66EE20EE66E010EE66E41
:100370007EECCAF0180E0101B95D07E1E351400BB4
:1003800004E0500E166F4C0E176F8EECDBF07CEC19
:10039000D8F00E0E136F146F7EEC78F0000907E0B2
:1003A0000101006B280EE66E24ECE2F0E552016AD2
:1003B000410E0101B95D08E16EC100F00168020162
:1003C0006E0EA46F010EA56F420E0101B95D08E12A
:1003D0006FC100F0016802016F0EA46F010EA56FDE
:1003E000200E0101B95D08E10201330EA46F010E78
:1003F000A56F33C100F00168160E0101B95D0BE174
:10040000050E3D03F350410F006E016802013D0EE1
:10041000A46F010EA56F1C0E0101B95D08E13F2913
:10042000006E016802013F0EA46F010EA56F180E49
:100430000101B95D26E18751FE0BE842006E020121
:10044000870EA46F010EA56F0101E3AD18D093C113
:1004500000F00201930EA46F010EA56F330E875DAD
:100460000AE101019551FE0BE842006E0201950E72
:10047000A46F010EA56F050E0002F3CF00F0016816
:100480002E88070E0101B95D65E1E95106E102011F
:10049000470EA46F010E40ECCBF00101E90506E127
:1004A00002017D0EA46F010E40ECCBF0020E0101A3
:1004B000E95D06E102014B0EA46F010E40ECCBF0AA
:1004C000030E0101E95D1DE1006B0701BEA30CD025
:1004D000EA0EE66EE20EE66E010E08ECCAF00201CC
:1004E0004D0EA46F010E0BD0E60EE66EE20EE66E28
:1004F000010E08ECCAF002014C0EA46F010E40EC94
:10050000CBF0040E0101E95D06E10201410EA46F8A
:10051000010E40ECCBF00168050E0101E95D17E129
:10052000016A62A306D0E20EE66EE20EE66E010EEE
:1005300005D0DE0EE66EE20EE66E010E08ECCAF0A5
:100540000201620EA46F010EA56F020EA66F0101DB
:10055000050E006F2A0EB95D1CE1026AD45102E05B
:10056000010E026E0250030D23ECD6F0B80E4926A0
:10057000020E4A220901E551B2ECD8F0020E09013F
:10058000E55D05E1190E28ECD6F01BECCEF0016814
:100590002E883D0E0101B95D0AE1D4C1E6FF56EC9B
:1005A0000DF0E5520168C4ECD1F00C0EA66F0150BD
:1005B00002E080ECE1F0160E0101B95D09E0180ED1
:1005C000B95D08E1E351400B05E007ECD5F002E02E
:1005D0000101148F3D0E0101B95D09E0180EB95DEE
:1005E0000CE1E351400B03E007ECD5F006E101011B
:1005F000135102E1100E136F158F0D0E0101B95D3D
:100600001FE1150E555D0BE1006BD50EE66EE20E97
:10061000E66E010EE66E1EECE2F0E5520AD055C120
:1006200000F080ECE1F0060EE66E050EE66E29ECB9
:1006300009F0E552E5520201550EA46F010EA56FB7
:100640003F0E0101B95D10E1D1AB02D0080E01D01F
:100650000E0E75ECCDF02E800201D10EA46F010EAE
:10066000A56F200EA66F2E88050E0101B95D0DE164
:100670000701BEB102D00E0E01D0080E75ECCDF010
:10068000C4ECD1F0010EA66F2E80060E0101B95DFB
:1006900017E10701BEB306D0E60EE66EE20EE66E87
:1006A000010E07D001010007D00EE66EE20EE66EE5
:1006B000010E08ECCAF0C4ECD1F0020EA66F2E8039
:1006C0000101B9052EE10B0E75ECCDF0010194513D
:1006D00006E1010E006F440E006E10EC26F00101E1
:1006E0009451010819E2006BC70EE66EE20EE66E49
:1006F000010E08ECCAF0050E0101945D02E1158FB0
:100700000BD0050E006F9405190DF350B9ECCEF027
:100710000101100E136F148F0201940EA46F010ECD
:10072000A56F110E0101B95D1EE12BC1E6FFF3DCDF
:10073000E55212C10EF113C10FF114C110F115C130
:1007400011F10101100E126F050E006FD2AB02D035
:10075000290E01D02A0EE66E24ECE2F0E552CAEC36
:10076000D1F0200EA66F2C0E0101B95D1AE18FECBD
:10077000CCF07CECD8F00B0E75ECCDF00101D2A1E1
:100780000BD0050E006FC30EE66EE20EE66E010E94
:1007900008ECCAF00101158FCAECD1F0010EA66F6A
:1007A0002E88230E0101B95D20E18FECCCF0010110
:1007B000030E006FBD0EE66EE20EE66E010E08EC53
:1007C000CAF00101D051010B05E0D051020B02E04B
:1007D000030E03D0D0A302D0020E126F0201D00E7E
:1007E000A46F010EA56F030EA66F20ECD3F029E1D4
:1007F0002250040B01E0010E010F0E6F030E006F7B
:1008000004902250040B01E0010E9FECCDF0EECFDE
:100810000EF0EDCF0FF09CEC26F00101100E116FE1
:100820002BB4156F2250040B01E0010E020DF3CF23
:10083000F3F6F4CFF4F68D0E0601F327020EF4233F
:100840002E88350E0101B95D01E019D124B80CD014
:10085000006BC3EC64F0B9ECCEF07CECD8F0CCECDF
:1008600064F0B9ECCEF00AD15CEC10F013ECCFF0F0
:100870005CEC10F00E500101D8270F50D923D8C1DD
:100880000EF0D9C10FF0010E0F0B04E055ECD2F0C1
:10089000E806FCE107010E500C5D0F500D5905E212
:1008A0000C510E5E0D510F5A02D00E6A0F6A0EC027
:1008B0000EF70FC00FF70201B0511CE0190E28EC23
:1008C000D6F0B0C23EF00BECD5F004E17EEC04F0C3
:1008D0000201B16FB1C200F00101126B58ECD8F007
:1008E0005AECFEF03EC013F13AC014F10101110EB2
:1008F000156F138FC3EC64F0026E006E2CA204D04F
:10090000CCEC64F0026E006E0201B05157E0960E1E
:100910000101D86FD96B1FA003D0F00ED86FD96B2F
:100920000CECD3F004E0320E0101D86FD96B010159
:10093000D8510E5CD9510F5810E2FFECD6F004E606
:10094000F00E495C000E4A5808E2002A640E0201CB
:10095000B05D1DE2190EB0271AD00C0E4A6AD825D8
:10096000496ED9514A2228ECD7F005E200506408BC
:1009700002E200060CD00201B05158ECCBF007E2C5
:100980004950C808000E4A5402E2C80EB06F025027
:10099000005C73E02CB208D0E66A0050E66ED5EC3D
:1009A00064F0E552E66E07D00050E66EE5EC64F0C8
:1009B000E552E66EE66A5FECCEF05FD02CB244D032
:1009C000C3EC64F0496E640E495C09E3C3EC64F067
:1009D0004A6E4B6A4B340DE236ECD2F00AE2C3ECBD
:1009E00064F00701266F510E20ECCBF055EC8EF031
:1009F00044D0E66AE66A5FECCEF00201FA0EB06F10
:100A00008CECD6F005E0D8900D330C33E806FBE112
:100A1000CCEC64F0496E640E495C09E3CCEC64F004
:100A20004A6E4B6A4B3408E236ECD2F005E2A00E77
:100A3000E66EE5EC64F0E552CCEC64F0E66EE66A56
:100A40005FECCEF02C8219D055EC8EF0CCEC64F03B
:100A5000496E640E495C09E3CCEC64F04A6E4B6A63
:100A60004B340AE236ECD2F007E2CCEC64F007013A
:100A7000266F540E20ECCBF02C9225822E88390E56
:100A80000101B95D18E1020E006F080E006E8AB117
:100A900002D00E0E006E10EC26F089C100F027EC9B
:100AA000CEF0100E136F158F02018A0EA46F010E87
:100AB000A56F010EA66F120E0101B95D25E1156B40
:100AC00015C114F1100E136F0D0E505D03E1010EF0
:100AD000146F17D0080E505D02E1050E09D0050E07
:100AE000505D02E1030E04D0030E505D03E1020EDF
:100AF000156F07D0500505E1010E156F006FEFEC83
:100B0000D9F00101158F2E883B0EB95D17E1020E59
:100B1000006F080E006E8AB302D00E0E006E10EC4D
:100B200026F07AC100F027ECCEF0100E136F020110
:100B30008A0EA46F010EA56F020EA66F370E01017B
:100B4000B95D1BE100EC6CF0050FB9ECCEF000ECE8
:100B50006CF0000904E124ECD3F0EFECD9F00201D1
:100B6000860EA46F010EA56F73ECCEF005E20201B4
:100B70007B0EA46F010EA56F2E88030E0101B95DD7
:100B800011E170C100F080ECE1F01E0E0101705D1A
:100B900004E1010E006FEFECD9F00201700EA46FBA
:100BA000010EA56F340E0101B95D11E1855104E11B
:100BB0000B0E75ECCDF006D085C100F080ECE1F0B5
:100BC0000101158F0201850EA46F010EA56F040EA1
:100BD0000101B95D1FE10201310EA46F010EA56F85
:100BE0000101040EF3ECD9F00101310506E1020E1A
:100BF000006F9E0E006E10EC26F0020E0101315DBA
:100C000009E1020E006FB70EE66EE20EE66E010E0F
:100C100008ECCAF0250E0101B95D11E1020188510D
:100C2000140DB8ECCAF08EECCFF00101100E116F6C
:100C3000006B328A0201880EA46F020EA56F270E88
:100C40000101B95D03E0380EB95D34E10CEC78F0D8
:100C5000026A080E025C2EE20150022465ECD4F018
:100C6000006E100E005C03E03AECCCF002E1020EE4
:100C700013D00050120802E2040E0ED000501008EB
:100C800002E2030E09D00E0E005C02E2006A05D0FB
:100C9000100E005C02E2010E006E410E00249CEC7E
:100CA000CBF0D00FE66E025004ECCBF07DECCCF034
:100CB000022ACFD7130E0101B95D0EE1100E146F99
:100CC00014C113F1110E156F2ABF152B0201CCECC4
:100CD000D4F0800EA66F2E80430E0101B95D18E19D
:100CE000050E006F52C100F00201520EA46F010EFA
:100CF000A56F0101E6A507D04AC100F002014A0E26
:100D0000A46F010EA56F80ECE1F00101148F2E8815
:100D10003A0EB95D4AE1006BB20EE66EE20EE66E87
:100D2000010E08ECCAF033B603D001010E0E0E6FAF
:100D300073ECCEF039E3050E006F85ECCBF003E1E8
:100D40005BECD4F01FD00101E49DB00E0D25ECEC5E
:100D5000CBF00F0E005C03E3005030080DE2230ED1
:100D6000006E0901EB510E0807E2310EEB5D04E263
:100D7000EBC900F00101E48D0101E4BD03D0005096
:100D8000D0ECD5F080ECE1F00101135102E1100E3E
:100D9000136F85ECCBF008E00101158F240E136F63
:100DA000E4AD02D0110E136F2E882E0E0101B95D35
:100DB00009E154EC09F09C0E0E5C630E0F5802E240
:100DC0008EECCFF0F8ECD2F001E022D1006BE7AB73
:100DD000F4D064ECD9F069ECCAF03D50B9ECCEF037
:100DE0000101240E0E6F9D0E20ECD8F00EC0DEFF28
:100DF0000FC0DDFFC80EC1ECD0F004E3840E80EC20
:100E0000D0F004E20701080E1FECD7F08EECCFF013
:100E10000101100E116F160E126FD1EC80F0F3CF9E
:100E200057F0F4CF58F057C0E6FF58C0E6FF68EC23
:100E3000D2F0E7CF58F0E552E7CF57F05750F32400
:100E4000556E5850F420566E55C0E6FF56C0E6FF6A
:100E500068ECD2F0E7CF56F0E552E7CF55F05550A9
:100E6000F324536E5650F420546E53C0E6FF54C022
:100E7000E6FF68ECD2F0E7CF54F0E552E7CF53F04D
:100E80005350F324516E5450F420526E51C0E6FF7B
:100E900052C0E6FF68ECD2F0E7CF52F0E552E7CF60
:100EA00051F05150F3244F6E5250F420506E4FC009
:100EB000E6FF50C0E6FF68ECD2F0E7CF50F0E55215
:100EC000E7CF4FF0B4ECCFF068ECD2F0E7CF4EF0C4
:100ED000E552E7CF4DF0BCECD3F074ECD4F068EC05
:100EE000D2F0E7CF4CF0E552E7CF4BF06BECCBF014
:100EF000030E0F0B03E094ECD0F0FDE152ECD0F0C8
:100F00000101E7AD58D0AA0EE66EE20EE66E010EC4
:100F100012ECCAF0020EDBCFD8F1030EDBCFD9F111
:100F200001017F0ED880D855050ED95505E207017D
:100F3000090E1FECD7F03FD047ECD4F0070E7CEC45
:100F4000D0F0FDE16A0E4924096ED8C149F080EC69
:100F5000D8F0FF0E005C2EE1010EDB50CDECD0F09E
:100F6000012ADF50CDECD0F001012A0E1C6FA50E36
:100F7000E66EE20EE66E010E48ECCAF0020EDBCF22
:100F8000E6FF030EDBCFE6FFD1ECD4F0A10EE66E58
:100F9000E20EE66E010E48ECCAF0DECFE6FFDDCFD2
:100FA000E6FFD1ECD4F09A0EE66EE20EE66E010E8C
:100FB00048ECCAF0096A25822AD069C11DF16AC1CC
:100FC0001EF16BC11FF16CC120F10A0E45ECD8F087
:100FD0001DC13BF01EC13CF01FC13DF020C13EF0E1
:100FE0002FECFDF03BC01DF13CC01EF13DC01FF1D8
:100FF0003EC020F1BDECE1F0E7ECE1F00101118F22
:10100000148F0701BEBB03D00101100E156F2E888F
:101010000490190E0101B95D06E138BF048083EC2C
:10102000D9F0800EA66F100E0101B95D09E13E51A5
:1010300001E004801BECD1F03E0EA46F010EA56F01
:10104000090E0101B95D0AE196BD04801BECD1F0E7
:10105000960EA46F010EA56F400EA66F310E010112
:10106000B95D22E136AD15D08EECDBF0930EE66E65
:10107000E20EE66E010E08ECCAF001013651070BD4
:10108000050DF3500A0F006E58ECD8F0C3ECD3F006
:1010900004D036BF0480C9EC80F00201360EA46F84
:1010A000010EA56FC70EA66F280E0101B95D06E1FE
:1010B00038B5048083ECD9F0040EA66F400E010110
:1010C000B95D0AE137B104801BECD1F0370EA46F93
:1010D000010EA56F010EA66F0C0E0101B95D23E193
:1010E000845106E1050E006F0B0E75ECCDF015D0A6
:1010F0008EECDBF00101840506E18A0EE66EE20E5D
:10110000E66E010E08D0020E845D07E1810EE66EE8
:10111000E20EE66E010E08ECCAF00201840EA46F26
:10112000010EA56F2E88170E0101B95D13E1050EA2
:10113000006F0E0E006E3BA904D04B0E006E040E25
:10114000006F02013B0EA46F010EA56F100EA66F7B
:10115000BDEC80F01F0E0101B95D23E156A50BD057
:10116000006B780EE66EE20EE66E010E08ECCAF039
:101170000101148F0ED056A108D0740EE66EE20E57
:10118000E66E010E08ECCAF004D00E0E006E10ECF4
:1011900026F00201560EA46F010EA56F050EA66F74
:1011A0002E800101B95106E133B40480C9EC80F00E
:1011B0002E88328A020E0101B95D4FE1006B6B0E81
:1011C000E66EE20EE66E010E08ECCAF00101006B5D
:1011D000800507E1620EE66EE20EE66E010E08EC97
:1011E000CAF0020E0101805D07E1590EE66EE20EC3
:1011F000E66E010E08ECCAF0030E0101805D07E106
:10120000500EE66EE20EE66E010E08ECCAF0040E19
:101210000101805D07E1470EE66EE20EE66E010E0B
:1012200008ECCAF0050E0101805D07E13E0EE66E96
:10123000E20EE66E010E08ECCAF0060E0101805DBA
:1012400007E1350EE66EE20EE66E010E08ECCAF01E
:101250000201800EA46F010EA56F0E0E0101B95D93
:101260003FE1835106E1010E006F440E75ECCDF0B5
:1012700032D083050DE1010E006F2D0EE66EE20EF9
:10128000E66E010EE66E1EECE2F0E552E55206D087
:1012900033AC06D0010EE66ED2ECE4F0E5521BD082
:1012A000030E006F270EE66EE20EE66E010E08ECEE
:1012B000CAF001018305040DF350006E58ECD8F01C
:1012C0005AECFEF03EC011F13AC012F10101115189
:1012D00002E1100E116F0201830EA46F010EA56FC3
:1012E0002D0E0101B95D12E10B0E006E04902AB3C0
:1012F000048004B004D0010E006F440E006EBDECFB
:1013000080F00201CCECD4F0020EA66F2F0E01018A
:10131000B95D0DE10B0E006E5FAF02D0CF0E006E17
:10132000BDEC80F0D0ECD1F0800EA66F2E88320E8E
:101330000101B95D08E12AB504801BECD1F0CCECC9
:10134000D4F0040EA66F0101040E006F1E0EB95DED
:101350000DE1050E006F020178B904801BECD1F09D
:10136000780EA46F020EA56F100EA66F220E01015B
:10137000B95D17E18DA908D0050E006FDE0EE66E8F
:10138000E20EE66E010E06D0006B1E0EE66EE20E59
:10139000E66E010E08ECCAF0CAECD1F0800EA66F22
:1013A0002E801A0E0101B95D3CE18EECDBF0110ECE
:1013B0000201702578ECCCF001010E6F140E0201D1
:1013C000702578ECCCF001010F6F0E6A0F6A0201F4
:1013D000705103E1C9ECCEF014D0700506E176EC53
:1013E00020F00101200E106F0CD0020E705D09E19B
:1013F000D6ECD4F00101395104E0EFC90EF0F0C988
:101400000FF00E0ED8800E54270E0F5402E20E6A13
:101410000F6A8EECCFF00101115102E1100E116F35
:10142000148F0A0EB95D19E1395103E0D9EC0BF0C4
:1014300014D0030E006F180EE66EE20EE66E010E7B
:1014400008ECCAF001015FA702D0020E156F328AC4
:101450002E80D0ECD1F0080EA66F0B0E0101B95D05
:1014600060E1395120E030A213D0040E006F090171
:10147000E85102E12A0E0FD0E80508E1130EE66EEE
:10148000E20EE66E010E08ECCAF008D04B0E03D057
:10149000010E006F440E006E10EC26F00201E80E03
:1014A000A46F090E3DD05AECBCF024ECD3F03A51B5
:1014B00002E1440E0CD03A0504E1040E006F2A0E3E
:1014C00006D0020E3A5D06E1040E006F4B0E75EC7D
:1014D000CDF020D0030E3A5D1DE33A5113081AE314
:1014E000550E75ECCDF0030E01013A5D006E080E4D
:1014F000005C04E21C0E146F00280BD0100E005C80
:1015000005E2130E146F070E005C03D0130E146F68
:10151000240E156F328A2E8002013A0EA46F010E3E
:10152000A56F210E0101B95D17E1395102E10E0EDF
:1015300003D0390504E1080E75ECCDF008D0006B3E
:101540000A0EE66EE20EE66E010E08ECCAF002012B
:10155000390EA46F010EA56F1B0E0101B95D3BE1B1
:101560002EA435D0016A1E0E015C0AE2CAECD3F04B
:10157000EF50E66ED1ECD3F07DECCCF0012AF3D73E
:101580009BECE2F0EFECE0F00101279D269D175067
:10159000800B0CE101012651400B08E12751400B63
:1015A00005E1A6EC53F0EBEC41F0F1D7016A1E0E19
:1015B000015C0AE2D1ECD3F0EF50E66ECAECD3F056
:1015C0007DECCCF0012AF3D7EFECE0F00101050E41
:1015D000F3ECD9F0328A300E0101B95D42E1050E1B
:1015E000F3ECD9F02EA23BD024ECD3F02F0E75EC07
:1015F000CDF08250010B03E08250020B0DE18EEC26
:10160000DBF00101010E106F82B202D0040E106FE8
:10161000050E006F006A1DD0066A060E065C1EE20B
:101620000650040DF3508309006E050E065C02E1BE
:10163000BB0E006E00501CECDAF01A080DE2F00E42
:10164000005C0AE28EECDBF006C010F10101050E31
:10165000006F80ECE1F002D0062ADFD725822E88C9
:10166000328A33ECD5F061E1D5CA03F0D251010BD7
:1016700010E03751080B0DE0040E036E1BA009D0DB
:10168000030E036E0A011C5104E1280E216F21CACA
:101690001CFA0201D65119E00101170E0E6F010E5E
:1016A000006F035064ECCFF0EF50B9ECCEF00101C5
:1016B000200E126F050E006F03506AECCFF0EF5052
:1016C000B9ECCEF00101128F2FD08EECDBF00501CA
:1016D000170506E1050EE66EE20EE66E010E05D078
:1016E000FF0EE66EE10EE66E010E08ECCAF01BA0DE
:1016F00009D024ECD3F0FA0EE66EE10EE66E010E90
:1017000008ECCAF005011751050D23ECD6F0140EB4
:1017100049260A0E4A220350B2ECD8F027ECCEF04C
:10172000135102E1100E136F2E883C0EB95D27E1B4
:101730008EECDBF022B406D0050EE66EE20EE66E0D
:10174000010E05D0FF0EE66EE10EE66E010E08EC0E
:10175000CAF02250040B01E0010E0201A46FA56B38
:10176000910EA427020EA52344ECD7F0EF50006E93
:1017700027ECCEF0135102E1100E136F2E880F0EDE
:10178000B95D1DE1050E006F51C100F080ECE1F084
:101790000101158F135102E1100E136F0601426B08
:1017A0000101515102010B5D05E20601700E426F0D
:1017B0005A0E436F0201510EA46F010EA56F290E40
:1017C0000101B95D0AE1775101E004801BECD1F021
:1017D000770EA46F010EA56F2E88260E0101B95D4C
:1017E0001AE1020E006F1E0E4325EBECD9F0010149
:1017F000006B1A0E4325EBECD9F00101136B100EB0
:10180000146F120E156F0E5102E1100E0E6F0F5174
:1018100002E1100E0F6F3E0EB95D17E1050E006F6D
:10182000420506E1F60EE66EE10EE66E010E05D00B
:10183000F20EE66EE10EE66E010E08ECCAF0020151
:10184000420EA46F010EA56F2E80140E0101B95D2A
:101850001BE14FA305D0040E006FB9ECD8F00DD0FA
:10186000006B640E75ECCDF05D0E006E01014FA1B2
:1018700002D0600E006E10EC26F002014F0EA46F35
:10188000010EA56F030EA66F150E0101B95D1EE1D5
:10189000040E006F4FBB11D01C0E0E6F160E0F6F93
:1018A000240E106F0D0E116F5D0E006E4FA902D049
:1018B000600E006E10EC26F002D0B9ECD8F00201F8
:1018C0004F0EA46F010EA56F300EA66F330E0101EF
:1018D000B95D02E123ECE4F0080E0101B95D1DE100
:1018E0008EECDBF001015FB90480C9EC80F08CEC78
:1018F000CAF083C33EF05AECFEF03EC012F13AC08B
:1019000013F18CECCAF084C33EF0C3ECD3F00101B8
:10191000148FD0ECD1F0100EA66F5CC305F005500B
:101920002EECCFF07CECD8F0440EB95D0BE1140E38
:10193000006E65ECDBF002E0110E006EBDEC80F095
:10194000328A2E88450E0101B95D14E132ECD7F0E0
:10195000496E4A6A40ECD8F0640D17ECCDF0030EE6
:10196000006F9CEC26F0060EE66E030E88ECCFF0BE
:10197000328A2E88460E0101B95D07E13BECD8F0B2
:10198000006E6EEC80F0328A2E88480E0101B95D3F
:1019900012E1CAECD9F0006E040E2EECD4F0100E59
:1019A000126FD4ECD9F002E10E0E126FCFECD9F029
:1019B000156F148F2E88470EB95D1FE1AEECD6F07F
:1019C00006E11BECCAF0D8ECD3F00A0803E11BECEB
:1019D000CAF0EF921BECCAF0060EEB50006E0050FE
:1019E00001E1002A80ECE1F00101135102E1100E47
:1019F000136F180E126F158F2E88490EB95D1DE1F9
:101A00001BECCAF0D8ECD3F0006E240E126F220E3D
:101A1000136F1E0E146FAEECD6F008E0010E0E6FC1
:101A20001E0E0F6F240E106F118F04D0005002E1B4
:101A30000528006E00C015F12E88129E129C2E50B3
:101A4000100B07E01E50040B04E11B50080B01E1D2
:101A5000128C200EB95D03E01C0EB95D05E1060E87
:101A6000E66E050E88ECCFF02A0E0101B95D08E1A3
:101A7000135106E1100E136F145102E1100E146F92
:101A8000040EE15C02E2E16AE552E16EE3EFC9F0C7
:101A900063ECD5F00101B951DE6EDD6A5AECCEF08F
:101AA000070EEC02F3CFEDFFEF02F3CFEEFFF450A1
:101AB000ED26026AF80E496ED60E4A6E010E4B6E86
:101AC0000250E76E000EDFCF4CF0010EDBCF4DF081
:101AD000E7504C26000E4D22EAECD5F0F550006E92
:101AE0002EECE2F0022A070E025CE4E3020EE15C57
:101AF00002E2E16AE552E16EE3EFC9F01200020191
:101B0000030E686FA46BA56BA6691996F8ECD2F06A
:101B100004E1E79DE79BC6EC0AF00601426BA5ECE9
:101B2000DFF024B8C2D820ECD3F003E03C0EB95D5E
:101B300006E12050040B03E0209455ECCEF082EC3B
:101B400009F02DA454D02D940E0E0101B95D1DE1B4
:101B5000339C83C100F00050010813E20004E66EDC
:101B600049ECE4F0E552338CC80E16ECCAF0E66A94
:101B7000D2ECE4F0E552000908E00201020E686FC1
:101B800004D0E66A49ECE4F0E5521EA602D0FCEC73
:101B900035F01E963BEC0EF04EEC0EF024A405D072
:101BA00076ECCFF0249425ECD4F01EA80BD01E9830
:101BB0000DC1E6FFDBEC5AF0E5520DC1E6FFF7EC94
:101BC0005AF0E5522EA60ED02E96D8EC5BF073ECB0
:101BD000CEF008E22DECCDF020ECCFF09EEC21F021
:101BE000ABEC2EF030AE03D0309E20EC78F018AC89
:101BF00003D0189CC8ECD4F01E941200BCEC0CF07E
:101C000029920201355101E1258AB5EC16F02E9496
:101C10002E920FEC0DF00601426B0101B593A5EC7D
:101C2000DFF0AFEC6FF02D9C0201686B0C0E076EBD
:101C30002AEC64F00101129C3B51010B01E0128C73
:101C4000129E3B51020B01E0128E17A004D0E66AEF
:101C50004D0E78ECCAF09C0E52ECCAF00101E79DE3
:101C6000E79B12000D500101B927B9AF02D0490E10
:101C7000B96FB951490801E2B96B1200230E00ECAB
:101C8000CBF0020E006E1A0E155C05E1005089ECD7
:101C9000CBF0320EEF6E12000101AE6BD890AC3378
:101CA000D890AC332896F1EFCDF007010B9FBCEC38
:101CB000C4F0AAECD7F0209C3386BBECD4F0249877
:101CC0002AECCFF0B2EF69F0E66AE66A5FECCEF09C
:101CD0000701086BF6ECC4F0BCEC16F08A96208C79
:101CE0003396BBECD4F007010B8FBCEFC4F0E7ECEC
:101CF000C9F0100EE1263250200B14E01D50040BE9
:101D000002E1A0EF96F01D50080B02E1A0EF96F063
:101D10003FECCDF002E1A0EF96F00FECD1F002E045
:101D2000A0EF96F002016851030A02E19EEF96F0DF
:101D3000010A1DE0030A02E0A0EF96F02D942E9018
:101D400024982E98329A189C0101B5830201A46B45
:101D5000A56BA669199669ECE3F01F960101269D13
:101D6000279D0201020E686F258297EC3DF02950F5
:101D7000020B16E02E50010B13E02E50100B10E159
:101D80006AEC7AF029922F88D8EC80F00101B58DA9
:101D9000B58F640EAC6F1EEC79F0B1DE57C2B9F1AD
:101DA00017AE3AEF96F093ECCFF0E5EC14F0FF08A5
:101DB00013E000EC15F0006E0101395105E01B0E37
:101DC000005C02E1C0ECD8F00101B59BB599179E0B
:101DD0002582238AA0EF96F02E50100B12E01E50A1
:101DE000040B0FE11B50080B0CE1090E155C09E018
:101DF0000C0E155C03E11750100B03E1F5EC08F035
:101E000004D00B0E155C04E17ADE179EA0EF96F06D
:101E100017A0DCEF94F028B6E0EF94F0090E155C03
:101E200002E1E6EF94F0A1ECCBF075E01750010B66
:101E300072E0100E155C09E0110E155C06E0080E4C
:101E4000155C03E0290E155C66E11550DF6E91C24A
:101E5000F9F692C2FAF68DC2F5F68EC2F6F68FC288
